:1000000000000220657D00008D7D00008F7D0000D6
:10001000917D0000937D0000957D000000000000B0
:10002000000000000000000000000000977D0000BC
:10003000997D0000000000009B7D00009D7D000078
:100040009F7D000051560000298100009D7C00002A
:10005000917C00009F7D00009F7D00009F7D00003F
:100060009D3700009F7D00009F7D00009F7D000068
:100070009F7D00009F7D00009F7D00009F7D000010
:100080009F7D0000AD8100009F7D00009F7D0000EE
:100090009F7D00009F7D00009F7D00009F7D0000F0
:1000A0009F7D00009F7D00009F7D00009F7D0000E0
:1000B0009F7D00009F7D0000000000000000000008
:1000C0009F7D00009F7D00009F7D00009F7D0000C0
:1000D0009F7D00009F7D00009F7D00009F7D0000B0
:1000E0009F7D0000000000000000000000000000F4
:1000F000000000009F7D0000000000009F7D0000C8
:1001000000000000000000000000000000000000EF
:1001100000000000000000000000000000000000DF
:1001200000000000000000000000000000000000CF
:1001300000000000000000000000000000000000BF
:1001400000000000000000000000000000000000AF
:10015000000000000000000000000000000000009F
:10016000000000000000000000000000000000008F
:10017000000000000000000000000000000000007F
:10018000000000000000000000000000000000006F
:10019000000000000000000000000000000000005F
:1001A000000000000000000000000000000000004F
:1001B000000000000000000000000000000000003F
:1001C000000000000000000000000000000000002F
:1001D000000000000000000000000000000000001F
:1001E000000000000000000000000000000000000F
:1001F00000000000000000000000000000000000FF
:1002000010B5054C237833B9044B13B10448AFF350
:1002100000800123237010BD440200200000000074
:10022000A4D6000008B5034B1BB103490348AFF344
:10023000008008BD0000000048020020A4D6000095
:10024000154B002B08BF134B9D46A3F5803A0021A8
:100250008B460F461348144A121A0AF029FA0F4B1C
:10026000002B00D098470E4B002B00D09847002061
:10027000002104000D000D48002802D00C48AFF307
:1002800000800AF0CDF92000290007F0A5FF0AF050
:10029000A1F900BF000008000000022000000000DB
:1002A00000000000440200208C90012000000000AB
:1002B0000000000010F0010310D104280CD90368DD
:1002C000C3F30F1343B1013B9B001A1DC1180979F9
:1002D00011B101339342F9D1184670470023FBE76F
:1002E000037883B11A0601D40130704703F0C003CC
:1002F000C02B08BF0130024610460132037803F0DC
:10030000C003802BF8D0704708B5002103780BB9E3
:10031000084608BDFFF7E4FF0131F7E738B50022D2
:1003200004460D46411C092003F06CFD40B16300FA
:10033000024643F0010342F8043F0023A34200DBDE
:1003400038BD55F8231042F8041F0133F6E70128A1
:1003500038B504DC1C20BDE8384001F0A3B90D68B5
:10036000EA0701D41120F6E74868C30706D4042839
:1003700004D9036803F00F03042B01D00E20EAE731
:1003800003F0A4FB6D10002D044603DDFFF7BCFF56
:10039000A84206DA1220DEE72046FFF7A1FF013D62
:1003A0000446012DF8D120787F2808DDDF280ADCFB
:1003B0006378800100F4F86003F03F0318434000C5
:1003C00040F0010038BDEF280ADC637800039B0190
:1003D00080B203F47C630343A07800F03F00EDE7B4
:1003E000F72810DC637880041B0303F47C3300F4EB
:1003F000E0101843E37803F03F030343A078800143
:1004000000F47C60DAE74FF0FF30D8E7486838B591
:10041000C3070D4606D4042804D9036803F00F026D
:10042000092A04D00B20BDE8384001F03BB94468EC
:10043000C3F30F1364105A1EA2420BD8032194FB7E
:10044000F1F16429A8BF64210329ACBF5918D91C54
:1004500003F014FD0368C3F30F13013B9C4208D261
:10046000A31C013464002A6840F8232044F00104EE
:100470004460002038BD01282DE9F84304DC1C202D
:10048000BDE8F84301F00EB902284E680CD08C6824
:10049000E70709D56410012CB8BF0124F50705D57D
:1004A0004FF0FF30BDE8F8830124F7E7042EF7D9B9
:1004B00033680D6803F00F02042A30D1E80706D430
:1004C000042D04D92B6803F00F03042B01D00E2058
:1004D000D6E73046FFF7EEFEA042E1DB304603F000
:1004E000F5FA0646284603F0F1FA03780146002B98
:1004F000D6D0601E30440AF0AAFC01460028CFD0B6
:10050000012433780BB18E4203D3640044F0010020
:10051000C8E73046FFF7E4FE01340646F1E7092A52
:1005200038D177687F10BC42BADCE90729D4042DA2
:1005300027D92B6803F00F03042B22D1284603F0A0
:10054000C5FA804604F1010956F82900854203D115
:10055000600040F00100A5E7C2070ED404280CD9C2
:10056000036803F00F03042B07D103F0AFFA014631
:1005700040460AF033FC0028C7D0B9454C46E1DDBF
:100580008EE7631C56F82320AA42BED0BB421C460D
:10059000F7DD85E7032A83D1C3F30F17C3F3417354
:1005A000C3EB8707BC423FF77BAFEB0728D4042D92
:1005B00026D9286800F00F03032B17D1C0F30F13BF
:1005C000C0F3417005F10408C0EB83003F1A013C01
:1005D00040440336BC423FF763AF3219434683427F
:1005E00019460FD315D1601C4000B2E7042B07D188
:1005F000284603F06BFA80462846FFF75BFEE5E7E6
:100600000F203DE712F8015F09788D4203F10103E5
:10061000E5D00134DEE7000001282DE9F0478A46E5
:1006200004DC1C20BDE8F04701F03CB80868C307B3
:1006300006D4042804D9036803F00F03042B01D067
:100640000E20EFE74B6813F00106F9D1042BF7D920
:100650001B6803F00F03042BF2D103F037FA0446B2
:10066000DAF8040003F032FA81460AF0C1FB804652
:100670002046B8F1000F16D1FFF746FE05460122CD
:10068000A918092003F0BEFB324F386068B900207A
:10069000BDE8F087494640440AF0D9FB3D466F1C4F
:1006A0000028F7D1EBE73546F9E76B0043F001038B
:1006B0004360B8F1000F18D12046FFF711FEB54294
:1006C000804601DC3868E3E7A8EB0401204603F02C
:1006D0001AFC0028DBD0B21C3B6843F822004046DD
:1006E000FFF7FEFD01364446E9E7012D03D1DAF8B4
:1006F00000308360CCE74946601C0AF0A8FB012665
:100700008246BAF1000F14D0B542DBDBAAEB04013C
:10071000204603F0F8FB0028B9D03B6801360AEB0D
:10072000080443F82600494620460AF090FB82461A
:10073000E7E7B542C6DB20460AF05AFB01462046F1
:1007400003F0E1FB0028A2D001363B6843F8260005
:10075000B8E700BF546D012008B503F09BF94000D5
:1007600040F0010008BDC30711D404280FD9026866
:1007700002F00F03032B0AD101F00303C3F10403BA
:100780005B0703F0C04322F0C0421343036070478D
:1007900001282DE9F0470546884604DC1C20BDE809
:1007A000F04700F07FBF4C6814F0010701D10D2025
:1007B000F5E7022802D08B68DA07F8D5D8F8006090
:1007C000F30700F1A980042E40F2A680326864107D
:1007D000012C02F00F03B8BF0124092B28D1766841
:1007E000022D4FEA660605D0D8F808305B109E420D
:1007F000A8BF1E46351B0135012225EAE575A9185B
:10080000092003F0FFFA074648B16D00034645F0A2
:100810000105D8F8002043F8045FA64202DA384602
:10082000BDE8F087013452F8241043F8041FF4E7C0
:10083000042B43D1304603F049F9FFF765FD022D43
:10084000824605D0D8F808305B109842A8BF9A4677
:10085000A24504DA0020BDE8F04703F04DBB304666
:1008600003F034F90546A74222DB304603F02EF9A7
:10087000A94606462846FFF733FD0134A245054642
:10088000F8DAA0EB0905284603F036FB07460028F6
:10089000C5D003F01BF90446D8F8000003F016F9A0
:1008A000A9EB060101442A46204609F0DDFEB6E721
:1008B0002846FFF715FD01370546D4E7032B2BD15A
:1008C000C2F30F13022DC2F34172C2EB830205D0B3
:1008D000D8F808305B109A42A8BF1A46A24206DA3E
:1008E000002211460320BDE8F04703F08BBA151B28
:1008F0000423291D002291FBF3F1032003F082FA67
:10090000074600288BD001352946FFF72CFFE11C54
:100910002A4631440430C8E7212040E70028F8B5D2
:1009200004DC1C20BDE8F84000F0BCBE0C6814F0EC
:10093000010711D06410FF2C01D91320F2E7002227
:100940000121032003F05EFA054618B10021FFF7EC
:100950000AFF04712846F8BD042CEED9256805F07D
:100960000F05042D19D12046FFF7A4FC3A46C11CFF
:10097000064691FBF5F1032003F044FA05460028F2
:10098000E8D03146FFF7EFFE204603F09FF83246ED
:100990000146281D09F068FEDCE7092D1DD16668B7
:1009A00076100423F11C3A4691FBF3F1032003F087
:1009B00029FA05460028CDD03146FFF7D4FE04348D
:1009C000B742C7DA54F8043FDA0704D55B10FF2BAF
:1009D000B3D8EA1913710137F2E7032DADD12546DB
:1009E000B8E77F2902DC017001307047B1F5006F74
:1009F0000CDA03468A1162F03F0203F8022B01F081
:100A00003F0161F07F01417018467047B1F5803FAA
:100A10000FDA0B1363F01F030370C1F3851301F0AA
:100A20003F0163F07F0361F07F0143708170033009
:100A30007047B1F5883F0DDAF023037090234370BF
:100A40008B1101F03F0163F07F0361F07F01837040
:100A5000C1700430704700000028F7B50F4603DC72
:100A60001C2000F01FFE0CE00A6812F001000AD002
:100A70006C4651102046FFF7B4FF011B204603F0DF
:100A800042FA044616E0042A3BD9136803F00F0328
:100A9000092B36D155681C496D100124AC420CDD80
:100AA00003F02AFA044628B13F6803F00FF8012644
:100AB000AE421DDD204603B0F0BD013452F82430B3
:100AC00013F0010601D10D20CBE75B107F2B09DD70
:100AD000B3F5006F08DBB3F5803F07DB8B42D4BF73
:100AE000042600263044D9E70226FBE70326F9E76F
:100AF000013657F82610CB07E5D54910FFF771FFEF
:100B0000D6E72120ADE700BFFF0F0100002838B570
:100B100004DC1C20BDE8384000F0C4BD0C68E307CD
:100B200001D40D20F6E7641024EAE474E11C0022ED
:100B30008910032003F066F9054610B12146FFF73E
:100B400012FE284638BD10B5044611F0010011D13F
:100B500004290ED90B6803F00F03042B09D10846B2
:100B600002F0B4FF014620460AF038F9B0FA80F0EE
:100B7000400910BD0020FCE70128F8B50E4604DC52
:100B80001C20BDE8F84000F08DBD4D6815F0010750
:100B900006D1042D04D92B6803F00F02092A01D0D5
:100BA0000B20EEE76C6809681F486410C3F30F134D
:100BB000A34298BF03F1FF34FFF7C5FF40B1012303
:100BC000BC4201DA0020F8BD013745F82730F7E7CD
:100BD00031681648FFF7B7FF50B1002CF2D0631C04
:100BE0000122013C944045F8232014436C60E9E75E
:100BF0003368DA0701D40D20C3E75B10002B0DDD4D
:100C00009C420BDB05EB830305EB84029A4207D180
:100C10000123013C9C4053601C43E7E71220B0E7EE
:100C2000996843F8041FF1E767BD00006BBD000041
:100C3000002310B50B70C3070C4606D50E494210B1
:100C40002046BDE810400AF08DB828B90B4920466F
:100C5000BDE810400AF0A6B8042801D10849F6E71B
:100C600009D9036803F00F03042B04D102F02EFF0F
:100C700004490246E4E710BD44C8000070BD00000E
:100C800076BD00007BBD00002DE9F04301288FB048
:100C900081460E4607DC1C2000F004FD0546284670
:100CA0000FB0BDE8F0830B6813F0010440F0A180A1
:100CB000042B40F2D5801B6803F00F03092B40D1B1
:100CC000274656F8273013F0010806D1042B04D923
:100CD000186800F00F00092801D02220DCE75B68CB
:100CE0000137B94504EB6304EBD10122A11803F0ED
:100CF00089F8054608B90025D1E7640044F00104ED
:100D00004460424600F1080456F822104B68086817
:100D10005B10C0F30F10984298BF00F1FF3304310D
:100D20000020834207DC013223EAE373BA4204EB7A
:100D30008304E9DBB3E751F804CF44F820C0013065
:100D4000EFE7032B40F08C80274656F8270010F081
:100D50000108C2D10428C0D9036803F00F02032A96
:100D600038D1C3F30F12C3F34173C3EB82031C44A6
:100D70000137B945E9D10423E11C002291FBF3F1CD
:100D8000032003F03FF805460028B4D02146FFF7C2
:100D9000EAFC00F1040956F82840E10720D4042CAD
:100DA0001ED9206800F00F03032B19D1C0F30F13D5
:100DB000C0F34170C0EB830003344B46A3EB090240
:100DC000824211DB08F101080028A8BF8144B84520
:100DD000E1DB64E7042A80D1FFF76CFA0444C7E73B
:100DE0002046FFF767FAE7E714F8012F03F8012B15
:100DF000E4E700252C4656F82500C20732D4042823
:100E000030D9036803F00F02042A32D1FFF752FAF7
:100E100004440135A945EED1204603F06DF805469E
:100E200000283FF468AF041DB04606EB890958F866
:100E3000046BF30728D4042E26D9336803F00F027D
:100E4000042A34D13046FFF735FA0746304602F01F
:100E50003DFE3A460146204609F006FC3C4421E0AE
:100E60002546C8E701A9FFF7E3FE01A809F0C0FF86
:100E7000CEE7032A7FF431AFC3F30F12C3F34173FC
:100E8000C3EB82031C44C4E701A93046FFF7D0FE40
:100E900001A809F0ADFF01A906460246204609F067
:100EA000E3FB3444C145C2D100232370F7E6032A93
:100EB000F8D1C3F30F17C3F34173C3EB87073A4667
:100EC000311DC8E72DE9F04F002893B00F4607DC2D
:100ED0001C2000F0E7FB0546284613B0BDE8F08F64
:100EE0000D6815F0010806D1042D04D92B6803F014
:100EF0000F03092B01D00B20EBE76E687610002E54
:100F000003DC404602F0F8FFE5E7012826D04868F8
:100F1000C20723D4042821D9036803F00F03042B4C
:100F20001CD102F0D3FD0446204609F061FF0435D0
:100F3000731E8146009303FB00FB05EB860A55F800
:100F4000040FC30771D404286FD9036803F00F029C
:100F5000042A05D1FFF7AEF983440AE0384CE3E7F1
:100F6000032A69D1C3F30F12C3F34173C3EB8203A6
:100F70009B44AA45E3D1584602F0BEFF054600282F
:100F8000AAD0D7F800A0B9F1000F03D0786802F01A
:100F90009DFD0446284602F099FD0AF10403074628
:100FA0000193019B53F804AF0193504602F08EFD6C
:100FB0001AF001030146029302D1BAF1040F04D8DA
:100FC00005A95046FFF734FE05A90846039109F02C
:100FD0000FFFDDE9023183468BB9BAF1040F0ED958
:100FE000DAF8000000F00F0CBCF1030F01BFC0F3F2
:100FF0000F13C0F341700AF10401C0EB830B3846B4
:101000005A4609F031FB5F44B9F1000F08D0009B4C
:10101000434505DD38464A46214609F025FB4F4445
:1010200008F101084645BCD156E705A9FFF700FEC7
:1010300005A809F0DDFE8FE702F048FDF9E700BFE3
:1010400032C20000002810B511DD0B6813F0010456
:1010500002D05C1024EAE4740122A118092002F0F5
:10106000D1FE18B1640044F00104446010BD0024B6
:10107000F2E70A6838B512F0010436D1042A34D9EF
:101080001368496803F00F00092818D15068C3F3AA
:101090000F134010834298BF03F1FF30151DA0428B
:1010A00005DC01330220984205DB002038BD45F8FD
:1010B000041F0134F3E742F820100130F3E703285E
:1010C00013D1C80704D41320BDE8384000F0EABAB1
:1010D0004910FF29F7D80432C3F30F1302EB83033F
:1010E0009A42E2D202F8011BFAE70B2000F0DAFA8A
:1010F000DBE700002DE9F0414E6816F00107884655
:1011000028D1042E26D9346804F00F03092B11D1FD
:101110007568C4F30F146D10AC4200D8651ED8F882
:101120000010CB071AD54C10002C01DDA54220DAA7
:10113000122034E0042B04D13046FFF7BBF80546FB
:10114000EDE7032B08D1C4F30F15C4F34174C4EBCE
:101150008505E4E70025E2E73D46E0E72848FFF79C
:10116000F2FCA8B109F096FD90FBF5F404FB150420
:101170000134002F41D1042E3FD9336803F00F030F
:10118000092B12D1013456F824402046BDE8F081E5
:10119000D8F800101B48FFF7D6FC20B91120BDE895
:1011A000F04100F07FBA2C46E3E7042B1DD1304616
:1011B00002F08CFC012C05460FDCFFF791F8461B72
:1011C000304602F099FE04460028DED002F07EFC94
:1011D0003246294609F048FAD7E72B78013C002B24
:1011E000A6D02846FFF77CF8E4E7032B05D134446A
:1011F000E478640044F00104C7E70B20CFE700BFA8
:1012000060BD00006BBD00002DE9F0414C6814F09A
:10121000010688462ED1042C2CD923688F6803F050
:101220000F02092A13D16568C3F30F136D10AB4287
:1012300000D85D1ED8F800102848FFF784FC68B37A
:10124000236803F00F03092B1ED1012317E0032AA3
:1012500010D1FA0704D41320BDE8F04100F022BAFF
:101260007E10FF2EF7D8C3F30F15C3F34173C3EB02
:101270008505DFE70B20EFE7013344F823709D423B
:10128000FADA0020BDE8F081032BFAD10334012300
:101290009D42F6DB04F8016F0133F9E7D8F800103E
:1012A000CB0706D54910002901DD8D4208DA12204E
:1012B000D2E70B48FFF747FC08B91120CCE72946D5
:1012C000236803F00F03092B03D1013144F8217087
:1012D000D7E7032B04BF6418E670D2E767BD0000B0
:1012E0006BBD0000086808B5C3071BD4042819D9D2
:1012F000036803F00F02092A01D1406808BD032AE0
:1013000009D1C3F30F12C3F34170C0EB8200400058
:1013100040F00100F2E7042A04D102F0D7FBFEF707
:10132000F3FFF4E70120E9E7024A03480D2104F046
:1013300059BA00BFF8BC0000F0BC000000207047A4
:101340000420704701207047002002F0D5BD002026
:101350007047002070470020704700207047002031
:101360007047002070470020704700207047000041
:10137000024A03480C2104F035BA00BF00BE000049
:1013800060BE00007047037883B11A0601D40130B3
:10139000704703F0C003C02B08BF0130024610465F
:1013A0000132037803F0C003802BF8D070470000AF
:1013B000F8B511F0010506461446084626D1042961
:1013C0003FD90B6803F00F03042B3AD1D30714D491
:1013D000042A36D9136803F00F03042B31D102F02D
:1013E00075FB0546204602F071FB0146284609F0D0
:1013F000F5FC00282DDB1ED126E002F067FB294614
:101400000A2209F0B9FD0546601011E012F001074B
:1014100015D1042A15D9136803F00F03042B10D13A
:1014200010464D1002F052FB0A22394609F0A4FD85
:1014300085420EDB08DD002E09DC00200CE04D109B
:10144000E2E7064B0F221A700136022EF5D804206F
:1014500002E0701700F00400F8BD00BF8402002015
:101460002DE9F0412B4F06460024E500EB191B79CE
:10147000032B07D00134FF2CF7D14FF0FF34204667
:10148000BDE8F081304609F0B3FC31460246E0B2D7
:1014900004F0E6F90028F2D1EB5959681A1D884288
:1014A000E8D052F8045FF02D00F10100F7D1800080
:1014B00008301A18D107DDD4042ADBD91B5803F0F1
:1014C0000F010429D6D1C3F30F13013302EB8300BC
:1014D000C507CFD40428CDD952F8233003F00F0329
:1014E000042BC7D102F0F2FA4FF003080546092198
:1014F000284609F066FC0028BCD0B8F1010800F1CC
:101500000105F4D13146284609F0A1FC8542B6D048
:10151000B0E700BF6086012010B510F0010402D0D2
:101520004410204610BD042812D9026802F00F02B0
:10153000042A07D102F0CAFA0A222146BDE8104067
:1015400009F01ABD032A03D10A2221460430F5E727
:10155000014B0D221A70E4E78402002010F0010212
:1015600010B516D1042802D90268C2F30F1211F087
:10157000010310D1042902D90B68C3F30F1393425E
:1015800016D1043000EB83020331904205D30120D1
:101590000BE00022EBE70023F1E710F8014B11F814
:1015A000013F1CB9B3FA83F0400910BD9C42ECD056
:1015B0000020FAE72DE9F74F804689469A46304FDA
:1015C000304E6AB102233B70012333603368DFF889
:1015D000D0B00024FC54444504DB03B0BDE8F08FD8
:1015E0003260F3E759F824003168C30707EB0105BF
:1015F000C1F5487105D5244A4310284609F07EFB01
:1016000004E0C8B9214A284609F078FB1C4809F0D3
:10161000EFFB3060BAF1000F0CD008F1FF33A342AA
:1016200008DDB0F5487F05D2431C20223A54002241
:10163000FA5433600134CEE7042801D1144AE2E7BA
:101640001BD9026802F00F03042B06D1019102F0AE
:101650003DFA104A01990346CFE7092B03D14368AD
:101660005A465B10C9E7032B08D1C2F30F13C2F32C
:101670004172C2EB8303084ABFE70123074ABCE774
:1016800085020020A805002044C8000070BD0000AD
:1016900076BD00006FCE0000DFC00000EAC0000091
:1016A000D0C00000014B1870002070478402002059
:1016B00010B501F00DFF084C231D01461F221846EE
:1016C00009F0B0FB09F094FB04308008000140F001
:1016D00004002060204610BD600200202DE9F04F7C
:1016E00085B000F1180104690291D0E90232824606
:1016F00001EB8404BC4F4169029800EB8109397801
:1017000003EB820529BB53F82230B84A1E1203F0BE
:101710007F03043552F82330904643F00103184705
:101720009AF8010004F0CCFC00238AF8003021E094
:101730003B7873B92B681E1203F07F03043558F809
:101740002330EAE7029A231D9A1AD82A26DD1A23A3
:101750003B70DAF808209AF8023039789AF80100DC
:10176000AA1A921043EA022204F0B0FC00238AF87D
:1017700000303B70DAF80830ED1A029BE41AA9EB4E
:101780000309AD10A4104FEAA903CAF80C50CAF817
:101790001040CAF8143005B0BDE8F08F22461C4650
:1017A0003B781660002BD4D12B681E1203F07F0308
:1017B000043558F82330B0E7029A231D9A1AD82A24
:1017C00002DD1A233B70C4E721461C462B680B60E0
:1017D0003B782A1D0BB11546BBE76B681E1203F060
:1017E0007F03083558F8233097E7029A231D9A1A89
:1017F000D82A02DD1A233B70ABE722461C463B7811
:1018000005EB86061660002BA3D12B681E1203F091
:101810007F03043558F823307FE7029A231D9A1A74
:10182000D82A02DD1A233B7093E722461C46704BF0
:1018300053F8263013603B78002B8AD12B681E1298
:1018400003F07F03043558F8233066E7684B54F8FB
:10185000042D43F826203B78002B7FF47AAF2B68C9
:101860001E1203F07F03043558F8233055E7DFF8E4
:1018700080B15BF82600FFF74FFE3A785AB9009026
:1018800054F8040DFFF748FE009B1844400040F058
:1018900001004BF826003B78002B7FF45AAF2B68F1
:1018A0001E1203F07F03043558F8233035E7029BFE
:1018B000221DD31AD82B02DD1A233B7049E7029B65
:1018C00021464B4534BF59F80C3C01230B603B7853
:1018D0001446002B7FF43DAF2B681E1203F07F03EC
:1018E000043558F8233018E7029B221DD31AD82B51
:1018F00002DD1A233B702CE7029B4B4518D259F8A6
:101900000C3C06F180465B10C3EB8373033E33440B
:1019100059F8233023603B781446002B7FF419AF2D
:101920002B681E1203F07F03043558F82330F4E6C9
:1019300018233B700023EDE7029B4B4518D259F862
:101940000C3C54F8042D5B1006F18046C3EB837306
:10195000033E334449F823203B78002B7FF4F9AE53
:101960002B681E1203F07F03043558F82330D4E6A9
:1019700018233B70F0E7029B4B4529D259F80C3CE9
:1019800006F180465B10033EC3EB8373334459F882
:101990002300FFF7C1FD834654F8040DFFF7BCFD9B
:1019A00059F80C3C5B10C3EB837358441E44400051
:1019B00040F0010049F826003B78002B7FF4C9AEC7
:1019C0002B681E1203F07F03043558F82330A4E679
:1019D00018233B70F0E7029A231D9A1AD82A09DDD2
:1019E0001A233B70B5E600BF84020020D0BE000081
:1019F000588E012022461C4659F8263013603B7849
:101A0000002B7FF4A6AE2B681E1203F07F03043573
:101A100058F8233081E654F8043D49F826303B78E5
:101A2000002B7FF496AE2B681E1203F07F03043563
:101A300058F8233071E659F826004FEA600B54F845
:101A4000040DFFF769FD584440003B7840F0010069
:101A500049F82600002B7FF47CAE2B681E1203F0A1
:101A60007F03043558F8233057E6029BA4EB860425
:101A7000A3420BD83B78002B7FF46BAE2B681E1271
:101A800003F07F03043558F8233046E6C24802F0DD
:101A90000DF83B78002B7FF45CAE2B681E1203F030
:101AA0007F03043558F8233037E6002E05EB860512
:101AB000FFF660AE3B78002B7FF44BAE2B681E1216
:101AC00003F07F03043558F8233026E654F8043D2C
:101AD000042B04D1002E05EB8605FFF64BAE3B78B8
:101AE000002B7FF436AE2B681E1203F07F03043503
:101AF00058F8233011E654F8043D042B04D0002E8E
:101B000005EB8605FFF636AE3B78002B7FF421AE61
:101B10002B681E1203F07F03043558F82330FCE5D0
:101B200054F8040CC307A4F1040B0BD54010013882
:101B300000280ADB400040F0010005EB8605CBF8E9
:101B4000000017E6FFF7E8FCF1E73B780BB15C46D5
:101B5000FFE52B681E1203F07F035C4658F8233024
:101B60000435DAE5730003F4FF7343F001032360E7
:101B7000DAF80830EB1A9D109AF8023043EA052390
:101B80005B0043F001036360029BA9EB0303224661
:101B90005B1043F00103361293608AF802607F4BBA
:101BA0003A78F6B20C4653F83630CAF808301AB113
:101BB00003F108058946CCE503F10C059B681E126C
:101BC00003F07F03894658F82330A6E5029B54F8BA
:101BD000046C4B452FD1F70720D4042E17D9336856
:101BE00003F00F03042B13D1304601F06FFF09F00F
:101BF000FFF8B0F5487F28BF4FF4487006306430D6
:101C000003F060FE70B9043DDDF80890B2E507D03E
:101C1000002E14BF4FF400700720F0E70A20EEE713
:101C20000720ECE731469AF8010004F066FA002339
:101C30008AF80030E8E759F80C3C58495A106FF020
:101C4000030353430C3B09EB030449F8036059F8C1
:101C5000083C5A108AF80220D2B2C3F3552351F837
:101C60003220CAF8082059F8041C4FEA6109029989
:101C700001EB89093978043402EB830500297FF4EC
:101C800068AD52F823301E1203F07F03043558F874
:101C9000233042E554F8040CFFF73EFC1E2883462F
:101CA000A4EB860425DC00280BDC3B78002B7FF4BA
:101CB00050AD2B681E1203F07F03043558F8233013
:101CC0002BE501F0EFFBABF1030B354E834401F044
:101CD000E9FBA0EB0B00B042F9D83B78002B7FF476
:101CE00038AD2B681E1203F07F03043558F82330FB
:101CF00013E501238AF8003001F0D4FB0A38584478
:101D0000CAF8040036E554F8040CFFF705FCA4EB10
:101D10008604061E0BDC3B78002B7FF41AAD2B6883
:101D20001E1203F07F03043558F82330F5E41D4BF1
:101D30009E4202DD1D233B700BE501238AF8003033
:101D400001F0B0FB4FF47A7303FB06000A38D7E7C3
:101D500000233046A4EB8604134E1A462146FFF7B3
:101D600029FC3168114802F0CEF8114B3168186037
:101D70000E4804F083F831680C4804F0C3F93B784E
:101D8000002B7FF4E6AC2B681E1203F07F030435B2
:101D900058F82330C1E400BFFCC000006086012079
:101DA0003F420F0080EE3600A8050020850200208B
:101DB000080000203B78A4EB8604002B7FF4C9AC1C
:101DC0002B681E1203F07F03043558F82330A4E477
:101DD000504603F0DBFD3B78002B7FF4BAAC2B6858
:101DE0001E1203F07F03043558F8233095E454F8AD
:101DF000043C002B44D154F80C0C10F0010B1ED005
:101E00004FEA600B4FEA4B0343F0010344F8083CF0
:101E1000BBF1000F40F388804FEA4B0343F001030E
:101E200054F80C0C44F8043C54F8083CC107CBEBC4
:101E300063032AD501335B0043F0010330E004283B
:101E40001BD9036803F00F02092A01D14068D7E7C4
:101E5000042A09D101F03AFE0378002BD2D0FFF713
:101E600092FA0BF1010BF7E7032A06D1C3F30F1B1C
:101E7000C3F34173C3EB8B0BC4E719233B7068E4D6
:101E80004FEA630B0BF1FF3BC2E7042849D9026814
:101E900002F00F02092A11D103F1020B50F82B3086
:101EA00049F826303B78002B7FF453AC2B681E1288
:101EB00003F07F03043558F823302EE4042A2BD195
:101EC000039309EB8603009301F000FE039B834616
:101ED0005E1C012E12DC5846FFF755FAA0EB0B06EC
:101EE000304602F009F8034670B1039001F0EEFDB0
:101EF0003246594608F0B8FB039B05E09BF80030DA
:101F0000013E23B912223A70009A1360CAE758467C
:101F1000FFF739FA8346DCE7032A02D11844037934
:101F200089E719233B7014E40435BBE7029A04EBFC
:101F300086039B1AD82B11DC0122002E06F1FF33F9
:101F400010DC3B78002B7FF404AC2B681E1203F0EE
:101F50007F03043558F82330FFF7DFBB1A233B70AB
:101F6000FFF7F7BB22601E460434E6E7029A231D02
:101F70009B1AD82B03DD1A233B70FFF7EABB029BA9
:101F80004B452AD254F8040CFFF7C6FA002821DD8D
:101F900059F80C3C5B1083421CDBC3EB8373184481
:101FA00000F180400438A4EB860359F820201A6021
:101FB0006FF0030303FB06443B780434002B7FF4EB
:101FC000C8AB2B681E1203F07F03043558F823308A
:101FD000FFF7A3BB20233B70EAE71823FBE7C14BC5
:101FE0001A68A4EB86031A606FF0030303FB064430
:101FF0003B780434002B7FF4ACAB2B681E1203F04B
:102000007F03043558F82330FFF787BB54F8043CAE
:10201000042B3B78A4F1040204BF05EB860522469D
:1020200013B11446FFF795BB2B681E1203F07F0314
:10203000144658F823300435FFF76FBB54F8043DBD
:10204000042B1CBF002323603B781CBF05EB8605D7
:102050000434002B7FF47DAB2B681E1203F07F034A
:10206000043558F82330FFF758BB002EA4EB860147
:1020700015DC1C233B7000226FF0030303FB0644B6
:102080003B780A600434002B7FF463AB2B681E128C
:1020900003F07F03043558F82330FFF73EBB0B688D
:1020A0004FF0000C5B1051F82C0010F0010202D12F
:1020B0000D233B70E0E7401083420CF1010CA8BFF8
:1020C00003466645EFDC5B0043F00102D4E7002ED7
:1020D000A4EB860115DC1C233B7000226FF0030388
:1020E00003FB06443B780A600434002B7FF431ABD9
:1020F0002B681E1203F07F03043558F82330FFF7D6
:102100000CBB0B684FF0000C5B1051F82C0010F06A
:10211000010202D10D233B70E0E7401083420CF135
:10212000010CB8BF03466645EFDC5B0043F00102DB
:10213000D4E754F8081C11F0010F4FEA86031FD0B2
:1021400054F8042C12F0010F1AD05210B2EB610FA8
:10215000A4EB0303D4BF002204221A606FF0030330
:1021600003FB06443B780434002B7FF4F2AA2B686F
:102170001E1203F07F03043558F82330FFF7CDBA61
:1021800054F8042C6FF00100A4EB030BFFF710F9D7
:10219000CBF80000E2E754F8081C11F0010F4FEAF9
:1021A00086031FD054F8042C12F0010F1AD05210DD
:1021B000B2EB610FA4EB0303B4BF002204221A6048
:1021C0006FF0030303FB06443B780434002B7FF4D9
:1021D000C0AA2B681E1203F07F03043558F8233081
:1021E000FFF79BBA54F8042C4FF0FF30A4EB030B1D
:1021F000FFF7DEF8CBF80000E2E754E90201814284
:102200004FEA860314D1E31A04221A606FF0030325
:1022100003FB06443B780434002B7FF49AAA2B6816
:102220001E1203F07F03043558F82330FFF775BA08
:102230000428A4EB030B01D8002315E0C307FBD44B
:10224000036803F00F03042BF6D1CB07F4D4042961
:10225000F2D90B6803F00F03042BEDD1FFF77EF9E1
:1022600000280CBF00230423CBF80030CEE754E94C
:10227000020181424FEA860314D1E31A00221A6058
:102280006FF0030303FB06443B780434002B7FF418
:1022900060AA2B681E1203F07F03043558F8233020
:1022A000FFF73BBA0428A4EB030B01D8042315E085
:1022B000C307FBD4036803F00F03042BF6D1CB074D
:1022C000F4D40429F2D90B6803F00F03042BEDD1E9
:1022D000FFF744F900280CBF04230023CBF800309B
:1022E000CEE700BF0800002054F8081C11F0010FD1
:1022F0004FEA86031FD054F8042C12F0010F1AD0B5
:102300005210B2EB610FA4EB0303CCBF00220422F6
:102310001A606FF0030303FB06443B780434002B80
:102320007FF417AA2B681E1203F07F03043558F8B8
:102330002330FFF7F2B954F8042C0120A4EB030B6F
:10234000FFF736F8CBF80000E3E754F8081C11F06B
:10235000010F4FEA86031FD054F8042C12F0010F2E
:102360001AD05210B2EB610FA4EB0303ACBF0022F2
:1023700004221A606FF0030303FB06443B78043425
:10238000002B7FF4E6A92B681E1203F07F030435AF
:1023900058F82330FFF7C1B954F8042C0220A4EBFD
:1023A000030BFFF705F8CBF80000E3E754F8043C13
:1023B000042BA4EB860314BF042200221A606FF0E2
:1023C000030303FB06443B780434002B7FF4C1A9CC
:1023D0002B681E1203F07F03043558F82330FFF7F3
:1023E0009CB954F8080CFFF797F8834654F8040C8E
:1023F000FFF792F85844A4EB8603400040F0010038
:1024000018606FF0030303FB06443B780434002B91
:102410007FF49FA92B681E1203F07F03043558F840
:102420002330FFF77AB954F8080CFFF775F88346A4
:1024300054F8040CFFF770F8ABEB0000A4EB860334
:10244000400040F0010018606FF0030303FB0644F6
:102450003B780434002B7FF47CA92B681E1203F018
:102460007F03043558F82330FFF757B954F8080CA8
:10247000FFF752F8834654F8040CFFF74DF800FBC1
:102480000BF0A4EB8603400040F0010018606FF0F1
:10249000030303FB06443B780434002B7FF459A963
:1024A0002B681E1203F07F03043558F82330FFF722
:1024B00034B954F8040CFFF72FF88346B8B91F233A
:1024C0003B70A4EB8603C3F800B06FF0030303FB7B
:1024D00006443B780434002B7FF43BA92B681E1282
:1024E00003F07F03043558F82330FFF716B954F88A
:1024F000080CFFF711F890FBFBFB4FEA4B0B4BF07E
:10250000010BDEE754F8040CFFF706F88346B8B970
:102510001F233B70A4EB8603C3F800B06FF00303E6
:1025200003FB06443B780434002B7FF412A92B688C
:102530001E1203F07F03043558F82330FFF7EDB87F
:1025400054F8080CFEF7E8FF90FBFBF303FB1B0BB2
:102550004FEA4B0B4BF0010BDCE754F8040CFEF791
:10256000DBFF0028B8BF4042A4EB8603400040F0E8
:10257000010018606FF0030303FB06443B7804344A
:10258000002B7FF4E6A82B681E1203F07F030435AE
:1025900058F82330FFF7C1B8A4EB860B012EDBF807
:1025A000000028D1FEF7B8FF32460346039300929D
:1025B00008F070FB039B009A012BB8BF012390FB2E
:1025C000F3F101FB130313445B0043F00103CBF869
:1025D00000306FF0030303FB06443B780434002B08
:1025E0007FF4B7A82B681E1203F07F03043558F858
:1025F0002330FFF792B8FEF78FFF0090DBF804005E
:10260000FEF78AFF009A0130831ACFE7A4EB860B0E
:102610005946304601F00CFE6FF0030303FB0644FD
:102620003B78CBF800000434002B7FF492A82B6891
:102630001E1203F07F03043558F82330FFF76DB8FE
:1026400054F8080CFEF768FF834654F8040CFEF7B4
:1026500063FF0BEA0000A4EB8603400040F001009A
:1026600018606FF0030303FB06443B780434002B2F
:102670007FF46FA82B681E1203F07F03043558F80F
:102680002330FFF74AB854F8080CFEF745FF83469D
:1026900054F8040CFEF740FF4BEA0000A4EB86035D
:1026A000400040F0010018606FF0030303FB064494
:1026B0003B780434002B7FF44CA82B681E1203F0E7
:1026C0007F03043558F82330FFF727B854F8080C77
:1026D000FEF722FF834654F8040CFEF71DFF8BEA39
:1026E0000000A4EB8603400040F0010018606FF08A
:1026F000030303FB06443B780434002B7FF429A832
:102700002B681E1203F07F03043558F82330FFF7BF
:1027100004B854F8040CFEF7FFFEC043A4EB860394
:10272000400040F0010018606FF0030303FB064413
:102730003B780434002B7FF40CA82B681E1203F0A6
:102740007F03043558F82330FEF7E7BF54F8080C30
:10275000FEF7E2FE834654F8040CFEF7DDFE0BFAAA
:1027600000F0A4EB8603400040F0010018606FF019
:10277000030303FB06443B780434002B7EF4E9AFEB
:102780002B681E1203F07F03043558F82330FEF740
:10279000C4BF54F8080CFEF7BFFE834654F8040C7F
:1027A000FEF7BAFE4BFA00F0A4EB8603400040F0BF
:1027B000010018606FF0030303FB06443B78043408
:1027C000002B7EF4C6AF2B681E1203F07F03043586
:1027D00058F82330FEF7A1BF54F80C0CFEF79CFE0E
:1027E000834654F8080CFEF797FE8BFB002354F841
:1027F000040CCDE90023FEF78FFEDDE90023C0F1D4
:10280000200CB0F1200103FA0CFC22FA00F040EA9F
:102810000C005CBF43FA01F108436FF00303A4EB23
:10282000860E400003FB06443B7840F00100CEF8E2
:1028300000000434002B7EF48CAF2B681E1203F0D2
:102840007F03043558F82330FEF767BFA4EB860BEF
:1028500059463046FEF7F6FB6FF0030303FB0644D0
:102860003B78CBF800000434002B7EF472AF2B6869
:102870001E1203F07F03043558F82330FEF74DBFD6
:10288000A4EB860421463046FEF7F3FB3B78002B91
:102890007EF45FAF2B681E1203F07F03043558F8F7
:1028A0002330FEF73ABFA4EB860B59463046FEF7BD
:1028B00021FC6FF0030303FB06443B78CBF80000D8
:1028C0000434002B7EF445AF2B681E1203F07F0307
:1028D000043558F82330FEF720BFA4EB86042146C8
:1028E0003046FEF791FC3B78002B7EF432AF2B682C
:1028F0001E1203F07F03043558F82330FEF70DBF96
:10290000A4EB860B59463046FEF7ECFC6FF0030350
:1029100003FB06443B78CBF800000434002B7EF424
:1029200018AF2B681E1203F07F03043558F82330CC
:10293000FEF7F3BE54F8040C01F0C8F854F8083C54
:10294000DA072AD4042B0CD91B6803F00F03013BD0
:10295000082B10D8DFE803F0052127230F0F0F0FF6
:102960002500CC4908F03AFAA4EB8603002814BFEE
:10297000002204221A606FF0030303FB06443B7835
:102980000434002B7EF4E5AE2B681E1203F07F03A7
:10299000043558F82330FEF7C0BEBF49E2E7BF490F
:1029A000E0E7BF49DEE7BF49DCE7029B261DF31ADB
:1029B000D82B03DD1A233B70FEF7CBBE00F07AFD67
:1029C0002346400040F0010018603B783446002B5D
:1029D0007EF4BFAE2B681E1203F07F03043558F857
:1029E0002330FEF79ABE029B261DF31AD82B03DD77
:1029F0001A233B70FEF7ADBE00F054FDAA4A2346F1
:102A000002EA400040F0010018603B783446002B99
:102A10007EF49FAE2B681E1203F07F03043558F836
:102A20002330FEF77ABE029B261DF31AD82B03DD56
:102A30001A233B70FEF78DBE00F03CFD9B4B1B68DC
:102A400098423DBFC3F5830303F63713C018C01A7D
:102A50004000234640F0010018603B783446002BCC
:102A60007EF477AE2B681E1203F07F03043558F80E
:102A70002330FEF752BE00F01DFD8C4B18603B78F2
:102A8000A4EB8604002B7EF464AE2B681E1203F0C8
:102A90007F03043558F82330FEF73FBE00F016FDE3
:102AA000B30068B9E41A3B78002B7EF452AE2B6871
:102AB0001E1203F07F03043558F82330FEF72DBEB5
:102AC000304627467A4EE41A01231A462146FEF77D
:102AD00071FD3068643002F0F5FE18B9043D3C46E3
:102AE000FEF748BE9AF801203168724803F01DFBDA
:102AF00001238AF8003000F0D5FC6F4A3368126871
:102B0000063302FB0300FFF7FBB800F0DFFCB30065
:102B100068B9E41A3B78002B7EF41BAE2B681E12BA
:102B200003F07F03043558F82330FEF7F6BD304636
:102B300027465F4EE41A002201232146FEF73AFDA4
:102B40003068643002F0BEFE0028C7D0594803F058
:102B500081F8CDE7FEF7ACFD6FF00303A4EB860B25
:102B600003FB06443B78CBF800000434002B7EF4D2
:102B7000F0AD2B681E1203F07F03043558F82330A4
:102B8000FEF7CBBD3B78A4EB8604002B7EF4E1ADD1
:102B90002B681E1203F07F03043558F82330FEF72C
:102BA000BCBDA4EB860B584600F0BDFC6FF00303E0
:102BB00003FB06443B78CBF800000434002B7EF482
:102BC000C8AD2B681E1203F07F03043558F823307C
:102BD000FEF7A3BDA4EB860B584600F0A6FC6FF0F1
:102BE000030303FB06443B78CBF800000434002BBE
:102BF0007EF4AFAD2B681E1203F07F03043558F846
:102C00002330FEF78ABDA4EB860B5946304600F010
:102C10008FFC6FF0030303FB06443B78CBF8000006
:102C20000434002B7EF495AD2B681E1203F07F0355
:102C3000043558F82330FEF770BDA4EB8604204617
:102C400000F0A8FC3B78002B7EF483AD2B681E12AD
:102C500003F07F03043558F82330FEF75EBDA4EB84
:102C6000860B5946304600F0CFFC6FF0030303FBA0
:102C700006443B78CBF800000434002B7EF469ADA9
:102C80002B681E1203F07F03043558F82330FEF73B
:102C900044BD00BF0CC1000014C100001BC10000F6
:102CA00022C1000027C10000FEFFFF7FB005002009
:102CB000A80500208502002004000020A4EB860463
:102CC000204600F05DFD3B78002B7EF442AD2B6882
:102CD0001E1203F07F03043558F82330FEF71DBDA4
:102CE0000121304600F01AFD3B78002B7EF431AD17
:102CF0002B681E1203F07F03043558F82330FEF7CB
:102D00000CBD0021304600F009FD3B78002B7EF41D
:102D100020AD2B681E1203F07F03043558F82330D2
:102D2000FEF7FBBCA4EB860B584600F0AFFC6FF03F
:102D3000030303FB06443B78CBF800000434002B6C
:102D40007EF407AD2B681E1203F07F03043558F89C
:102D50002330FEF7E2BCA4EB860B584600F0AAFC39
:102D60006FF0030303FB06443B78CBF80000043408
:102D7000002B7EF4EEAC2B681E1203F07F030435AB
:102D800058F82330FEF7C9BCA4EB8604204600F0B7
:102D900065FC3B78002B7EF4DCAC2B681E1203F044
:102DA0007F03043558F82330FEF7B7BCA4EB860444
:102DB000204603F01BFE3B78002B7EF4CAAC2B6848
:102DC0001E1203F07F03043558F82330FEF7A5BC2C
:102DD000A4EB860B584603F0C9FE6FF0030303FB18
:102DE00006443B78CBF800000434002B7EF4B1ACF1
:102DF0002B681E1203F07F03043558F82330FEF7CA
:102E00008CBCA4EB8604204603F05EFD3B78002BCF
:102E10007EF49FAC2B681E1203F07F03043558F834
:102E20002330FEF77ABCA4EB860B584603F068FD0E
:102E30006FF0030303FB06443B78CBF80000043437
:102E4000002B7EF486AC2B681E1203F07F03043542
:102E500058F82330FEF761BCA4EB860421463046C7
:102E600001F08AFC3B78002B7EF473AC2B681E12B9
:102E700003F07F03043558F82330FEF74EBCA4EB73
:102E800086042146304601F09DFA3B78002B7EF403
:102E900060AC2B681E1203F07F03043558F8233012
:102EA000FEF73BBCA4EB86042146304601F09AFBBA
:102EB0003B78002B7EF44DAC2B681E1203F07F0391
:102EC000043558F82330FEF728BCA4EB86042146CD
:102ED000304601F0ADFB3B78002B7EF43AAC2B681A
:102EE0001E1203F07F03043558F82330FEF715BC9B
:102EF000A4EB860B5946304603F070FF6FF00303D6
:102F000003FB06443B78CBF800000434002B7EF42E
:102F100020AC2B681E1203F07F03043558F82330D1
:102F2000FEF7FBBBA4EB860B5946304603F05EFF71
:102F30006FF0030303FB06443B78CBF80000043436
:102F4000002B7EF406AC2B681E1203F07F030435C1
:102F500058F82330FEF7E1BBA4EB860B5946304608
:102F600003F04CFF6FF0030303FB06443B78CBF800
:102F700000000434002B7EF4ECAB2B681E1203F02F
:102F80007F03043558F82330FEF7C7BBA4EB860B4C
:102F90005946304603F04CFB6FF0030303FB064435
:102FA0003B78CBF800000434002B7EF4D2AB2B68C6
:102FB0001E1203F07F03043558F82330FEF7ADBB33
:102FC000A4EB86042146304601F026FA3B78002B1C
:102FD0007EF4BFAB2B681E1203F07F03043558F854
:102FE0002330FEF79ABBA4EB86042146304601F05D
:102FF00047FB3B78002B7EF4ACAB2B681E1203F032
:103000007F03043558F82330FEF787BBA4EB860B0B
:103010005946304601F0AEFA6FF0030303FB064455
:103020003B78CBF800000434002B7EF492AB2B6885
:103030001E1203F07F03043558F82330FEF76DBBF2
:10304000A4EB86042146304601F058FA3B78002B69
:103050007EF47FAB2B681E1203F07F03043558F813
:103060002330FEF75ABB002E5ADD012E54F804BC63
:1030700039D11BF0010F43D1BBF1040F40D9DBF86C
:10308000003003F00F03042B3AD1584600F01EFD28
:10309000FEF7E6F90028A4EB860441DB022E3DD1C1
:1030A0001BF0010F35D1BBF1040F32D9DBF8003032
:1030B00003F00F03092B2CD1DBF80460211FC6F3AA
:1030C00047060123B3421EDD04EB860446EA0026D0
:1030D000029B04F10C01CB1AD82B7EF743AD1A23C7
:1030E0003B70FEF736BB022E0AD154F8080CC3071A
:1030F00006D4042804D9036803F00F03042BC5D0B9
:103100004FF0FF30C6E701335BF8232041F8042F6E
:10311000D8E7C4F800B001260434D7E70026D5E785
:10312000002323603B78221D13B11446FEF711BB28
:103130002B681E1203F07F03144658F82330043521
:10314000FEF7EBBA029BE31A9B10A4EB8604CAF8C5
:1031500010302146304602F0BDFD3B78002B7EF456
:10316000F8AA2B681E1203F07F03043558F82330A9
:10317000FEF7D3BA029BE31A9B10A4EB860BCAF8A6
:1031800010305946304602F0A5FD6FF0030303FBF3
:1031900006443B78CBF800000434002B7EF4D9AA17
:1031A0002B681E1203F07F03043558F82330FEF716
:1031B000B4BA00BF2DE9F84F224D0023002B03F1D4
:1031C000FF3706DA01F07AFB02F094FE03F00CF808
:1031D00019270026DFF878803046D8F80020B24260
:1031E00015DD2B68184C01339342A8BF00232B60D8
:1031F000D5F80090F02303FB09F304EB030AE35C2A
:10320000A346EBB1022B04D15046FEF767FA3B46CA
:10321000D4E7012B0ED108B900F044F9F02303FBE9
:1032200009F39B440949DBF80420821A8A429CBFB7
:103230000222E254F02303FB09F3E35C022BE3D008
:103240000136CAE700000020007D01203F420F0048
:10325000AC0500200A4B4FF480721A60094B012123
:103260001964D3F840250532C3F84825C3F84C2526
:103270004FF44022C3F80423034B1970704700BF7A
:1032800000E100E000800040D705002004207047E6
:10329000F8B5D1E9004514F001002DD015F001007A
:1032A0002AD064101C2C3CD81F4F6D1041F2883678
:1032B0003B5DAE42A8BF2E46012B05D00121204622
:1032C00005F00EF901233B55184B1B780BB9FFF79E
:1032D000C1FF002D4FF00003154A0EDC154940F2E6
:1032E000DC50FF25D65CB44204BF21F81300D5544E
:1032F0000133042BF6D10420F8BDD15C8C4203D1FC
:103300000C4A22F81360F6E70133042BF5D10023B1
:10331000D15CFF2901D1D454F2E70133042BF7D15A
:10332000E9E70020E8E700BFB8050020D705002046
:103330001C0000200E00002070B5D1E9004514F0FB
:1033400001001BD015F0010018D064101D2C28BFFF
:103350001B24154E335D012B05D00121204605F0BD
:10336000BFF801233355114B6D10A5F110029A429D
:103370000F4B04D94FF0FF321A60042070BD1C605F
:103380000C4B0D4890FBF5F018800C4B1B780BB9DB
:10339000FFF760FF0A4B01229A64D3F848251044D6
:1033A000C3F84805E9E700BFB80500209086010092
:1033B000180000200C00002020A10700D7050020E5
:1033C0000080004070B50D680128CCBF4C68012416
:1033D00015F0010042D014F001003FD06D10002D17
:1033E00005DC1F4B0122C3F80825002036E06410DD
:1033F0001C2CFAD81B4E335D012B05D00121204631
:1034000005F06EF8012333550A22174B93FBF5F3B1
:10341000053393FBF2F3154A154952F82420154859
:10342000120242F00312C1F810250D4AC2F810052D
:10343000C2F814150121C2F80415A2F5A8321069CA
:103440000020C2F810054FF6FF708342A8BF034664
:10345000C2F840350420C2F80012116070BD00BFF0
:1034600000F00140B805002000B4C40408D20000F8
:103470000060004040A10040002802DC1C20FEF754
:1034800011B90120704704207047002802DC1C207D
:10349000FEF708B90B68DB0701D40D20F8E7002020
:1034A00070470000024B01221A64D3F840057047B0
:1034B00000800040044B01221A64D3F840054FF409
:1034C0007A73B0FBF3F07047008000400120704732
:1034D0000048704790C100001D20704770B5054D31
:1034E0002B5C8B4204460E4602D004F0F9FF2E55A9
:1034F00070BD00BFB805002070B50024084D2646F9
:10350000635D012B08D10021204605F013F800214E
:10351000204604F0E5FF665501341D2CF0D170BD46
:10352000B805002070470F2070473B20704700000F
:10353000F8B50B68DA0707460D4604D40D20FEF7F0
:10354000B1F8012007E05B10062B05D103F0EAF982
:10355000400040F00100F8BDF3D80C4A0C4E52F880
:103560002340335D2BB10021204604F0B9FF002336
:103570003355012F06DD6B68042B03D10221204651
:1035800004F0AEFF204604F0B5FEE1E774C1000090
:10359000B805002070B50468E20702D54568EB075E
:1035A00004D40D20BDE87040FEF77CB864101C2CDC
:1035B00023D8124E335D012B18D00121204604F090
:1035C0008FFF01231B2C335510D10D4BDA6E0D4BA1
:1035D000202AB8BF4FF0A04302F01F0203EB820382
:1035E000D3F8002742F44072C3F80027A5F34A013C
:1035F0002046BDE8704004F021BF70BDB805002032
:1036000008D200000003005070B50C68E30704D432
:103610000D20FEF747F8012070BD64101C2C14D853
:10362000012814DD4B68042B14BF002502250A4E27
:10363000335DAB4204D02946204604F051FF355596
:10364000204604F093FF012803D00020E4E7002582
:10365000EDE70420E0E700BFB805002013B50A4AF3
:10366000044692E8030022686B46042A83E80300BC
:1036700019464FF0020003D100F0B4FF02B010BDB4
:1036800000F0D6FFFAE700BF34C1000010B5084CC7
:1036900063792BB10021052004F022FF0023637120
:1036A000052004F063FF00280CBF0420002010BD9B
:1036B000B805002010B5084CE37A2BB100210B208F
:1036C00004F00EFF0023E3720B2004F04FFF0028EC
:1036D0000CBF0420002010BDB805002010B50B4A17
:1036E0000B4C0C480C490023C2F80035A2F5C83237
:1036F000C2F810350122626042604A60C4F80035A9
:10370000C0F80035C1F8003510BD00BF00F0014021
:1037100000C0014000100240002002401C2870B58B
:1037200004460D4625D8134E335C012B04D00121ED
:1037300004F0D6FE012333551C2C12D1FFF7CEFF27
:103740000D4B1A6F0D4B202AB8BF4FF0A04302F06B
:103750001F0203EB8203D3F8002742F44072C3F840
:103760000027291C204618BF0121BDE8704004F045
:10377000E1BE70BDB805002008D200000003005073
:103780000368D90702D40D20FDF78CBF41680A1FDA
:10379000514251415810FFF7C1BF0000F8B5324CFB
:1037A000D4F84831ABB10023D4F84855C4F84831B7
:1037B0002E4B186800280CDB2D4A1178B1FA81F1E4
:1037C0004909117004F0B6FE2A4B1B882B44C4F83B
:1037D0004835254BD3F84C21002A37D00021264EFE
:1037E000D3F84C45C3F84C113378244D33B12B68D2
:1037F000032B03D8224AD05C04F09CFE2B68204F98
:1038000001335A4202F0030203F0030358BF53424C
:103810002B600022042B194619D00133F81810F838
:10382000010CFF2801D10122F4E702B12960012136
:1038300004F080FE012333702A68124B33F8122003
:1038400004F10C031344084AC2F84C35F8BD4FF09C
:10385000FF3304F58C44044A2B605C34002333703E
:10386000C2F84C45F2E700BF00800040180000207D
:10387000D60500200C000020D5050020B40500204E
:103880001C0000200E000020094B0A4940F2DC52C7
:103890001A805A809A80DA80074A00231370074AF8
:1038A000FF20087048708870C8701360704700BFB0
:1038B0000E0000201C000020D5050020B4050020CB
:1038C000024B4FF0FF321A60704700BF1800002013
:1038D000024A0348072101F085BF00BF3CC1000038
:1038E00076C9000038B54FF4E131284804F0D8FA21
:1038F000274B012200211A61C3F804150321C3F8E4
:1039000008150421C3F810151A604FF080430221F6
:10391000C3F818159A604FF01023D3F80C32DB0768
:103920000FD51C4BC3F80425D3F80024002AFBD084
:103930004FF010226FF00101C2F80C120022C3F800
:1039400004250A2004F0D0FC134A0023FF219954D7
:1039500001331D2BFBD1114B114D01221A600020A8
:10396000104A042301461468002CFCD02C68116016
:10397000013B44EA0020F6D10B4B01221A6004F00F
:10398000E9FBBDE8384001F035B800BF807C01207C
:103990000080004000E00140B805002000D0004059
:1039A00008D5004000D1004004D00040F8B50646DC
:1039B0000948094F0C4604F0B3FA8442A8BF0446F4
:1039C0003546AB1B9C4205DD384604F0AFFA05F8DE
:1039D000010BF6E72046F8BD807C01200146014836
:1039E00004F063BA807C012010B5054C204604F039
:1039F00069FA20464FF4E131BDE8104004F050BAB6
:103A0000807C0120C3070CD4064B1B68834208D876
:103A1000054B1B68984204D850F8043C002B18BF93
:103A200018467047E0050020DC0500200B4908B56A
:103A30000122002341F823200133642BFAD1084BE3
:103A40001A60084B084A1846002106F031FE074B61
:103A500040F8043F064B186008BD00BF588E012097
:103A600008000020E405002070670100A09D05000B
:103A7000D8050020034B044A1A60044B044A1A601C
:103A8000FFF7D4BFE0050020E4050020DC0500209E
:103A9000546D0120044B1B681868C0F30F100238E6
:103AA00020EAE070704700BFD805002000B59BB049
:103AB0000246054901A807F055F901A802F0E7F808
:103AC00002F092FBFCE700BF22C20000C30713D440
:103AD000042802D812D00B487047036803F00F0384
:103AE000042B01D104307047092B09D0064A07483E
:103AF000032B18BF104670470548704705487047AC
:103B00000548704770BD00000DC2000016C20000DD
:103B1000FCC1000076BD000006C20000064B07494C
:103B200000201A6843F8040CC2F30F12023203EBB0
:103B300082038B42F5D37047E8050020546D0120C5
:103B40002F4B304A1868304B2DE9F0411C682F4D3F
:103B5000136803F00F01072928D81368C3F30F1364
:103B6000023302EB8302AA42F2D32949002251F820
:103B70002200FFF747FF41F822000132642AF6D104
:103B8000244A1068FFF73EFF1060234A106810B106
:103B9000FFF738FF1060214B214C1E680021F027F1
:103BA0004FF03C08B14214DBBDE8F081C3F30F13C2
:103BB00002EB83039A42D0D01968CE0707D488421B
:103BC00005D28C4203D351F8041C01B11960043BA7
:103BD000F0E707FB01F31A191B5D0BB90131E1E7AF
:103BE0001269551E08FB012204EB82021832002DD7
:103BF000F4DB52F8040DFFF705FF013D1060F6E716
:103C0000E0050020E8050020DC050020546D0120BF
:103C1000588E012008000020546D0120AC050020C2
:103C2000007D0120C307F0B540D4214B1C68A042A1
:103C30003CD3204B1D68A84238D850F8043CABBB9D
:103C400003680246C3F30F13012673B9904242F88A
:103C5000046C2BD0116851F8043C51F823701760A4
:103C600041F82320013B0A46EFE752F82310CF0723
:103C700002EB830C18D48C4216D88D4214D351F821
:103C8000047C8FB90F6807F00F0EBEF1070F08D93B
:103C9000CCF8007042F8043C0B680A60C3F30F13C1
:103CA000E1E741F8046CD0E7013BCEE7F0BD00BF8F
:103CB000E0050020DC0500200D4930B50D4C0B4619
:103CC0001A6853F8045CC2F30F12901C65B18B4262
:103CD00014BF0A46002243F8042C01EB800103EBD9
:103CE0008003A342ECD330BD12011A60F7E700BF96
:103CF000E8050020546D0120144B2DE9F041144CCF
:103D00001E464FF000083268C2F30F1712070FD09B
:103D10007D1C9E424FEA850505D018462A4631464D
:103D200006F0ADFC03465A1904352B44C2F8008056
:103D3000023706EB8706A642E5D3E41AA410013C3D
:103D4000044A24011C601360BDE8F081E8050020EE
:103D5000546D0120D80500202DE9F0419AB0FFF7FD
:103D6000A1FB214D0746002455F824000134FFF73C
:103D700059FF642CF8D11D4B1868FFF753FF1C4BFB
:103D8000186808B1FFF74EFF1A4DDFF8748000265F
:103D9000D8F800309E4218DBFFF78EFFFFF7D0FE09
:103DA000FFF7AAFFFFF77EFB134B14491B681B6844
:103DB000C3F30F13C21B023B01A806F0D3FF01A8F7
:103DC00001F065FF1AB0BDE8F0812B7813B9013618
:103DD000F035DDE72C69013C002CF8DB05EB8403B2
:103DE0009869FFF71FFFF6E7588E012008000020B2
:103DF000546D0120007D0120D8050020DCC10000A9
:103E0000AC0500202DE9F8431B4C23681B684D1CB2
:103E1000C3F30F139D42064688461746A1460CDBA6
:103E2000FFF79AFF23681B68C3F30F139D4204DB5F
:103E30000A20BDE8F843FDF735BC08F10202D9F8C5
:103E400000009B1A1B0140F82230002340F8043C7C
:103E500006F00F06034646EA0816940043F8046B82
:103E60000119083CC9F800101C44A34201D3BDE865
:103E7000F88343F8047BF8E7D8050020F8B510F084
:103E8000010704460E462CD1174B1B68834228D8E5
:103E9000164B1B68834224D9154D28600068012207
:103EA00000F00F00FFF7AEFF2C682F600546C0B191
:103EB0002146043051F8042BC2F30F12B242A8BFBE
:103EC0003246920006F0D0FBFFF728FE44F8045C6F
:103ED000FFF736FE2268074B44F8047C134023604A
:103EE0002C462046F8BD00BFE0050020DC05002080
:103EF000546D0120F0FF0F00011D0022042091FBF2
:103F0000F0F1FFF77FBF38B5054608460C46FFF7CE
:103F1000F3FF50B1C21C2B46591B8C4206DC002C0F
:103F2000ACBF0419041C0023237138BD13F8011B16
:103F300002F8011FF0E7F0B502289BB00C4604DC44
:103F40001C20FDF7AFFB1BB0F0BD0868C20706D40C
:103F5000042804D9036803F00F03042B01D00E20BA
:103F6000EFE74B6813F00107F9D1042BF7D91B6871
:103F700003F00F03042BF2D18B68DB0701D40D2073
:103F8000DFE7FFF7A3FD06466068FFF79FFDA56822
:103F90001AAC014604F8647D6D10304603F0B3FAA4
:103FA00029466423224603F010FB204606F020FF3A
:103FB00001462046FFF7A7FFC5E7000010B50446FD
:103FC000ADF5806D10B9FFF797FF0BE003F0C1F975
:103FD0000138062827D8DFE800F008081017280461
:103FE000230000200DF5806D10BD204603F02BFA54
:103FF000011B2046FFF787FFF4E7204603F0D7F9BF
:10400000400040F00100EDE769464FF48062204631
:1040100003F0E7F9684606F0EBFE01466846E9E77B
:1040200004210348E6E70020CDE70420DAE700BFDB
:1040300068C20000022838B50C4604DC1C20BDE82C
:104040003840FDF72FBB0868C10706D4042804D9FF
:10405000036803F00F03042B01D00E20EFE7636821
:10406000DA07FAD4042BF8D91B6803F00F03042BEA
:10407000F3D1A368DB0701D40D20E0E7FFF726FDAD
:1040800005466068FFF722FDA468014664102846D3
:1040900003F039FA214603F075FABDE83840FFF71E
:1040A0008DBF012838B50C4604DC1C20BDE8384023
:1040B000FDF7F8BA0868C10706D4042804D90368D4
:1040C00003F00F03042B01D00E20EFE76368DA073B
:1040D000FAD4042BF8D91B6803F00F03042BF3D197
:1040E000FFF7F4FC05466068FFF7F0FC0146284640
:1040F00003F009FA03F085FA400040F0010038BDF2
:10410000012870B505460C4604DC1C20BDE8704053
:10411000FDF7C8BA0868C10706D4042804D90368A3
:1041200003F00F03042B01D00E20EFE76368DA07DA
:10413000FAD4042BF8D91B6803F00F03042BF3D136
:10414000FFF7C4FC06466068FFF7C0FC022D01467D
:1041500015D0A468E30712D56410304603F0D3F9F4
:10416000054603F0F6F8012812D1002C02DD0135D6
:10417000012C07D12846BDE87040FFF71FBF4FF064
:10418000FF34EAE7284603F06DF9013C0546EFE706
:104190000228EFD1002CEDDD0135012CEAD0002200
:1041A0001146284603F088F903F05CF9013C054606
:1041B000F3E70000086810B510F001041AD04410AD
:1041C00007EE904A9FED187AF8EEE77A67EE877A65
:1041D00017EE900A05F0AAFE04F0D0FA0022134B65
:1041E00005F0FCFE04F080FA06F0A8F9400040F06B
:1041F000010010BD042812D9036803F00F03042B3B
:1042000007D1FFF763FC0A22214606F0B5FE0446FB
:10421000D6E7032B03D10A2221460430F5E70D200F
:10422000FDF740FACCE700BFD30237390000D04099
:10423000086808B5C30706D4042804D9036803F046
:104240000F03042B04D00E20BDE80840FDF72ABA66
:10425000FFF73CFC0378232B08BF0130102200211C
:1042600006F08AFE00F10053B3F1804F01D3142011
:10427000EAE7400040F0010008BD0000024A0348A0
:10428000062101F0AFBA00BF38C2000033C20000FF
:10429000002070471E20FDF705BA1E20FDF702BA68
:1042A0001E20FDF7FFB91E20FDF7FCB91E20FDF70B
:1042B000F9B91E20FDF7F6B91E20FDF7F3B91E204F
:1042C000FDF7F0B91E20FDF7EDB91E20FDF7EAB9A4
:1042D0001E20FDF7E7B91E20FDF7E4B91E20FDF70B
:1042E000E1B91E20FDF7DEB91E20FDF7DBB91E2067
:1042F000FDF7D8B9024A0348112101F073BA00BF93
:10430000A4C200002CC30000034B01221A60034B1F
:104310001868904010437047746D0120586D01205B
:104320002DE9F041EFF31082012302F0010883F33D
:1043300010881549154C0968154D164E01398B40EA
:1043400003274FF00E0C4FF00B0E002B18D02168F6
:10435000296018420AD0724611000139FDDC21683B
:10436000316039000139FDDC5B08EEE739000139C5
:10437000FDDC21683160624611000139FDDCF3E7A4
:1043800088F31088BDE8F08120000020686D0120CE
:10439000080500500C05005070B5084E084D00246B
:1043A00056F824000021FFF799F855F82400002161
:1043B0000134FFF793F8052CF2D170BD18C400004A
:1043C00064C7000008B5054B00221A60044B1B6847
:1043D0000BB102F05DFF002008BD00BF706D012031
:1043E000E47A012010B5041E0ADA0024074B53F8C2
:1043F000242001239340064A1360064A136010BD2F
:10440000FFF76AF8A042F0DDF0E700BF08D2000035
:10441000686D0120180500502DE9F843344B1B68E6
:104420000C461BB94FF0FF30FFF7DCFF246814F097
:10443000010525D0C4F34743C4F34720C4F3470222
:1044400040F2596540435B4390FBF5F193FBF5F077
:10445000000240EA01401346534393FBF5F318432F
:10446000244B1B68202B01BF234BC4F3456453F836
:10447000243043EA0020FFF753FF0020BDE8F88313
:10448000042CFAD9236803F00F03092BF5D154F853
:10449000046FDFF86080DFF86090761040F25967B3
:1044A000B542EADA54F8042FD3071FD5C2F34743C5
:1044B000C2F34720C2F3470140435B4390FBF7FC44
:1044C00093FBF7F0000240EA0C400B464B4393FB92
:1044D000F7F31843D8F80030202B02BFC2F345622F
:1044E00059F8223043EA0020FFF71AFF0135D7E7D9
:1044F000686D01202000002008C6000008B50B6888
:10450000DA074CBF5B104FF0FF3301280DDD4A681E
:10451000042A14BF18222022054918460A60FFF712
:1045200001F8FFF75FFF002008BD1822F4E700BF85
:104530002000002010B510F0010402D044102046E5
:1045400010BD042812D9026802F00F02042A07D114
:10455000FFF7BCFA0A222146BDE8104006F00CBD68
:10456000032A03D10A2221460430F5E70D20FDF786
:1045700099F8E4E7086810F0010370B51CD0FFF764
:10458000D9FF0346203B5E2B27D8154C03EB830352
:104590000022012110462344052A1AD09E5C0524DE
:1045A00010252E4218BF4018013C4FEA41014FEA46
:1045B0006505F6D10132EFE70428E3D9026802F07D
:1045C0000F010429DED1C2F30F13002BDAD00379D7
:1045D000D8E7400040F0010070BD0120FCE700BFBB
:1045E0002CC4000038B508680D46FFF7A3FF044649
:1045F0006868FFF79FFF621E042A014612D8431E17
:10460000042B0FD8084803EB8303134405680122E9
:1046100002FA03F32B430360044B1B6813B12046DB
:1046200002F037FE002038BD706D0120E47A0120D1
:1046300038B508680D46FFF77DFF04466868FFF748
:1046400079FF621E042A014614D8431E042B11D898
:10465000094803EB83031344012202FA03F30268BF
:1046600022EA0302054B02601B681BB100222046B0
:1046700002F00FFE002038BD706D0120E47A0120A9
:104680002DE9F04F054685B008680C46FFF752FF4C
:10469000022D01903CDD6068FFF74CFF0746A068E3
:1046A000FFF748FF0446231DDFF8C8A00293661EEB
:1046B0004FF00108029B9E4206F1010935D006EB3E
:1046C0008602531E07F1050B3D460393AB4522D0EE
:1046D000042E19D86A1E042A16D8039B019ADAF808
:1046E00000005919224B4FF0010C18EA020E0CFA87
:1046F00001F11B6811D00143CAF8001023B16246D2
:104700004946284602F0C5FD4FEA48080135DDE775
:1047100001242746C7E74E46CCE720EA0101CAF844
:104720000010002BF0D07246EAE73D1D042D1BD887
:10473000012C19D1DFF83C80DFF834900026D8F83E
:10474000003004FA05F223EA0203C8F80030D9F871
:104750000030013623B100223146781D02F099FD68
:10476000052E05F10505EAD1002005B0BDE8F08F62
:10477000E47A0120706D0120086808B5C30703D5ED
:10478000FFF7D8FE054B1860054B1B681BB1034BA8
:10479000186802F07FFD002008BD00BF706D012089
:1047A000E47A01202DE9F3413F4D4FF441732C6829
:1047B000ADF804300A238DF806305CBBFFF7ECFD42
:1047C000DFF8F480264658F8267001213846FEF7B7
:1047D00085FE01360021384603F0ACFE052EF2D1ED
:1047E00000260DF1040816F8087001213846FEF77E
:1047F00075FE01360121384603F09CFE032EF2D1EE
:10480000FEF750FE294B186001232B60204602B0B2
:10481000BDE8F081012C1CD1244C2668FEF742FE35
:10482000864298BF801BC72801D80024EEE70021EC
:104830000420FEF753FE00210320FEF74FFE002167
:104840000A20FEF74BFEFEF72DFE022320602B60B0
:10485000EBE7022C21D1154B1C68FEF723FE8442A6
:1048600098BF001BB0F57A6FDFD3042003F042FD40
:104870000446032003F03EFD06460A2003F03AFDFD
:1048800034442044C0F53F6003230D3090FBF3F027
:10489000074B1860012003F02DFD064A00232B6012
:1048A00013600124B2E700BF646D01206C6D01202C
:1048B000586D0120746D012064C700002DE9F84394
:1048C000434E326852B9434B1B683BB9424B1B689D
:1048D000002B74D0BDE8F843FFF764BF3F4D2C6850
:1048E00084BB3D4B1B68002B65D13A4A3368106886
:1048F0001146002865D13A4F3A4EDFF8F4800B603C
:10490000002157F82400FEF7E9FD56F82490012114
:104910004846FEF7E3FDB9F1220F10D858F82920D8
:10492000314B1F2AD8BF4FF0A04302F01F0203EB08
:104930008203D3F8002742F44072C3F80027013401
:10494000052CDDD12B68264EDFF88890254F002BF3
:10495000CCBF03F1FF330423002156F82300FEF7F8
:10496000BDFD2A68214B53F82280002404EB84010A
:1049700001EB0803D9F8001057F82400194101F0A1
:104980000101013403F0D6FD052CEFD12B68012184
:1049900056F82300FEF7A2FD2B68002156F82300ED
:1049A00003F0C8FD2B68013393FBF4F404EB84049B
:1049B0001C1B2C6003E0FFF7F5FE002895D1BDE835
:1049C000F883002B97D11360BDE8F843FFF7E4BCF0
:1049D000706D0120606D0120746D01205C6D0120FF
:1049E00018C4000064C700000003005008C700009E
:1049F00008D200004FF0FF30FFF7F4BC024A034832
:104A0000092100F0EFBE00BF1CC7000078C70000FE
:104A10004FF0805310B51A69094B0224C3F80445BE
:104A200022F00302884203D30022C3F8042510BDFC
:104A3000D3F80044002CFBD0C3F808051044F1E77C
:104A400000E00140002815BF4FF4D2214FF4B421FB
:104A50004FF4B4204FF49620FFF7DABF00280CBFC4
:104A60004FF496234FF4B4231868030E532B0CBF56
:104A700020F07F4000207047064B0122C3F8042538
:104A8000D3F80024002AFBD000220160C3F80425DB
:104A9000704700BF00E00140002821F07F4141F055
:104AA000A6410CBF4FF496204FF4B420FFF7E4BFAB
:104AB0000A4B30B50124C3F80445002903DC002269
:104AC000C3F8042530BD52F8044BD3F80054002D30
:104AD000FBD040F8044B0139EFE700BF00E0014094
:104AE00038B54C68023405460A462146FFF7E0FF18
:104AF00005EB840038BD0000124B1B68002B0BBF78
:104B00004FF4B4224FF4D2224FF496234FF4B4233F
:104B100028B91A1DDB79522B08BF10467047824214
:104B20000DD9C378522B0AD14368023300EB8300BE
:104B3000824204D9C378522B18BF0020704700204E
:104B4000704700BF786E01202DE9F0410020B4B01D
:104B5000FFF7D2FF0024DFF8A4800546274626464B
:104B60004DBB224D2868FFF779FF3B463246CDE921
:104B700000401F4902A806F0F5F802A801F087F8E6
:104B80001C4B1A682B68002B0CBF4FF496234FF474
:104B9000B423D21A4FF4704164235343009193FB22
:104BA000F1F302A8144906F0DDF802A801F06FF84D
:104BB00034B0BDE8F08169682A6801918B1C1F44FC
:104BC000D1B2C2F307239C42C2F30742009102A86C
:104BD0004146B8BF1C4606F0C5F802A801F057F8D8
:104BE0002846FFF789FF01360546B9E7786E0120B0
:104BF00082C800007C6E01202CC800006EC8000036
:104C000070B50020FFF72AFF05460120FFF726FFB9
:104C10000C4B1E68B6FA86F485424FEA5414B8BFAE
:104C2000054620461C60FFF70DFF074A074B002E84
:104C300018BF1346064A691C2046BDE87040136041
:104C4000FFF72ABF786E012004B0040004A005001D
:104C50007C6E012070B50020FFF700FF02460120A6
:104C6000FFF7FCFE1F4E204C054672B968B94FF4A1
:104C7000D2214FF49620FFF7CBFE01212846FFF703
:104C80000BFF1A4B3560236029E0AA4208DD0023A0
:104C90003360164B23604FF4B4212368002017E0E3
:104CA00001233360124B23604FF4D221F5E7120E3B
:104CB000522A08D000B123600E4800F0E8FFBDE89A
:104CC0007040FFF79DBF5A68023203EB8203012058
:104CD0008B4205D21A68551CE9D10028D3D170BD8A
:104CE0002160FCE7786E01207C6E012004B0040096
:104CF00004A0050047C8000010B50020FFF7FCFE27
:104D0000014608B9084610BD8478FFF7F5FEDA2C95
:104D100008BF0146F5E700002DE9F04F4FF480721F
:104D20009FB05F4C5F48002105F0C2FC4FF48072D9
:104D300000215D4805F0BCFCD4F80090B9FA89F870
:104D40004FEA58184046FFF77DFEA246574B584C95
:104D50000020B9F1000F08BF1C46FFF7CDFF064643
:104D600038BB4846FFF77AFE524D411C4046FFF7DC
:104D700093FECAF800802C60FEF736FEDAF80030A9
:104D80002A68002B0CBF4FF496234FF4B423D21A99
:104D90004FF4704164235343009193FBF1F305A852
:104DA000454905F0DFFF05A800F071FF1FB0BDE821
:104DB000F08F3568C5F30743A3F10A02092AC5F34A
:104DC000072546D8374B595D91BB10223B48DFF889
:104DD000ECB005F06DFC37463A68C2F307218D420E
:104DE00009D1C2F307410B2926D013292BD00A2958
:104DF00001D1CBF800703846FFF77EFE0746002849
:104E0000EAD12E4F396881B12046FFF769FE0123B0
:104E1000044657F8231029B120460393FFF760FE9C
:104E2000039B04460133042BF3D11E4A012353553F
:104E30003046FFF761FE92E7D2B2022ADBDC0BEBD1
:104E400082025760D7E710220021584605F030FC57
:104E5000D1E7A3F11502082AEAD8134A525D002AC5
:104E6000E6D1152B0CBF3146002130460368C3F351
:104E70000742152A0ED01D2A08BF0021FFF73CFE6D
:104E80000028F3D119B12046FFF72AFE044601237A
:104E9000054ACCE7C3F307239D4208BF0146EDE76F
:104EA000786E0120786D0120806E012004A005003D
:104EB00004B004007C6E012011C80000E88F0120BE
:104EC000FFF72ABF2DE9F84FDFF8A8B0274F0333CB
:104ED0009246042293FBF2F6DBF80030B41C002B60
:104EE0003B684FEA84040CBF4FF4B4224FF4D22243
:104EF00023449A4281460D46B84614D2FFF70CFF70
:104F0000DBF80030002B3B680CBF4FF4B4224FF4A9
:104F1000D22223449A4206D2154800F0B8FE002758
:104F20003846BDE8F88F2D025FFA8AF141F0A441BE
:104F3000ADB2D8F800700D434FEA094101F47F018A
:104F400029433846FFF798FD07F108053146381D1B
:104F5000C8F80050FFF790FD1EB10A9A2846FFF7E7
:104F6000A7FD083C2544C8F80050D9E77C6E012015
:104F7000EBC70000786E012030B59BB0FFF76AFEEA
:104F800000214FF4FF621D4805F092FBFFF7B4FECD
:104F90001A490024A0B9194B024653F8301001B148
:104FA00001320130FF28F8D1154901A805F0DAFED9
:104FB00001A800F06CFE134800F069FE1BB030BD84
:104FC0000368C3F307420A2A0BD1C3F30722FF2A5F
:104FD00004D001EBC20541F832002B71FFF78CFDC4
:104FE000D8E7132AFAD1C3F30723FF2B1EBF01EB27
:104FF000C30241F833401471F0E700BF608601201E
:10500000B7C80000CBC800000A4B0022C3F800213B
:1050100001225A60D3F80021002AFBD00022C3F8F5
:105020000C2101229A60044B0222C3F880211A60ED
:10503000704700BF0010004000E100E0074B022273
:10504000C3F88020064B0022C3F8102101221A6108
:10505000D3F81021002AFBD0704700BF00E100E028
:105060000010004008B504490A780AB1FFF7E6FFCE
:105070000020087008BD00BF816F01204FF08053F1
:10508000586E400040F0010070470000024B186865
:10509000400040F00100704704700120024B186886
:1050A000400040F00100704724000020024B1868C7
:1050B000400040F0010070470870012070B50446C0
:1050C0000D461646FEF7F6F94FF0805301225B6E4F
:1050D0006270E270020A23F00043A271020CE271D6
:1050E0001A0A002160716372000EA2721A0C1B0E64
:1050F0002670A17025712072E272237370BD0000CA
:1051000010B5054C204605F073FE01462046BDE86B
:105110001040FEF7F8BE00BF0D700120104B1B6859
:105120005A1C10B514D0CBB1012B13D0022B13D0C5
:10513000042B13D00B4C0C4A052B08BF14462046F9
:1051400005F056FE01462046BDE81040FEF7DBBEE6
:10515000064CF4E7044CF2E7054CF0E7054CEEE7AB
:105160002800002061C9000067C900005CC9000078
:105170001BC1000014C1000010B521480278002AAC
:105180003DD14FF08043C3F8002101221A60D3F8CB
:105190000021002AFBD01B4B1B4C00220721C3F827
:1051A0000C25C3F808151949C3F81025C3F81C15B8
:1051B000C3F824250121C3F82C250822C3F8301593
:1051C000C3F81425C3F818450224C3F834454FF634
:1051D000FF74C3F83C450E4CC3F838451824C3F897
:1051E0005445C3F80423D3F8002242F01002C3F858
:1051F0000022084AC3F80425FFF706FF017010BD1E
:10520000816F012000100040200004027469627563
:1052100021100100826F0120F8B5104B1B78044665
:105220000BB9FFF7A9FF0E4E3378ABB10D4A1278D8
:10523000D21A02F003010C4A02EB411202F12007DC
:1052400010685168254603C50832BA422C46F7D18A
:10525000013B33700120F8BD1846FCE7816F012047
:105260000C700120806F0120826F012030B5002872
:1052700089B02ADD0D6815F0010426D1042D26D948
:105280002B6803F00F03092B21D16B683F2B1EDD28
:105290006846FFF7C1FFB0B19DF800200435A24277
:1052A000A8BF1DF8043004F10104A6BF5B0043F061
:1052B00001030123202C45F8043FF0D1054BDDF814
:1052C00009201A60042009B030BD0020FBE7204609
:1052D000F9E700BF0870012030B5384B1B788BB060
:1052E0000BB9FFF749FF02A8FFF796FF10B900209E
:1052F0000BB030BD9DF808300B2BF8D99DF8093064
:10530000012BF4D19DF80B30012BF0D12C4D2D4CFD
:105310002D4ADDF8111000232B6023709DF80C300E
:1053200013602A4A116023B9DDF815302B60002381
:105330000FE0012B11D1DDF815309DF819202B60FD
:105340000DF11A010E239342A8BF134600229A4280
:1053500030D10022E2540420CAE7022B05D19DF887
:10536000152012230DF11601EDE7042B0DD10AAA29
:105370006B4652F8130D516803C3DDE9000103F0D9
:1053800025F905F0DBF82860D1E7052BCFD10AAA73
:105390006B4652F8130D516803C3DDE9000103F0B9
:1053A00015F905F0CBF89DF81D2028600A230DF1B2
:1053B0001E01C8E7885CA0540132C8E7816F012054
:1053C000047001200D7001202800002008700120C9
:1053D00010B5154B1B7804460BB9FFF7CDFEFFF750
:1053E0002DFE124B0022C3F80445C3F80021012210
:1053F0001A60D3F80021002AFBD00022C3F80C2148
:1054000001229A60094AD2F80C31002BFBD0084BDC
:105410001978084B03EB4113C2F80435FFF70EFE71
:10542000BDE81040FFF7F0BD816F01200010004083
:10543000806F0120826F012000B5002889B01DDD3A
:105440000B6813F0010219D1042B17D9196801F068
:105450000F01092912D159683F290FDD043353F890
:10546000040F10F0010118BFC0F347010DF802103E
:105470000132202AF3D16846FFF7AAFF002009B0C5
:105480005DF804FB002810B511DD0C68E3070ED5AC
:105490006410532C0BD8074B1B780BB9FFF76CFE2D
:1054A000FFF7CCFD044BC3F80845FFF7ADFD002026
:1054B00010BD00BF816F012000100040002810B512
:1054C0000DDD0C68E3070AD56410FF2C07D8054BE7
:1054D0001B780BB9FFF750FE034BC3F8244500209F
:1054E00010BD00BF816F012000100040002813B5DF
:1054F00015DD0C68E10712D564100A4A0A4B072C27
:10550000CDE900230BD8094B1B780BB9FFF734FE0C
:1055100002AB1C44064B14F9082CC3F80C250020E0
:1055200002B010BDE2ECF0F4F8FC0004816F012041
:105530000010004070B5002888B020DD086810F029
:1055400001041CD104281AD9036803F00F03042BAB
:1055500015D1FEF7BBFA064605F04AFC122828BF13
:105560001220054600F10D0202216846FFF7A6FD54
:105570008DF80D50A54205DC6846FFF729FF002095
:1055800008B070BD0DEB0403325D9A730134F1E78E
:105590002DE9F041012888B00D4630DD086810F093
:1055A00001042CD104282AD9036803F00F03042B2B
:1055B00025D14B68DB0722D5FEF788FA804605F037
:1055C00017FC6D680E2828BF0E206E10074600F1EC
:1055D000110201216846FFF771FD6B128DF80D6015
:1055E0006D14360E8DF80E308DF80F508DF810605A
:1055F0008DF81170A74206DC6846FFF7E9FE00202F
:1056000008B0BDE8F0810DEB040318F804209A748B
:105610000134EFE730B5002889B016DD0C68E307E8
:1056200013D56510684610220021FFF747FD63126D
:105630008DF80D5064142D0E68468DF80E308DF8DF
:105640000F408DF81050FFF7C3FE002009B030BDA9
:10565000174BD3F8002122B10022C3F80021012208
:105660009A60D3F80C2102B30021C3F80C11D3F8CF
:105670000024012A0F4A19D1D3F848355B42136040
:105680000D4A1378032B9CBF013313700B4A137818
:10569000013303F003031370094A02EB4313044A76
:1056A000C2F80435024B01229A6070471160F9E795
:1056B00000100040240000200C700120806F0120A9
:1056C000826F0120024A0348102100F08BB800BF0E
:1056D000DCC80000D3C80000044A05491368C85458
:1056E0000133C3F309031360704700BF3C7401200A
:1056F0003C70012070B51149114A0B68834202DCED
:1057000000230B6017E0855CA5F1FA06012E00F17D
:10571000010405D89C420FDAA55C013D1F2D01D97B
:105720002046EBE70446151A165D2E550134A342B8
:10573000FADC181A086070BD1570FAE74878012085
:105740004874012008B5FDF7ADFE074B1A68824288
:1057500084BF00221A601B68C01A44F62063984276
:1057600094BF0020012008BD3870012070B5094C9D
:10577000094D0A4E23682A68934200D170BDF05C3F
:10578000FEF72CF90028F9D023680133C3F309038D
:105790002360EFE7407401203C7401203C7001203D
:1057A00070B5074E074D044633682A689B1ADB43E1
:1057B000C3F30903A34200DB70BDFFF7D7FFF3E794
:1057C0003C7401204074012010B5FFF795FA04469F
:1057D00008B9204610BD83781D2B08BF0446FFF78B
:1057E0008BF9F5E7F0B5074D2B680B2B08DC064F5E
:1057F0000C245C433E19C6E90112013338512B6079
:10580000F0BD00BF44740120F88F012008B5FBF7FC
:105810008BFDFFF7F3F8FBF7ABFDFEF759F8FEF74A
:105820002DFDFEF767FDFFF74DFF01F0D5F801F004
:1058300007FD01F031FDBDE8084001F067BF000041
:1058400008B54FF416620021034804F031FF034B02
:1058500000221A6008BD00BF007D0120AC050020B9
:10586000174B53F83000836803F07F031C2B70B58F
:105870000D46144601D0002070BDC36803F07F02BE
:10588000042AF8D1026902F07F02192AF3D11B0A17
:1058900000EB83001030FEF719F90378064633B1A8
:1058A00005F0A6FAA042E6D10023A34201DB0120C5
:1058B000E2E7F15CEA5C9142DDD10133F5E700BF3C
:1058C00060860120064B074A1B6812689B1ADB435F
:1058D000C3F309038342D4BF00200120704700BFF7
:1058E0003C74012040740120F8B507460E4614466A
:1058F0001D4673B90320FFF7E5FF10B3FA20FFF749
:10590000EBFEF8B2FFF7E8FEF0B2BDE8F840FFF7B3
:10591000E3BE501DFFF7D6FF98B1FB20FFF7DCFE7A
:10592000F8B2FFF7D9FEF0B2FFF7D6FEE0B2FFF70C
:10593000D3FEC4F30720FFF7CFFE2E46731B9C4215
:1059400000DCF8BD16F8010BFFF7C6FEF6E7000015
:10595000F8B50C4E0C4D0024F0273368A34203DC4D
:10596000BDE8F840FFF76CBF07FB04F359195B5D16
:105970002BB100231A4649781120FFF7B5FF0134F7
:10598000EBE700BFAC050020007D0120F8B50E4C10
:105990000E4E07460025BC4205F1010511D02378C3
:1059A00053B100231A4661781120FFF79DFFF022C2
:1059B0000021204604F07CFE0A2D04F1F004EAD117
:1059C000F8BD3560F8E700BF007D0120AC05002080
:1059D0002DE9F04F12F00106ADF54F7D82468B4662
:1059E00017D001238DF8143042FA03F354128DF8C6
:1059F000153052141B0E8DF817208DF818308DF8C5
:105A0000164005AB0522FFF76FFF0DF54F7DBDE892
:105A1000F08F042A2CD9116801F00F03042B38D120
:105A200005AD022310462B70FEF750F8044605F032
:105A3000DFF9B0F5487F034604F1FF31A8BF4FF40A
:105A400048739E4206F101020DD1B0F5487F06D998
:105A50006D4B19889B78ADF832138DF834332B4693
:105A600059465046CFE7164611F8012FAA55E8E7E8
:105A700040F0C680A2F1040CDCF100024FF00303F9
:105A800042EB0C028DF814308DF8152005AB022284
:105A9000E6E7092B40F09180154604238DF8143079
:105AA00055F8043F4FEA6308B8F1200F8DF81580D0
:105AB0004FEA6323A8BF4FF020088DF816308DF809
:105AC000178006AC03220521B04502DC05ABE21AC3
:105AD000C6E755F8040F10F0010706D1042847D98E
:105AE000036803F00F03022B0DD14FF00103237065
:105AF0004310637047121B0E4014A770E0702371AF
:105B000005340136E0E7042B30D123464FF0020C78
:105B100003F802CBCDE9012100930393FDF7D6FFF3
:105B2000814605F065F90C28DDE901210AD8009BC2
:105B30006070874201D1DC19E3E719F80740DC55B2
:105B40000137F6E723460C2003F8010F09F1FF3077
:105B500009F1080910F8017F03F8017F4845F9D1E0
:105B60002E23E372237363730E34CAE7012B08D12B
:105B70002346071F03F8022B7842784160701C46C9
:105B8000BFE7092B09D104232370436858106070C4
:105B90005B12A370E7700434B3E7032B0AD12170C2
:105BA0000368C3F30F10C3F34173C3EB8003637047
:105BB0001B12EEE727700134A3E7032B7FF425AF18
:105BC00005238DF81430C1F30F13C1F34171C1EBFC
:105BD000830164294FEA21238DF81510A8BF6421A1
:105BE0008DF816308DF8171003328E4205AB01DBAD
:105BF0000A1D35E7334412F8010F18710136F4E736
:105C0000002A7FF402AF35E780BD00000F4970B570
:105C1000F022002402FB04135D78854203D0013496
:105C20000A2CF7D170BDF0221846002104F040FD87
:105C3000074A1368013BA34200D1146000232946A0
:105C40001A461120BDE87040FFF74EBE007D0120CE
:105C5000AC05002030B5B3B032AC0223054604F8E1
:105C6000C83D05F0C5F8C72828BFC720691E002316
:105C7000984207DC421C2346FE211420FFF734FE25
:105C800033B030BD013311F8012FE254F0E770B5A5
:105C9000B2B032AC0223054604F8C83D05F0A8F8BE
:105CA000C72828BFC72006460023681E9E420BDC7B
:105CB00006F13200FFF774FD2346721CFF21142009
:105CC000FFF712FE32B070BD013310F8012FE2541D
:105CD000ECE700002DE9F04F0128B9B08146884675
:105CE00003DC1B20FBF7DEFC57E00868C20729D461
:105CF000042827D9036803F00F03042B22D1FDF7F2
:105D0000E5FE0546D8F80400C3071DD404281BD9B6
:105D1000036803F00F03042B16D1FDF7D7FE0646E8
:105D2000204B1B6803930027039BBB420EDC0096AD
:105D30002B461D4AC82106A804F0E0FF06A8FFF77D
:105D4000A6FFCEE7194DDDE7184EE9E70C237B43AC
:105D5000174A2946985803EB020B05F03FF8044612
:105D600018B9DBE9013A9C4201DB0137DCE70AEBB9
:105D7000C40231465AF834000593049205F02EF817
:105D8000DDE90423834658B9536808F10801A9F1F5
:105D900002009847074BC3F800B039B0BDE8F08F58
:105DA0000134E0E74474012038CA000032C2000028
:105DB000F88F0120546D01202DE9F0411F4F204A3A
:105DC000D7F8008005460023F02098450EDC00241B
:105DD000F02000FB04F15318565C8EB101340A2CFC
:105DE000F7D11848BDE8F041FFF751BF00FB03F1C0
:105DF00054186478AC4201D1515CE9B90133E4E74D
:105E0000F0223146184604F053FC0F49457051F812
:105E1000351085700222A0450270C0E90212C0E967
:105E2000046601DC01343C60002329461A46102038
:105E3000BDE8F041FFF758BDBDE8F081AC0500209A
:105E4000007D012081CE00006086012070B5FFF743
:105E50007FFD094EFF246FF0070505FB046393F8EF
:105E6000FC37043B012B03D8E043C0B2FFF7A4FF8B
:105E7000013CF2D170BD00BF608601202DE9F041E8
:105E800006460F46FEF73FF80D4BDFF838801860E6
:105E9000002408EBC4031B79062B01D0032B09D186
:105EA000E5B23A4631462846FFF7DAFC10B12846FB
:105EB000FFF782FF0134FF2CEBD1BDE8F08100BF7A
:105EC0000800002060860120F8B5094F0546FF2430
:105ED0006FF0070606FB047393F8FC37AB4203D15F
:105EE000E043C0B2FFF768FF013CF3D1F8BD00BF4B
:105EF000608601202DE9F84FFDF7D4FA584B1A6857
:105F0000824284BF00221A601A6842F20F71821A1C
:105F10008A420BD95349186000235A181279073A5C
:105F2000022A0FD90833B3F5FF6FF6D1BDE8F88F19
:105F30000720FFF7C9FF8AF800802EE00820FFF74E
:105F4000C3FF3FE0FDF7B6FA002814BF0446012462
:105F50000020FDF79BFB81460020FDF7ABFB424D87
:105F6000424E0746B9F1000F17D02B68002B70D1B5
:105F700033682C60002B6FD0DFF8F8B0DFF8F0A0AA
:105F80009BF800304FF00108002BD1D10920FFF71A
:105F90009BFF8AF800808BF80080AFB133689BB913
:105FA0002B6834601BB3DFF8C8B0DFF8C8A09BF8DB
:105FB00000304FF00108002BC0D10920FFF784FF0B
:105FC0008BF800808AF800802B6883B1284A11780A
:105FD000904661B99C4238BF2C602B68E31A312B84
:105FE00005D90720FFF770FF012388F800303268D9
:105FF00082B1204B1978984661B9A24288BF3460BB
:106000003368E41A312C05D90820FFF75DFF01231E
:1060100088F800302B685BB1B9F1000F08D1144C3F
:10602000227812B90720FFF74FFF00232B6023705F
:106030003368002B3FF47AAF002F7FF477AF0D4C1D
:10604000227812B90820FFF73FFF00233360237046
:106050006CE7002FA2D1B9E7002FA1D1B4E700BFB0
:106060003470012060860120247001202C700120F2
:10607000287001203070012037B50546FFF768FC15
:1060800002A8002440F8044DFDF7E8FA2146204616
:10609000FEF798F9FEF712FCFDF720FBFDF7F4FB85
:1060A000FDF70EFCFEF7A6FCFDF726FA25B1FDF77D
:1060B000BDFC0248FFF7EBFD03B030BD72CE00001F
:1060C000002301461A461120FFF70EBC07B5131234
:1060D0008DF801208DF802301314120E8DF8001087
:1060E0008DF803308DF8042001466B4605221320FD
:1060F000FFF7FAFB03B05DF804FB0A4601461220E5
:10610000FFF766BC70B505460C46FDF7DFF958B1E0
:1061100004F13200FFF744FB2B46224600211B20EE
:10612000BDE87040FFF7E0BB70BD10B414460346F5
:106130000A46142021465DF8044BFFF7D5BB00004A
:1061400030B5084C01444FF0FF33884201D3D843A7
:1061500030BD10F8015BDAB26A4054F8222082EABE
:106160001323F2E754CA0000FE2837B5044614D8BA
:106170000B4B53F8300080B1416808308900FFF7BD
:10618000DFFF02AD45F8040D0920FFF709FB2B46A0
:10619000042221461720FFF7A7FB03B030BD00BF44
:1061A00060860120F8B50746FFF70EFB4FF0FF357C
:1061B00004460CB92846F8BD2668C6F30743152BDC
:1061C0000CD104F10801384604F008FE08B9C6F302
:1061D00007252046FEF790FC0446EAE71D2B08BF82
:1061E0004FF0FF35F5E700002DE9F047BF4CC04DFB
:1061F0009CB0FFF7BBFA2068C0F580612844FDF72A
:10620000D5FB23680344064623607BB1B94F002EBB
:106210000FDC2B78FA2B40F030812368022B16DC40
:10622000FFF790FA10B10120FFF764FA1CB0BDE847
:10623000F0872068C0F580612844FDF7B7FB23682C
:10624000034406462360FDF72DF93860DFE76878E0
:10625000AC78831E182B00F20681DFE813F01900DA
:106260002D00310035003800410004014B00800052
:106270008A008E00A400E000F10004010401040182
:106280000401040104010401040104010401FF00EC
:10629000FF2C0FD02046FFF7B9FC974A002342F8A5
:1062A000343002EBC40221461371132000931A46C6
:1062B000FEF708FE0320B7E72046FFF77DFDF9E76C
:1062C0002046FFF7A3FCF5E7FFF7C0FDF2E7FFF775
:1062D0003FFB0020FFF7D0FE8848FFF7D8FCE9E736
:1062E000632CE7D8864B214653F824201520FFF76E
:1062F0006FFBDFE7FFF768FA6FF007080446002C32
:10630000D8D02768C7F30743152B04D02046FEF7E3
:10631000F3FB0446F3E704F10806304604F068FD99
:1063200005460530FFF73CFAFB20FFF7D5F91D20A5
:10633000FFF7D2F9C7F30720FFF7CEF9E8B2FFF76E
:10634000CBF9C5F30720FFF7C7F9A8EB0407F3194A
:106350009D42DBDD16F8010BFFF7BEF9F7E70023DE
:1063600000931A4619461D20FEF7ACFDFDF75EFBB3
:10637000A0E72046FFF7F8FE9CE7FDF7A9F8614A81
:1063800000906421604B03A804F0B8FC022303A82A
:106390008DF80C3004F02CFD03AB024600211620D2
:1063A000FFF7A2FA86E7544F002557F8354007EB70
:1063B000C5035CB3D4F8048093F804A04FEA8806C0
:1063C000B01DFFF7EDF9FB20FFF786F9012006F17C
:1063D0000109FFF781F9E8B2FFF77EF95FFA89F06A
:1063E000FFF77AF9C9F30720FFF776F95046FFF770
:1063F00073F9083404EB0609A1450BD8FFF7B6F989
:1064000006EB080001F0C4FEFFF7B0F90135FF2DDF
:10641000CBD14FE714F8010BFFF75EF9ECE700244E
:10642000FFF796FA2246214600942346DA20FEF72B
:1064300049FD4FF4FF6221462F4804F039F995E7F2
:10644000012C02D1FEF780FB34E7022C02D1FEF7CB
:1064500037FD2FE70120FFF70FFE2BE700231A4639
:1064600021461A209CE7A0F1C803052B3FF622AF76
:1064700000221146FAF786FF1CE7FB2B7FF4D3AE10
:106480002268042A7FF7CCAEB5F8037040F2F633E9
:106490009F423FF7C8AE3B1D9A427FF7C1AEEB5C0F
:1064A000FE2B7FF4C0AE6878AC781B2807F1FF366E
:1064B0007AD02DD807285ED0082837D001282CD1D3
:1064C000FF2C11D02046FFF7A1FB6D790F4B0093F5
:1064D0002146BB1E2A460A20FEF7F4FC064B43F871
:1064E000340003EBC4042571781D9DE64878012033
:1064F00048740120387001206086012054CE0000CD
:10650000588E01206BCE000066CE00004E74012034
:106510001D285BD04DD31E2870D0A0F1C803052BD9
:10652000E2D83F4A3146FAF72DFFDDE7632CDBD88E
:106530006B79022B0CD0032B14D0012BD4D1D5F8BE
:106540000630384A5B0043F0010342F82430CBE7C1
:10655000002EC9DDB91E3448FDF7D5FC314B43F898
:106560002400C1E7AB79002B2E4B0CBF0022042284
:1065700043F82420B8E7632EB6DC3246284903A846
:1065800004F072F81CAB1E4403A8002306F8643C18
:10659000FFF708FE0028A7DB224B214653F82020F6
:1065A0001520FFF715FA9FE731461D48FFF766FCF7
:1065B0009AE7FF2C98D06A79022A95D81A4B009353
:1065C0002146BB1E0B20FEF77DFC8DE7632EA8BF86
:1065D0006326002303A9B3420BDB1CAA26EAE67359
:1065E0001344002203F8642C15200091731C2146EB
:1065F000E9E7EA185279CA540133ECE7012C7FF439
:1066000073AF002E7FF770AF6B791BB1322BA8BF31
:1066100032231C4664235C43044B1C6064E700BFC8
:106620004D740120588E01204E740120040000207A
:10663000084B01221A60084A1368002BFCD0074B54
:106640001868042390FBF3F00638400040F0010086
:10665000704700BF00C0004000C1004008C50040B6
:106660000120704710B5064C204601F065F9054938
:10667000204601F0C7F9044B01221A6010BD00BF8B
:10668000087B0120801A06004C78012010B5064CCA
:10669000204601F051F90549204601F0B3F9044BB9
:1066A00001221A6010BD00BFC47B0120801A0600C1
:1066B000507801201FB500210E20FCF70FFF0121AB
:1066C0000F20FCF70BFF01210D20FCF707FF1D48F1
:1066D00001F08AF81C4B1D491B681D4A8B42127839
:1066E0000FD84FF000730193002303938DF8082017
:1066F00004AB13E90E00134805B05DF804EB01F09C
:1067000089B814498B4202D84FF08063EBE71249F5
:106710008B4202D84FF00063E5E710498B4202D864
:106720004FF08053DFE70E498B4202D84FF0005301
:10673000D9E70C498B4294BF4FF080434FF00043A0
:10674000D1E700BFE87A01203000002048E80100CE
:106750002C00002090D0030020A1070040420F0031
:1067600080841E0000093D00002814DD0B68DA0754
:1067700011D50D4A5B10012813600C4A09D04B68F3
:10678000D90706D55B10022B09D0032B09D0012BAA
:1067900003D002231360002070470023FAE703238D
:1067A000F8E70123F6E700BF300000202C000020AE
:1067B0002DE9F8430C68E30704D40D20BDE8F84345
:1067C000FAF770BF64102FD4FCF786FEA0422BDBD3
:1067D00000212046FCF782FE4FF4FA620121204698
:1067E00001F00EFD00B3DFF86C8000254FF00109C9
:1067F000002707264FF47A720121204601F000FDA0
:1068000090B12828C4BF09FA06F31F4316F1FF36DA
:10681000F0D205F808700135052DE9D101220621D5
:106820000920FDF7EFFA08B900200FE003460B221C
:1068300043F8042F064900F1180411F8012F520003
:1068400042F0010243F8042F9C42F6D1BDE8F883E0
:106850005378012054780120F0B5002885B00C460B
:106860002DDD0B6813F0010529D1042B27D91B68F6
:1068700003F00F03032B22D14FF000730193039514
:106880008DF8085004AB13E90E000E480D4F00F0D0
:10689000C1FF266856F8033BC3F30F14C3F34173DB
:1068A000C3EB8404AC4207DD16F8011F384600F044
:1068B000BEFF01353070F5E7024800F0B7FF002059
:1068C00005B0F0BDE87A012010B50468E30704D4F0
:1068D0000D20BDE81040FAF7E5BE6410FF2C01D989
:1068E0001720F6E7FFF7E6FEE1B2044800F09FFF4D
:1068F000024800F09BFF002010BD00BFE87A012095
:1069000038B5074DFFF7D6FE0021284600F08FFF6F
:106910000446284600F08AFF600040F0010038BDC0
:10692000E87A0120274A82B001210023ADF8063021
:10693000C2F8F015C2F8001519461A0102F180429A
:1069400002F5E0420133082BC2F81415C2F8101505
:10695000F3D11C4B4FF4E062C3F818250422C3F8AE
:106960001425C3F810250DF10602C3F82C260122C8
:10697000C3F830261A60D3F80021002AFBD0002289
:10698000C3F8002101225A600E4B1A46D3F80411B5
:106990000029FBD00021C3F8041101219960D2F82D
:1069A0001431002BFBD00020C2F81401C2F80005FE
:1069B000BDF806301BB28342C8BFA3F50B70400080
:1069C00002B070470070004008B5FFF7ABFF400011
:1069D00040F0010008BD0000024A03480D21FEF707
:1069E00001BF00BF98CE000000CF000070B5066860
:1069F000F10705D54568EA0702D58468E30704D4A2
:106A00000D20BDE87040FAF74DBE7610802E01D9FA
:106A10001520F6E76D10FF2D01D91620F1E764105F
:106A2000FF2C01D91720ECE70A4B1B680BB9FFF7C5
:106A300019FEF1B2084801F063F8E9B2064800F027
:106A400043FFE1B2044800F03FFF034801F0C3F800
:106A5000002070BD4C780120087B01200C4B1B6886
:106A600070B506460D4614460BB9FFF70FFEF1B29E
:106A7000084801F045F8E9B2064800F025FFE1B208
:106A8000044800F021FF0348BDE8704001F0A3B8BE
:106A900050780120C47B012001282DE9F0415EDD02
:106AA0000D68EA075BD52F4B4C681B686D100BB95E
:106AB000FFF7D8FDE9B22C4801F022F814F00106E6
:106AC00013D06410FF2C02D91720FAF7EBFDE1B2C6
:106AD000254800F0F9FE244801F07DF818B1232084
:106AE000FAF7E0FD0020BDE8F081042CF3D923681B
:106AF00003F00F02092A1AD154F8047FDFF86880E6
:106B00007F10B742E7DD54F8045FEB070BD56D103B
:106B1000FF2D02D91720FAF7C5FDE9B2404600F073
:106B2000D3FE0136EDE71720FAF7BCFDF9E7032A9B
:106B3000D1D1261DC4F1FF24C3F30F1504F57F0442
:106B4000C3F34173084FC3EB8505FC343319AB42E3
:106B5000C1DA16F8011B384600F0B6FEF6E7012050
:106B6000C1E700BF4C780120087B012038B50468DC
:106B7000E20702D54568EB0704D40D20BDE8384094
:106B8000FAF790BD6410802C01D91520F6E76D103E
:106B9000FF2D01D91620F1E7124B1B680BB9FFF747
:106BA00061FDE4B22146104800F0AAFFE9B20E48A8
:106BB00000F08AFE00210C4800F0ACFF20B14042FA
:106BC000400040F0010038BD01222146064800F097
:106BD00094FF054800F06FFE0028F1D0024800F055
:106BE0006DFEEDE74C780120087B012038B5124B93
:106BF0001B6804460D460BB9FFF748FDE4B2214679
:106C00000E4800F07DFFE9B20C4800F05DFE0B4835
:106C100000F0E1FF08B1404238BD0122214607489B
:106C200000F06BFF054800F046FE0028F4D0034852
:106C3000BDE8384000F042BE50780120C47B0120FE
:106C400038B50D211D20FFF7D1FF5A28174C0CD164
:106C5000012222702A211D20FFF700FF022001F0EF
:106C600097FA134B01221A6038BD0F211920FFF744
:106C7000BDFF332805D1022323708F222021192044
:106C8000EAE70D211E20FFF7B1FFC7280AD103252F
:106C900000222A211E202570FFF7E0FE2A462A2125
:106CA0001E20D9E700232370D8E700BF340000205E
:106CB0005C780120002838B504DC1C20BDE8384091
:106CC000FAF7F0BC0B6813F0010401D10D20F5E7D1
:106CD0005B10012B2ADD022B03D0052BB4BF02244D
:106CE0000324194B1B680BB9FFF7AAFF174B93F945
:106CF0000050022D1CD0032D1ED0012D11D1032CCC
:106D000008BF022400222A211D20FFF7A7FE2246E9
:106D10000E211D20FFF7A2FE2A462A211D20FFF783
:106D20009DFE022001F034FA002038BD0024D8E78F
:106D3000220123211920F2E7032C14BF224602224C
:106D40000E211E20EBE700BF5C78012034000020FC
:106D5000204B1B6810B504460BB9FFF771FF1E4BA3
:106D600093F90030022B0AD0032B25D0012B26D11A
:106D700021461D20FFF73AFF4FF0FF3405E0012CBC
:106D800013D129211920FFF731FF7F28C8BFA0F5B3
:106D900080706FF07E039842B8BF1846C8235843EE
:106DA0007F2390FBF3F0604310BD032C0BD12B210C
:106DB0001920DFE72D21FBE721461E20DAE74FF0FF
:106DC000FF340020EAE7052CF4D04FF0FF34002018
:106DD000DFE700BF5C7801203400002008B5012007
:106DE000FFF7B6FF400040F0010008BD08B50320E2
:106DF000FFF7AEFF400040F0010008BD08B50520D8
:106E0000FFF7A6FF400040F0010008BD38B5134B66
:106E10001B6813B90120FFF79BFF114B93F900305A
:106E2000013301D1FFF70CFF0120FFF791FF04466A
:106E30000320FFF78DFF05460520FFF789FF6D430F
:106E400004FB045400FB004003F05EF801F0DAFCA0
:106E500003F074FB400040F0010038BD5C78012075
:106E6000340000200128F8B535DD0F68FB0732D566
:106E70004D6815F001062ED1042D2CD92B6803F096
:106E80000F03092B27D16C68144B64101B68202C4E
:106E9000A8BF20240BB9FFF7E5FBC7F34701224643
:106EA0000F480F4F00F029FE0435A64211DA0C48B6
:106EB00000F001FD18B9700040F00100F8BD38463F
:106EC00000F0FCFC400040F0010045F8040F0136E2
:106ED000EBE76000F0E70120F0E700BF4C7801200D
:106EE000087B01200A4B0B4A30B5D3F834450A4BD6
:106EF000A34208BF1346013B0246FF24151AA942CC
:106F000005DD13F8015F02F8015B1C70F6E730BD88
:106F1000008002406478012064790120064B012240
:106F20005A60DA60D3F85821002AFBD00022C3F857
:106F30000025024B1A6070470080024060780120F3
:106F400070B5104E04460D46002D14DDD6F82031E4
:106F500093B1802D10DC0C4B621914F8011B03F85F
:106F6000011FA242F9D1074B0022C3F84855C3F8CC
:106F7000202101229A6070BDFDF7A0FC012001F0E4
:106F800007F9E1E700800240637A012070B5174DF0
:106F9000174CD5F83435174E9C4214BF2346334660
:106FA0004FF480721846FF2103F082FB4FF4807388
:106FB000C5F83405C5F838350023C5F80831012374
:106FC0002B60D5F83405844208BF344604F1FF0035
:106FD000A21E0178FF2900F1FF3301D19A4202D1AC
:106FE000001B013070BD1846F3E700BF008002406F
:106FF0006479012064780120002838B504DC1C2065
:10700000BDE83840FAF74EBB0D68EB0706D4042DF7
:1070100004D92B6803F00F03032B01D02420EFE7E2
:10702000124B1B680BB92520EAE7114BD3F8083146
:107030000BB9012038BDFFF7A9FF041EF9D001DA12
:107040001B20DDE7284650F8043BC3F30F12C3F3BF
:107050004173C3EB82039C4228BF1C462146FFF7C5
:1070600041FF600040F00100E4E700BF60780120CC
:10707000008002400028F8B504DC1C20BDE8F84080
:10708000FAF710BB0968CB0701D40D20F6E71E4DB7
:107090001E4C2B68491023B1D4F800350BB1FFF713
:1070A0003DFF1B4B1A68C4F814255B68C4F80C3507
:1070B0004FF486734B43C4F82435164B4FF480725B
:1070C000FF21184603F0F4FA4FF48073C4F8340536
:1070D000C4F83835104BC4F844358023C4F848351B
:1070E0002023C4F80032002601270823C4F8003505
:1070F0000520C4F808612760C4F84865A76001F05E
:1071000047F82F603046F8BD6078012000800240CB
:1071100008D2000064780120647A012006490A68D8
:1071200008B52AB1054BD3F800350BB1FFF7F6FED1
:107130000020086008BD00BF607801200080024088
:1071400038B51C4B1B6823B92520BDE83840FAF739
:10715000A9BA194BD3F8083113B9184D284638BDD0
:10716000FFF714FF041EF8D001DA1B20EDE7E11C45
:10717000002289100320FCF745FE054608B90A20C5
:10718000E3E721460430FFF7ADFEEB07E6D4042D1C
:10719000E4D92A6802F00F03032BDFD104F00303C4
:1071A000C3F104035B0703F0C04322F0C042134362
:1071B0002B60D3E760780120008002403800002077
:1071C000002837B504DC1C20FAF76CFA03B030BD98
:1071D0001A4B1B680BB92520F6E7086810F001046C
:1071E00008D0431002A8012100F8013DFFF7A8FED6
:1071F0000020EBE7042813D9036803F00F02042AE8
:1072000010D1FCF763FC054603F0F2FD802801462F
:1072100003D92620FAF746FAEAE72846FFF790FE58
:107220002046D3E7032AFBD1C3F30F11C3F3417305
:10723000C3EB81018029ECDC0430EFE760780120AA
:10724000024A03480521FEF7CDBA00BF8CCF0000EB
:10725000B4CF000000207047012070470020704725
:1072600000207047002070470120704700207047C1
:1072700000207047002070470020704700207047B2
:1072800000207047002070470020704700207047A2
:107290007047704770470000024A03480F21FEF70D
:1072A000A1BA00BFD0CF000048D00000024610466F
:1072B00001320378013B1F2BF9D9704708B5FFF75E
:1072C000F5FF0378002B39D0222B00F1010011D1FA
:1072D000037823B1222B00F1010204D11046BDE84E
:1072E0000840FFF7E3BF5C2B02D1437803B1821C57
:1072F0001046EDE73A2BF2D02C2BF0D07B2B0BD1A4
:10730000FFF7D4FF0378002BE9D07D2B01D10130AA
:10731000E5E7FFF7D3FFF5E75B2B10D002461046F9
:1073200012F8013B002BDAD0202BD8DD2C2B05D016
:1073300003F0DF015D2901D0222BF0D108BDFFF75A
:10734000B5FF0378002BCAD05D2BE0D0FFF7B6FF66
:10735000F7E708B5F0B1FFF7A9FF0378222B1AD0A1
:107360007B2B1AD05B2B1AD0A3F13002092A05D946
:107370002D2B05D14278303A092A07D8032009E09D
:10738000742B0ED0662B0ED06E2B0ED0181C18BF8F
:107390000120404208BD0420FCE70220FAE701205A
:1073A000F8E70520F6E70620F4E70720F2E738B50E
:1073B000FFF77CFF03782D2B11D101304FF0FF3404
:1073C000431E00210A2501E005FB012113F8012FCE
:1073D000303AD0B20928F7D904FB01F038BD0124B6
:1073E000EEE710B51446FFF761FF0378222B02D0B9
:1073F00000230B7010BD621E01300378222BF7D0E2
:10740000002BF5D05C2B07D0441C002AF0DD01F8DE
:10741000013B013A2046F0E74378622B00F1020479
:1074200009D0662B09D06E2B09D0722B09D0742B92
:1074300008BF0923E9E70823E7E70C23E5E70A2368
:10744000E3E70D23E1E710B50446FFF737FF0346F6
:10745000A342184605D90278013A1F2A03F1FF33E7
:10746000F6D910BD08B590B1037883B1FFF71EFFC0
:10747000037803F0DF035D2B09D0FFF71FFF0378CC
:107480002C2B08BF0130BDE80840FFF70FBF0020DC
:1074900008BD38B50D1E0DDD03785B2B0AD1013018
:1074A000FFF704FF0124A54205D0FFF7DBFF10B171
:1074B0000134F8E7002038BD38B5154609B100237E
:1074C0000B70F8B10378E3B1FFF7F0FE03782C2BD3
:1074D000044603D10130FFF7E9FE044623787D2BF3
:1074E0000FD019B12A462046FFF77BFF2046FFF751
:1074F000E5FE03783A2B05D10130BDE83840FFF7AF
:10750000D5BE002038BD2DE9F0410D469AB00446A5
:107510002F789FB32E21284603F053FC804690B16C
:10752000461B303F092F13D82846FFF740FF01467E
:107530002046FFF7AEFF044604B3B8F1000F1DD09C
:1075400001363544E4E7284603F052FC0646E8E7F6
:1075500023787B2B11D1601C642201A9FFF7ACFFBB
:10756000044658B13246294601A803F049FC0028D8
:10757000E2D02046FFF7A2FEEEE7002420461AB034
:10758000BDE8F08138B50D1E04461CDDFFF7E1FEB5
:10759000012807D1601C012D00D138BDFFF762FF23
:1075A000013DF8E702280ED100221146601CFFF7CA
:1075B00083FF012DF1D0FFF755FF00221146FFF7A1
:1075C0007BFF013DF5E70020E7E7F8B50C1E074615
:1075D00015461E4613DDFFF7BCFE02280FD13246CA
:1075E0002946781CFFF768FF012C00D1F8BDFFF792
:1075F00039FF32462946FFF75FFF013CF4E70020E0
:10760000F4E710B50446C8B1FFF750FE03787B2BB2
:107610000AD10130002400221146FFF74DFF68B166
:10762000FFF74CFE0134F6E75B2B06D10130002456
:10763000FFF718FF10B10134FAE70024204610BD0F
:10764000002870B514DD0D68EB0711D56D10013DF4
:10765000FDF752FB00264FF0FF3460B916B33046F9
:1076600003F0C6FB01463046BDE87040FCF74BBC5A
:107670004FF0FF35ECE70368C3F30742152A0BD13F
:10768000C3F307239C42B8BF1C469D4201D100F1C1
:107690000806FDF731FAE0E71D2A04BF00264FF087
:1076A000FF34F6E7601C400040F0010070BD0000B0
:1076B00010B508680C46FCF709FAFEF773FD0028C0
:1076C000A2BF034B626843F82020002010BD00BF1A
:1076D000588E012008B50868FCF7F8F9FEF762FD3E
:1076E0000028AABF024B012053F8200008BD00BFAC
:1076F000588E012008B50868FCF7E8F9FEF752FD3E
:107700000028ACBF0420002008BD0000024A034846
:107710000421FEF767B800BFE4D00000DED000000F
:1077200008B5FCF7DFF8FCF7A5F9FEF76FF8044899
:10773000FEF7ADFAFDF720FCBDE80840FEF786BB7A
:1077400033D10000FBF736BD38B50025057329B9E4
:107750000B4B0C4A0C48252102F018FF01600B4925
:1077600051F82220027151F8233083719DF81030B6
:1077700051F8233043710223C371856038BD00BFC7
:107780004BD10000AAD1000059D1000008D200005E
:10779000037B23B94373837303610123037370472E
:1077A00084B00DF1100C0CE90E009DF80810026871
:1077B00000230129C2F80035039B12D00BD3032903
:1077C0000CD0C2F85435019BC2F824350123C2F80D
:1077D000003504B0704743F00203F2E743F00403BE
:1077E000EFE743F00603ECE710B5FFF7D1FF0368BE
:1077F0008279C3F808254279C3F80C250279C3F8C9
:107800001025034BBDE810400ECBFFF7C9BF00BFEA
:10781000FC7A012010B485B001AC84E80E0094E835
:107820000E0005B05DF8044BFFF7BABF7047036860
:10783000C3F81C15D3F80821002AFBD0D3F818058B
:107840000022C3F80821C0B27047000007B5094BF9
:1078500009490A484FF080421A6000229A600222C9
:107860001A710F2300930E220D23FFF76DFF03B053
:107870005DF804FBFC7A012000300240E87A012028
:107880002DE9F84380460D46174601EB02090C46E8
:107890004C45A4EB05060BD0D8F8003014F8011BBA
:1078A0001B68404698470028F2D13046BDE8F8836F
:1078B0003E46FAE77047203000F03CBA203000F036
:1078C0002BBA203000F03CBA38B5437F0D460BB9D7
:1078D000002038BD00F16804204600F039FA002885
:1078E000F6D12046294600F008FA0120F1E7000011
:1078F0002DE9F0411E4600254FF47A73C0E901538B
:107900000C4B044640F8203B8846174600F0ECF943
:1079100004F1680000F0E8F99DF8183063769DF8EE
:107920001C302676C4E90487A37665772046BDE837
:10793000F08100BFF0D10000F0B5837E2E4C2F4DBA
:107940000121C17654F82320437E54F8233012F0ED
:10795000200F14BF2F464FF0A04702F01F0213F074
:10796000200F03F01F0308BF4FF0A04502F5E0729F
:1079700003F5E07340F20C6647F8226045F8236097
:1079800003694FF0CC72C3F8242503690622C3F8BB
:107990000025827E036954F82220C3F80825427E20
:1079A000036954F82220C3F80C2590F91830144AC2
:1079B0005C0903F01F03994004F1600342F82310AF
:1079C00090F91830002BBDBF03F00F0302F6FC3214
:1079D000D2189B18B5BF40234022137683F80023AA
:1079E00090F918300122590903F01F0302FA03F33A
:1079F000034A42F82130F0BD08D2000000030050D5
:107A000000E100E0C37EA3B103690022C3F80025B2
:107A10000A4B99420ED90A4B994294BF4FF08061AC
:107A20004FF0C8610369C3F8241503690622C3F83F
:107A3000002570474FF0CC71F4E700BFA08601002D
:107A400090D003002DE9F041044688461F461546B4
:107A5000002A50D000F12006304600F059F9236981
:107A6000C3F88885236901221A622369C3F8346543
:107A70002369C3F8385523691A602269D2F84C315A
:107A80001BB9D2F82431002BF8D00023C2F84C31B6
:107A90002269D2F85C311BB9D2F82431002BF8D01E
:107AA0000023C2F85C3122696FB9D2F8243153B98E
:107AB0000123D3612369D3F84821002AFBD0002297
:107AC000C3F8482109E0012353612369D3F8042155
:107AD000002AFBD00022C3F804212369D3F8242113
:107AE00012B10022C3F824212369D3F83C05206693
:107AF000C0B2BDE8F0811046FBE70123FFF7A2BF4B
:107B000010B5044680F8B010683000F001F9012388
:107B1000637710BDF8B500234377036990F8B02070
:107B2000C3F88825036901261E62036900F1680510
:107B30000446C3F8445528460F4600F0FBF8236975
:107B4000C3F8480523699E602369D3F850211AB908
:107B5000D3F82421002AF8D00022C3F85021284667
:107B600000F0E8F8236930B1D3F860211AB9D3F8EE
:107B70002421002AF8D00022C3F8602123696FB9BC
:107B8000D3F8242152B90122DA612369D3F84821BC
:107B9000002AFBD00022C3F8482109E001225A61E3
:107BA0002369D3F80421002AFBD00022C3F8042162
:107BB0002369D3F8240168B10022C3F82421236982
:107BC000D3F8C404C3F8C404022803D004280CBFAB
:107BD00003200420F8BD0121FFF79CBF70B5436965
:107BE000D3F86421044692B10022012500F1200659
:107BF000C3F864210577304600F08AF86369C3F85A
:107C0000346563694022C3F8382563691D6363697D
:107C1000D3F86821DAB10025C3F8685104F1680689
:107C2000012363772577304600F072F8D4F8B4303A
:107C300003B19847636965773046C3F8446500F03F
:107C400079F86369C3F84805636901225A63636977
:107C5000D3F8042162B10022C3F80421237F3BB191
:107C60006369D3F83C05D4F8B830206603B198476F
:107C70006369D3F8242152B10022C3F82421636937
:107C8000D3F8D024C3F8D024636901225A6170BDAF
:107C90000148FFF7A3BF00BF087B01200148FFF7A1
:107CA0009DBF00BFC47B012007B514231322CDE97B
:107CB00000324FF04022114604230848FFF718FE17
:107CC000074A08481E231F21CDE90031032311462E
:107CD000FFF70EFE03B05DF804FB00BF087B012038
:107CE00000300040C47B012008B54022002102F092
:107CF000DFFC0022C0E9102208BD026C10B5531C45
:107D0000446C03F03F039C421CBF8154036410BDCC
:107D10000023C0E910337047D0E9102393421FBFFE
:107D2000C25C013303F03F03436414BF10464FF0BD
:107D3000FF307047D0E91030181A48BF4030704704
:107D4000D0E91023934214BFC05C4FF0FF3070475E
:107D5000036C406C013303F03F031B1A5842584137
:107D6000704700000649074A074B9B1A03DD043B96
:107D7000C858D050FBDC00F013F8F8F761FA0000A7
:107D8000B0D600000000002044020020FEE7FEE71D
:107D9000FEE7FEE7FEE7FEE7FEE7FEE7FEE7FEE7BB
:107DA000394B1A680D2A08D14FF080420021C2F8E1
:107DB0000C11C2F81011C2F838151B680D2B46D1F2
:107DC0004FF08052314BD2F80414C3F82015D2F88A
:107DD0000814C3F82415D2F80C14C3F82815D2F8E7
:107DE0001014C3F82C15D2F81414C3F83015D2F8B7
:107DF0001814C3F83415D2F81C14C3F84015D2F87F
:107E00002014C3F84415D2F82414C3F84815D2F846
:107E10002814C3F84C15D2F82C14C3F85015D2F816
:107E20003014C3F85415D2F83414C3F86015D2F8DE
:107E30003814C3F86415D2F83C14C3F86815D2F8A6
:107E40004014C3F86C15D2F84424C3F870250E4BC7
:107E50001B680D2B09D14FF08043D3F80024D207C3
:107E600044BF6FF00102C3F80024094AD2F88830F9
:107E700043F47003C2F88830BFF34F8FBFF36F8FA6
:107E8000044B054A1A6070473001001000C00040E2
:107E900000ED00E03C0000200090D003012070477E
:107EA00003681322DB69184770470369C3F81C1580
:107EB0000369D3F81C21002AFBD00022C3F81C213F
:107EC0000120704710B490F95C30144C590901221C
:107ED000203103F01F0302FA03F344F82130036951
:107EE0005DF8044B0421C3F8081303695A60036961
:107EF000DA6003690022C3F8002502694FF0FF33FE
:107F0000C2F80C350269C2F814350269C2F80835A6
:107F100002691430C2F81035FFF7FABE00E100E044
:107F20001430FFF707BF1430FFF70ABF1430FFF714
:107F3000F3BE0000036990F85E2010B5C3F80C256D
:107F4000036990F85D20C3F8142590F86120036957
:107F5000012A01BF90F85F40C3F81045036990F80B
:107F6000604006BFC3F8084503690022B1F5966F6B
:107F7000C3F86C2569D9B1F5166F69D9B1F5965F6B
:107F800069D9B1F5165F68D9B1F5615F67D9B1F507
:107F9000964F66D9B1F5E14F65D9B1F5164F64D961
:107FA000B1F5614F64D9B1F5963F64D9B1F5E13FC0
:107FB00063D9B1F5613F63D9364B994263D9B1F5C5
:107FC000E12F63D9B1F5612F94BF4FF070634FF08B
:107FD00080530269C2F8243503690422C3F80025DE
:107FE00001690023C1F808310169C1F81C31016938
:107FF00001230B6001698B600169C1F8042390F9CA
:108000005C20510902F01F0293406031224A42F87D
:10801000213090F95C30002BBDBF03F00F0302F656
:10802000FC32D2189B18B5BF60236022137683F808
:10803000002390F95C300122590903F01F0302FA72
:1080400003F3154A42F8213010BD4FF49E23C0E7D8
:108050004FF41D23BDE7114BBBE7114BB9E7114BA3
:10806000B7E7114BB5E7114BB3E74FF41D03B0E78A
:108070004FF46B03ADE70E4BABE74FF0EB73A8E7A4
:108080004FF06C73A5E74FF08063A2E74FF0E86311
:108090009FE700BF90D0030000E100E000B01300B4
:1080A0000050270000F03A0000A04E0000C075000C
:1080B00000903A012DE9F0411E4600254FF47A73F5
:1080C000C0E901530D4B044640F8143B174688465F
:1080D000FFF70AFE0A4AC4F8108084F85C7052F870
:1080E000263084F85D309DF8183052F8233084F83B
:1080F0005E3084F861502046BDE8F0819CD20000DB
:1081000008D2000010B50369D3F8082104464AB12B
:10811000D3F818151430C9B2FFF7EFFD2369002218
:10812000C3F8082110BD00000148FFF7EBBF00BFF6
:10813000807C012007B522230093022221230349DA
:108140000348FFF7B7FF03B05DF804FB00200040D1
:10815000807C012008B102F079BD70470A4B196894
:108160000A4B30B5D3F804050C060D0A44EA0002A8
:108170004FF47A712B46A2FB014501FB0355E00B3E
:1081800040EA454030BD00BFE47C012000100140C2
:1081900038B5044648B1FFF7E1FF054600F01AF88C
:1081A000FFF7DCFF401BA042F8D338BD074B00228D
:1081B000C3F8042182B0D3F80431054A0193019B2E
:1081C00013680133DBB2136002B070470010014046
:1081D000E47C01207047704708B500F067F8FFF7AE
:1081E000FAFF0120FFF7D4FFFFF79AFA034CFFF7DD
:1081F000A9FA002CFBD0AFF30080F8E700000000E4
:1082000038B5174B174D53F82030174813F0200F8F
:108210004FF0010403F01F0304FA03F408BF4FF00A
:10822000A04000292B681149B3FBF1F300F5A260CF
:1082300002FB03F321464FF00A02B3FBF2F314BF33
:108240002246002200F014F842F2107358434FF413
:108250007A722B68B3FBF2F3B0FBF3F038BD00BFCA
:1082600008D200003C0000200003005040420F00F4
:1082700030B504680C40944206D1013B002BF8D184
:1082800012E0013B002B0FD004680C409442F8D15F
:10829000002405680D40954204D101349C42F8D178
:1082A000002002E0201C00E0181C30BD0D4BE02235
:1082B00083F811234FF40032C3F880211A604FF085
:1082C00080430122C3F818259A6003F58833002102
:1082D000C3F808150221C3F80413C3F844131A6045
:1082E000704700BF00E100E0014B1860704700BF1D
:1082F00058000020222837B50CD84B4B53F82030BB
:10830000052B00F0828007D8032B12D07BD8022BDC
:1083100000F08180002074E01D2B78D003D81C2B46
:10832000F8D1052206E01E2B73D01F2BF2D10822B4
:1083300000E002223D4B196808296EDD0A296FDD35
:108340000D29B5BF0C240E24022303233848C0F89E
:10835000F0350123C0F8003500200546030103F184
:10836000804303F5E04301300828C3F81455C3F8EF
:108370001055F3D12F4B18682F4B1B6800021B03BD
:1083800003F4805300F4E0601843294BC3F8180548
:10839000C3F81425C3F810250DF10602C3F82C26E6
:1083A0000122C3F830261A60D3F80021002AFBD03E
:1083B0000022C3F8002101225A601D4B1A46D3F84F
:1083C00004010028FBD00020C3F8040101209860BC
:1083D000D2F81431002BFBD00023C2F81431BDF9C0
:1083E00006209A42124AB8BFADF80630A142C2F840
:1083F0000035BDF9060004D035BF611A091BC8401D
:10840000884003B030BD032294E7042292E706229D
:1084100090E707228EE701228CE70824002395E7E6
:108420000A24012392E700BF08D200005000002078
:108430000070004054000020F07C0120222830B55C
:108440003CD8224B53F82000214B00221D4653F804
:108450002240B4F1FF3F32D11E4C45F822006FEAB2
:1084600041411D4D1D4B246853F822306FEA5141A4
:1084700025F81210012101FA04F4C3F86005013C4B
:10848000C3F8640505EB4202C3F86805C3F86C0540
:108490000020C3F80015C3F80C05C3F80405C3F8A1
:1084A0000845C3F81405C3F81005C3F82025C3F820
:1084B0002415C3F82815C3F82C05996030BD8442F3
:1084C000CAD00132042AC2D1F8E700BF08D20000A6
:1084D0004000002058000020E87C0120C4D20000A9
:1084E000222815D8114B124A53F8203013F0200FD0
:1084F00008BF4FF0A04203F01F03032908D8DFE8AC
:1085000001F00210080C03F5E073002142F823107B
:10851000704703F5E0730C21F8E703F5E0730421DD
:10852000F4E703F5E0730321F0E700BF08D2000091
:1085300000030050222813D80A4B53F820000A4B9E
:1085400010F0200F4FF0010200F01F0008BF4FF0A5
:10855000A043824011B9C3F80C257047C3F8082521
:10856000704700BF08D2000000030050222810D836
:10857000094B0A4A53F8203013F0200F08BF4FF080
:10858000A04203F01F03D2F81005D84000F001000C
:1085900070470020704700BF08D200000003005061
:1085A0002DE9F04106460D4601EB02080C46444514
:1085B000A4EB050707D0336814F8011B1B6830468D
:1085C00098470028F3D13846BDE8F0812DE9F04105
:1085D000C1F30A57A7F2FF35132D82B002460B46AE
:1085E0000C464FEAD178064633DC002D4EDB3C4981
:1085F000294103EA0100104326D049080B4052EA02
:1086000003060CD04FF48023132D24EA010143FA12
:1086100005F444EA01040CBF4FF00046002631493E
:1086200001EBC8082346D8E90045324620462946D2
:1086300001F01EFBCDE9000122462B46DDE90001D9
:1086400001F014FB02460B461046194602B0BDE885
:10865000F081332D07DDB5F5806FF5D101F008FB12
:1086600002460B46F0E7A7F213474FF0FF31F940FF
:108670000842E9D049080842D1D04FF0804320EAAF
:10868000010143FA07F741EA0706C8E721F0004174
:108690000143D9D0C3F3130101434E420E43114DA0
:1086A0005C0C360B640406F4002305EBC80243EAB5
:1086B0000401D2E900450B4602462946204601F056
:1086C000D7FACDE9000122462B46DDE9000101F091
:1086D000CDFA21F00041024641EAC873B4E700BF79
:1086E000FFFF0F00D8D20000F8B5C1F30A57A7F278
:1086F000FF35132D02460B460C4610DC002D29DBFE
:108700008C461D4929410B422AD04FF400242C41AC
:10871000644424EA0104002621463046F8BD332D86
:1087200005DDB5F5806F1ED010461946F8BDA7F2DD
:1087300013474FF0FF3121FA07F73842F4D00123F5
:10874000C5F1330503FA05F5461928BFE41826EAF2
:108750000706E1E7013501F0004407D00026DBE71A
:108760000028D2D1E0E701F083FAF8BD44F07F544D
:1087700044F440140026CFE7FFFF0F0030B51F4A36
:1087800021F00043934287B01CDD1D4A934205DD72
:1087900002460B4601F06AFA07B030BD02AA00F0AB
:1087A0008FF800F003000128DDE9042312D002282D
:1087B0001CD0A0B1DDE9020100F066FB01F100412F
:1087C00007B030BD002300930022002301F084F89D
:1087D00007B030BDDDE9020100F056FBDCE7012403
:1087E000DDE90201009401F077F8D5E70124DDE925
:1087F0000201009401F070F8E0E700BFFB21E93FBF
:10880000FFFFEF7F2DE9F04F8BB004460D4600F0DF
:1088100079FA294B93F900A0BAF1FF3F06460F46BB
:1088200012D022462B462046294601F071FE83468F
:1088300050B94FF000084FF0000920462946424643
:108840004B4601F03DFE20B9304639460BB0BDE83D
:10885000F08F0122194BCDF820B00092CDE90445EC
:10886000CDE902450193BAF1000F17D042464B46BD
:108870004046494601F0DCFCBAF1020FCDE90601A1
:108880000ED101F0A1FE21230360089B73B9DDE93D
:108890000667304639460BB0BDE8F08FCDE9068952
:1088A000684601F055F90028EFD1EAE701F08CFEA7
:1088B000089B0360EBE700BF5C000020E8D20000EB
:1088C0002DE9F047CA4B21F000479F4290B0804607
:1088D000894640F38F80C74B9F420C46924626DC68
:1088E0000029B9A3D3E9002340F38F8001F0BEF93A
:1088F000C14B9F4204460D4600F04781B4A3D3E923
:10890000002301F0B3F902460B46CAE900232046D2
:10891000294601F0ABF9AEA3D3E9002301F0A6F993
:108920000125CAE90201284610B0BDE8F087B34B23
:108930009F4240F38980B24B9F4200F31C813D155A
:10894000A5F21645A7EB055319461F46064601F04A
:10895000F5FD01F0D9FA8046894642464B4630463D
:108960003946CDE90A8901F081F90022A54B01F0D1
:1089700035FB8946804601F0E1FD01F0C5FA064667
:108980000F4632463B4640464946CDE90C6701F06A
:108990006DF900229B4B01F021FB00220023CDE961
:1089A0000E0101F083FD002800F0608100233046B5
:1089B0003946002201F07AFD002814BF012302236A
:1089C000914A019202212A4600910AA8514600F0DC
:1089D00083FB002C054614DADAF80420DAF80C30B0
:1089E00002F1004203F100434542CAF80420CAF8EC
:1089F0000C3006E000200021C2E90089C2E9020132
:108A00000025284610B0BDE8F08701F031F97A4B17
:108A10009F4204460D4600F00B816DA3D3E900236D
:108A200001F026F902460B46CAE9002329462046F2
:108A300001F01CF966A3D3E9002301F019F94FF006
:108A4000FF35CAE90201DCE700F0FCFF62A3D3E9CD
:108A500000238046894601F0C1FA00226B4B01F0E9
:108A600007F901F06BFD054601F04EFA56A3D3E974
:108A70000023CDE9060101F0B1FA02460B4640465B
:108A8000494601F0F3F852A3D3E900238046894612
:108A9000DDE90601CDE9028901F0A0FA1F2D0246A9
:108AA0000B46CDE9042340F3B380DDE90423DDE97F
:108AB000020101F0DBF8804689463F15C9F30A53ED
:108AC000FB1A102B40F3B18045A3D3E90023DDE965
:108AD000060101F083FA8046894602460B46DDE92D
:108AE000020101F0C3F802460B46DDE90201CDE9BF
:108AF000082301F0BBF842464B4601F0B7F83AA311
:108B0000D3E9002380468946DDE9060101F066FAD3
:108B100042464B4601F0AAF80B46CDE90401024655
:108B2000DDE9080101F0A2F8C1F30A53FF1A312F61
:108B30008046894600F39C809DED087BCAE9008948
:108B40008DED027B42464B46DDE9020101F08EF8D5
:108B5000DDE9042301F08AF8002CCAE90201BFF61E
:108B600050AF09F1004401F100436D42CAE90084AD
:108B7000CAE9020345E702460B4601F077F80025F3
:108B8000CAE90201CAE900013BE715A3D3E90023C2
:108B900001F06CF814A3D3E900230D46044601F05C
:108BA00065F802460B46CAE900232946204601F033
:108BB0005DF80DA3D3E9002301F058F80125CAE9B7
:108BC00002011EE7AFF3008000004054FB21F93F93
:108BD0003163621A61B4D03D83C8C96D305FE43F30
:108BE0000000601A61B4D03D7370032E8A19A33B54
:108BF000FB21E93F7BD90240FB21F93FFB213941B1
:108C0000FFFFEF7F0000704170D300000000E03FE5
:108C10004046494601F02AF8394B6A1E804653F80F
:108C20002230BB4289463FF448AFCAE9008989E750
:108C30002BA3D3E9002301F01BF82BA3D3E90023D6
:108C40000D46044601F014F802460B46CAE900231B
:108C50002946204601F00AF823A3D3E9002301F0B6
:108C600007F84FF0FF35CAE90201CAE60323A7E679
:108C70001FA3D3E90023DDE9060101F0AFF90646A1
:108C80000F4602460B46DDE9080100F0EFFF804683
:108C9000894602460B46DDE90801CDE9028900F06C
:108CA000E5FF32463B4600F0E1FF13A3D3E9002382
:108CB00006460F46DDE9060101F090F932463B46D3
:108CC00000F0D4FF02460B4640464946CDE9042356
:108CD00000F0CCFF80468946A7E700BFAFF30080D5
:108CE0000000601A61B4D03D7370032E8A19A33B53
:108CF0000000002E8A19A33BC14920259A837B39A5
:108D0000F0D200005E4A8A432DE9F04104460D4648
:108D100000F0958000290B460646844656DD0F1567
:108D200000F0A580C3F31303A7F2FF3743F48013C9
:108D30004FEADC72F80702EB43034FEA4C0504D517
:108D4000ED0F05EB43034FEA8C0500267F10B44678
:108D500016224FF400110CEB010098424FEAD57433
:108D60004FEA450503DC1B1A00EB010C0E44013AE7
:108D700004EB43034FEA5101EDD1104696462024FF
:108D80004FF0004209E051D05B00013C03EBD5738A
:108D90004FEA52024FEA450537D0634502EB0E0118
:108DA000F1DD002901EB020E0ADBE046A3EB0C0328
:108DB000A94288BF03F1FF336D1A1044C446E3E7AC
:108DC000BEF1000FF1DB0CF10108EFE721F00042EA
:108DD000024329D0002942D10146CA0A153B490560
:108DE000002AFAD012F4801001D044E0604652000C
:108DF000D40200F1010CF9D5CCF1200401FA0CFCED
:108E0000E1401F1A41EA02038CE72B4321D14408B9
:108E1000731003F17F53F20703F5001348BF44F0CA
:108E2000004403EB07512046BDE8F081A942ABD8CE
:108E3000002901EB020EC3DB98460023BCE7024683
:108E40000B4601F0CBF822462B4600F011FFBDE89F
:108E5000F081411C16BF421C01365408D8E7024677
:108E600000F004FF02460B4601F0E2F9DCE71A4687
:108E700031463B46B6E78C4620244FF0FF30BFE733
:108E80000000F07F000000002DE9F04F21F00048C5
:108E9000B8F1795F85B006460F4692469B466BDA7D
:108EA00001F04CFB002800F0E18032463B463046A2
:108EB000394601F093F874A3D3E9002304460D4624
:108EC00001F08CF872A3D3E9002300F0D1FE224612
:108ED0002B4601F083F870A3D3E9002300F0C6FE0F
:108EE00022462B4601F07AF86DA3D3E9002300F067
:108EF000BFFE22462B4601F071F86BA3D3E9002395
:108F000000F0B4FE22462B4601F068F868A3D3E9CE
:108F1000002300F0ADFE22462B4601F05FF8CDE9BC
:108F200000010022664B2046294601F057F8DDE992
:108F30000023804689462046294601F04FF85246D4
:108F400004460D465B463046394601F047F8024676
:108F50000B462046294600F089FE02460B46404655
:108F6000494600F083FE02460B460020554900F0BA
:108F70007DFE05B0BDE8F08F02460B4601F02EF8ED
:108F800041A3D3E9002304460D4601F027F840A38E
:108F9000D3E9002300F06CFE22462B4601F01EF8B8
:108FA0003DA3D3E9002300F061FE22462B4601F0E9
:108FB00015F83BA3D3E9002300F05AFE22462B46C6
:108FC00001F00CF838A3D3E9002300F04FFE22464D
:108FD0002B4601F003F836A3D3E9002300F048FE46
:108FE0002B46224600F0FAFF374B9845CDE90001A9
:108FF00097DD364B98453EDCA8F500130022002093
:1090000030499046994600F031FECDE90201002238
:109010002B4B2046294600F0E1FF42464B4600F02C
:1090200025FEDDE90023804689462046294600F0DA
:10903000D5FF524604460D465B463046394600F0A1
:10904000CDFF02460B462046294600F00FFE0246A1
:109050000B464046494600F009FE02460B46DDE954
:10906000020100F003FE05B0BDE8F08F15490020B5
:1090700005B0BDE8F08F9FED107B4FF000088DED3F
:10908000027BDFF84C90C2E7D43888BEE9FAA8BD6D
:10909000C4B1B4BD9EEE213EAD529C804F7E923E47
:1090A0009015CB19A001FA3E7751C1166CC1563FFD
:1090B0004C5555555555A53F000000000000E73FB1
:1090C0000000E03F0000F03F3233D33F0000E93FB3
:1090D0000000D23F000000002DE9F04FADF5197DF2
:1090E000BE4CA29EBE4D54F826600793D41E85FB4D
:1090F0000475E417C4EBA50424EAE4741D46631C5C
:10910000A3EB8303013D02EBC3030593731904969C
:109110000994019503900B91A4EB05071AD43B44E5
:10912000002400255E1C0DF18008DDF88C9208E01B
:1091300059F8270000F0E8FE0137B742E8E80201DD
:1091400008D0002FF4DA013720462946B742E8E874
:109150000201F6D1049B002B079B4FEAC303029345
:109160002ADB039A20A902EB030801EB0309049B05
:1091700072AA02EBC30B0DF5E07A019B002B4FF0B6
:1091800000064FF0000711DB039C4D4675E90223F2
:10919000F4E8020100F022FF02460B463046394651
:1091A00000F066FD444506460F46EFD1EAE8026747
:1091B000DA4509F10809E0D1DDE902040499204407
:1091C0008B0082460BA8A3F10802C31808930CABCE
:1091D00013440A938B4698AB03EBCB03BBF1000F10
:1091E00053E9284529DD70AB03EBCB080DF13009BD
:1091F00000227C4B2046294600F0F0FE01F09EF94B
:1092000000F082FE0022784B06460F4600F0E6FE94
:1092100002460B462046294600F028FD01F08EF953
:1092200078E9022349F8040B3946304600F020FD66
:1092300070AB984504460D46DAD1DDF8149020460F
:1092400029464A4600F088FC00224FF07F5304462E
:109250000D4600F0C3FE00F0FBFB0022634B00F064
:10926000BDFE02460B462046294600F0FFFC0D4697
:10927000044601F063F9804600F046FE0B460246C4
:109280002946204600F0F2FC4B46002B06460F46CE
:1092900040F3E1800BF1FF320CA9C9F1180351F83A
:1092A000225045FA03F101FA03F30CA8EB1A40F837
:1092B0002230C9F11705884443FA05F5002D2CDD4D
:1092C000BBF1000F08F1010840F381820C9C002CD7
:1092D00040F0A780BBF1010F0AD00CA9012251F880
:1092E000044F531C002C40F09E809B451A46F6D13B
:1092F000059B002B0EDD012B00F0D980022B09D13C
:109300000BF1FF320CAB0CA953F82230C3F3150359
:1093100041F82230022D00F0AF80002200233046B9
:10932000394601F0C3F8002800F05382049B0BF18A
:10933000FF394B4510DC0BF180430CAA013B089828
:1093400002EB8303002253F80419834242EA01022C
:10935000F9D1002A40F0B680049B0CAA013B52F8D8
:109360002330002B40F0A1800A9A012352F80419FF
:1093700001330029FAD05B440BF1010999450693AA
:109380004CDC099A079909EB020801EB0B0508F17F
:10939000804802EB030BA39B08F1FF3803EB88081E
:1093A00070AB03EBC909A39B20A903EB8B0301EB73
:1093B000C505029358F8040F00F0A6FD0B4601996D
:1093C0000246002905F1080BC5E900234FF000060D
:1093D0004FF000071CDB039C0CE000BFB8D400007A
:1093E000ABAAAA2A0000703E000070410000204095
:1093F00075E90223F4E8020100F0F0FD02460B4695
:109400003046394600F034FC544506460F46EFD14D
:10941000029B9845E9E802675D46CBD1DDF818B0BC
:10942000D9E6012300220CA9C4F180749B4541F8C0
:1094300022400EDD51F8232001EB8B0001EB83036A
:109440006FF07F4100E01A688A1A43F8042B8342C8
:10945000F9D101244CE706D10BF1FF330CAA52F8E5
:109460002350ED152AE700227B4B01F03DF8002840
:1094700040F0A381054650E732463B46002077493D
:1094800000F0F4FB06460F46002C3FF446AF059A69
:109490007249002000F060FB02460B463046394618
:1094A00000F0E4FB06460F4637E7012363E70BF1C4
:1094B000FF320CAB0CA953F82230C3F3160341F86A
:1094C000223027E70CAB059A53F82930183ACDE93A
:1094D000068505926BB909F18043013B0CA901EBAC
:1094E000830353F8041909F1FF39183A0029F8D019
:1094F0000592059A5949002000F02EFBB9F1000FA2
:1095000004460D46C0F2C0814FEAC90370AA02EBBF
:10951000030808930CAB03EB8906DFF844B14FF066
:10952000000A08F10807043656F8040D00F0ECFCB8
:1095300022462B4600F052FD5B4667E90201524687
:109540002046294600F04AFD0CAB9E4204460D46DB
:10955000EAD148AB03930193CDF8149009F10103CC
:10956000DDF810900293C3464FF0000AB9F1000FE6
:10957000C0F22A81DFF8EC805D4635A3D3E90023F1
:1095800000260027002403E0544510DCF8E80223FD
:10959000F5E8020100F022FD02460B46304639464E
:1095A00000F066FB0134A14506460F46ECDA019B4C
:1095B000E3E802670193029B0AF1010A9A45ABF1C5
:1095C000080BD3D1A29BDDF81490032B39D8DFE828
:1095D00013F0D900060006004D0048AB0393B9F123
:1095E000000F4FF000004FF0000109DB039D05EB79
:1095F000C904083474E9022300F03AFBA542F9D10A
:10960000079B002B40F01E810B9BC3E900010B461A
:1096100003990246D1E9000100F028FBB9F1000FDF
:109620000CDD4AAD01240134F5E8022300F020FBF3
:10963000A145F8DA079B002B40F014810B9BC3E98E
:109640000201069B03F007000DF5197DBDE8F08FC0
:1096500000000040FB21F93F0000E03F0000F03F28
:109660000000703E80D4000048AB0393B9F1000FB6
:1096700040F32781039ACDF810904FEAC903019374
:10968000D318D3E900AB09F10053013B02EBC90841
:109690000293914678E9026752465B463046394666
:1096A00000F0E6FA04460D4602460B4630463946BF
:1096B00000F0DCFA52465B4600F0DAFAC145A246F9
:1096C000AB46C8E90201C8E90045E3D1DDF81090D6
:1096D000B9F1010F40F3F580019B039A02991344FD
:1096E000C900D3E9006701F1080A019192440DF520
:1096F000947B7AE9028932463B464046494600F06F
:10970000B7FA04460D4602460B464046494600F06D
:10971000ADFA32463B4600F0ABFAD34526462F461B
:10972000CAE90201CAE90045E3D1019C039B103458
:10973000002000211C4403F1100574E9022300F00D
:1097400097FAA542F9D1039C079ED4E90023D4E9F6
:109750000245002E00F08A8003F1004701F100432A
:109760000B99C1E90403069B2646944605F1004483
:1097700003F00700C1E900C7C1E902640DF5197DD6
:10978000BDE8F08F089C039D0834002000212C4484
:1097900074E9022300F06CFAA542F9D1079B13B1DA
:1097A00001F1004319460B9BC3E90001069B03F03E
:1097B00007000DF5197DBDE8F08FBBF1000F08F132
:1097C000010874DD022581E500260027EFE600246C
:1097D0008EE5CDE90685059D304639466A4200F0A2
:1097E000BBF90022384B06460F4600F07DFE00B361
:1097F0000022364B3046394600F0F0FB00F09EFE6A
:10980000044600F081FB00222F4B00F0E7FB0B46E3
:1098100002463946304600F029FA00F08FFE0BF17F
:1098200001090CAB183543F82B00059543F8294086
:109830005FE63046394600F081FE0CABD94643F86E
:109840002B0056E60B9C01F10043C4E900030B46D4
:1098500003990246D1E9000100F008FAB9F1000FBE
:109860003FF7DFAE01F100431946E7E60B9EC6E97C
:109870000023069BC6E9040103F00700C6E9024580
:109880000DF5197DBDE8F08FA29B032B3FF6D9AEF5
:1098900001A252F823F000BFA9980000DB95000058
:1098A000DB950000699600000020002176E7324633
:1098B0003B460020064900F0D9F9022506460F462E
:1098C0002BE5002000213EE7000070410000703EC3
:1098D0000000F03F000000002DE9F04F21F00046AD
:1098E000B6F1795F85B004460D469046994604DA94
:1098F00000F024FE002800F0858022462B462046FA
:10990000294600F06BFB06460F4602460B462046F2
:10991000294600F063FB41A3D3E9002382468B462E
:109920003046394600F05AFB3EA3D3E9002300F04D
:109930009DF932463B4600F051FB3CA3D3E900239E
:1099400000F096F932463B4600F048FB39A3D3E9D4
:10995000002300F08BF932463B4600F03FFB37A373
:10996000D3E9002300F084F90E9BCDE900019BB3FD
:109970000022294B4046494600F030FBDDE9002338
:10998000CDE902015046594600F028FB02460B463D
:10999000DDE9020100F06AF932463B4600F01EFBA9
:1099A00042464B4600F062F919A3D3E9002306466C
:1099B0000F465046594600F011FB02460B46304612
:1099C000394600F055F902460B462046294600F07C
:1099D0004DF905B0BDE8F08F02460B4630463946DA
:1099E00000F0FCFA0AA3D3E9002300F03FF9524645
:1099F0005B4600F0F3FA22462B4600F039F905B039
:109A0000BDE8F08F2046294605B0BDE8F08F00BFC5
:109A1000495555555555C53F0000E03F7CD5CF5AB7
:109A20003AD9E53DEB9C2B8AE6E55A3E7DFEB157DF
:109A3000E31DC73ED561C119A0012A3FA6F8101148
:109A40001111813F21F000431946704700000000CA
:109A50002DE9F041C1F30A57A7F2FF35132D024655
:109A60000B460C46884606461DDC002D3CDB364F77
:109A70002F4101EA070C5CEA000C19D030A3D3E9AE
:109A8000002300F0F5F80022002300F037FDC8B3F2
:109A9000002C04DA4FF4801343FA05F5A84428EAB1
:109AA000070400262EE0332D06DDB5F5806F2DD09E
:109AB00010461946BDE8F081A7F213474FF0FF3C6E
:109AC0002CFA07F70742F3D01DA3D3E9002300F0D7
:109AD000CFF80022002300F011FD98B1002C21DB0B
:109AE00026EA070644460DE015A3D3E9002300F05B
:109AF000BFF80022002300F001FD18B1002C08DBA4
:109B00000026344621463046BDE8F08100F0B0F82A
:109B1000D0E724F000430D4A1E43002E18BF144620
:109B20000026EFE7142D08D00123C5F1340503FA10
:109B300005F5AE1928BF9844D2E704F10108CFE734
:109B40009C7500883CE4377EFFFF0F000000F0BFEB
:109B50000020704700000000F8B5C1F30A53044626
:109B60000D460E4617460BBB21F000460346334315
:109B70001BD0354B002200F031FA344B9F42044693
:109B80000D4635DBC1F30A530E46363B3B4440F2EB
:109B9000FE72934232DC002B11DD26F0FF4626F4E4
:109BA000E00646EA035520462946F8BD40F2FF721A
:109BB0009342EBD102460B4600F05AF8F8BD13F180
:109BC000350F28DA4CF250339F4222462B460ADDED
:109BD00019A1D1E9000100F03DF817A3D3E9002352
:109BE00000F0FCF9F8BD16A1D1E9000100F032F84F
:109BF00013A3D3E9002300F0F1F9F8BD22462B4668
:109C00000DA1D1E9000100F025F80BA3D3E9002351
:109C100000F0E4F9F8BD26F0FF4626F4E0063633FE
:109C200046EA0355204629460022094B00F0D6F9A2
:109C3000F8BD00BFAFF300809C7500883CE4377E20
:109C400059F3F8C21F6EA50100005043B03CFFFF5E
:109C50000000903C03F0004321F0004242EA03017F
:109C6000704700BF81F0004102E000BF83F0004375
:109C700030B54FEA41044FEA430594EA050F08BFA7
:109C800090EA020F1FBF54EA000C55EA020C7FEA6B
:109C9000645C7FEA655C00F0E2804FEA5454D4EBE8
:109CA0005555B8BF6D420CDD2C4480EA020281EAB2
:109CB000030382EA000083EA010180EA020281EAEA
:109CC0000303362D88BF30BD11F0004F4FEA01313C
:109CD0004FF4801C4CEA113102D0404261EB41014B
:109CE00013F0004F4FEA03334CEA133302D05242D1
:109CF00063EB430394EA050F00F0A780A4F101048D
:109D0000D5F1200E0DDB02FA0EFC22FA05F28018C6
:109D100041F1000103FA0EF2801843FA05F35941AC
:109D20000EE0A5F120050EF1200E012A03FA0EFC2B
:109D300028BF4CF0020C43FA05F3C01851EBE37155
:109D400001F0004507D54FF0000EDCF1000C7EEB72
:109D500000006EEB0101B1F5801F1BD3B1F5001FB0
:109D60000CD349085FEA30004FEA3C0C04F10104CF
:109D70004FEA445212F5800F80F09A80BCF1004FF8
:109D800008BF5FEA500C50F1000041EB045141EA7A
:109D9000050130BD5FEA4C0C404141EB010111F47B
:109DA000801FA4F10104E9D191F0000F04BF014626
:109DB0000020B1FA81F308BF2033A3F10B03B3F104
:109DC00020020CDA0C3208DD02F1140CC2F10C0294
:109DD00001FA0CF021FA02F10CE002F11402D8BFF2
:109DE000C2F1200C01FA02F120FA0CFCDCBF41EABE
:109DF0000C019040E41AA2BF01EB0451294330BD8D
:109E00006FEA04041F3C1CDA0C340EDC04F1140469
:109E1000C4F1200220FA04F001FA02F340EA030040
:109E200021FA04F345EA030130BDC4F10C04C4F186
:109E3000200220FA02F001FA04F340EA0300294666
:109E400030BD21FA04F0294630BD94F0000F83F4B0
:109E5000801306BF81F480110134013D4EE77FEA93
:109E6000645C18BF7FEA655C29D094EA050F08BFDF
:109E700090EA020F05D054EA000C04BF19461046C0
:109E800030BD91EA030F1EBF0021002030BD5FEA04
:109E9000545C05D14000494128BF41F0004130BD2C
:109EA00014F580043CBF01F5801130BD01F0004580
:109EB00045F0FE4141F470014FF0000030BD7FEAF3
:109EC000645C1ABF194610467FEA655C1CBF0B46EE
:109ED000024650EA013406BF52EA033591EA030F05
:109EE00041F4002130BD00BF90F0000F04BF0021FD
:109EF000704730B54FF4806404F132044FF0000530
:109F00004FF0000150E700BF90F0000F04BF0021A8
:109F1000704730B54FF4806404F1320410F000450E
:109F200048BF40424FF000013EE700BF42004FEA09
:109F3000E2014FEA31014FEA02701FBF12F07F4386
:109F400093F07F4F81F06051704732F07F4208BF3D
:109F5000704793F07F4F04BF41F40021704730B544
:109F60004FF4607401F0004521F000411CE700BF90
:109F700050EA010208BF704730B54FF000050AE013
:109F800050EA010208BF704730B511F0004502D514
:109F9000404261EB41014FF4806404F132045FEA16
:109FA000915C3FF4D8AE4FF003025FEADC0C18BFBF
:109FB00003325FEADC0C18BF033202EBDC02C2F1B1
:109FC000200300FA03FC20FA02F001FA03FE40EA43
:109FD0000E0021FA02F11444BDE600BF70B54FF047
:109FE000FF0C4CF4E06C1CEA11541DBF1CEA135525
:109FF00094EA0C0F95EA0C0F00F0DEF82C4481EA8D
:10A00000030621EA4C5123EA4C5350EA013518BFAC
:10A0100052EA033541F4801143F4801338D0A0FB99
:10A0200002CE4FF00005E1FB02E506F00042E0FB46
:10A0300003E54FF00006E1FB03569CF0000F18BF4C
:10A040004EF0010EA4F1FF04B6F5007F64F54074F4
:10A0500004D25FEA4E0E6D4146EB060642EAC62187
:10A0600041EA55514FEAC52040EA5E504FEACE2EF4
:10A07000B4F1FD0C88BFBCF5E06F1ED8BEF1004FF7
:10A0800008BF5FEA500E50F1000041EB045170BD73
:10A0900006F0004646EA010140EA020081EA0301B7
:10A0A000B4EB5C04C2BFD4EB0C0541EA045170BDB3
:10A0B00041F480114FF0000E013C00F3AB8014F12D
:10A0C000360FDEBF002001F0004170BDC4F1000476
:10A0D000203C35DA0C341BDC04F11404C4F12005F7
:10A0E00000FA05F320FA04F001FA05F240EA020052
:10A0F00001F0004221F0004110EBD37021FA04F688
:10A1000042EB06015EEA430E08BF20EAD37070BD41
:10A11000C4F10C04C4F1200500FA04F320FA05F0A0
:10A1200001FA04F240EA020001F0004110EBD370A2
:10A1300041F100015EEA430E08BF20EAD37070BD12
:10A14000C4F1200500FA05F24EEA020E20FA04F3EB
:10A1500001FA05F243EA020321FA04F001F000419A
:10A1600021FA04F220EA020000EBD3705EEA430E0B
:10A1700008BF20EAD37070BD94F0000F0FD101F03A
:10A180000046400041EB010111F4801F08BF013C73
:10A19000F7D041EA060195F0000F18BF704703F0B1
:10A1A0000046520043EB030313F4801F08BF013D38
:10A1B000F7D043EA0603704794EA0C0F0CEA1355F4
:10A1C00018BF95EA0C0F0CD050EA410618BF52EAAE
:10A1D0004306D1D181EA030101F000414FF00000B4
:10A1E00070BD50EA410606BF1046194652EA4306C2
:10A1F00019D094EA0C0F02D150EA013613D195EA36
:10A200000C0F05D152EA03361CBF104619460AD17D
:10A2100081EA030101F0004141F0FE4141F4700187
:10A220004FF0000070BD41F0FE4141F4780170BD77
:10A2300070B54FF0FF0C4CF4E06C1CEA11541DBFDC
:10A240001CEA135594EA0C0F95EA0C0F00F0A7F8DE
:10A25000A4EB050481EA030E52EA03354FEA01310B
:10A2600000F088804FEA03334FF0805545EA13131E
:10A2700043EA12634FEA022245EA111545EA1065E6
:10A280004FEA00260EF000419D4208BF964244F17D
:10A29000FD0404F5407402D25B084FEA3202B61A9C
:10A2A00065EB03055B084FEA32024FF480104FF470
:10A2B000002CB6EB020E75EB030E22BFB61A7546E4
:10A2C00040EA0C005B084FEA3202B6EB020E75EB77
:10A2D000030E22BFB61A754640EA5C005B084FEADF
:10A2E0003202B6EB020E75EB030E22BFB61A7546AC
:10A2F00040EA9C005B084FEA3202B6EB020E75EBB7
:10A30000030E22BFB61A754640EADC0055EA060E77
:10A3100018D04FEA051545EA16754FEA06164FEABA
:10A32000C30343EA52734FEAC2025FEA1C1CC0D166
:10A3300011F4801F0BD141EA00014FF000004FF0F3
:10A34000004CB6E711F4801F04BF01430020B4F1B4
:10A35000FD0C88BFBCF5E06F3FF6AFAEB5EB030C6C
:10A3600004BFB6EB020C5FEA500C50F1000041EB69
:10A37000045170BD0EF0004E4EEA113114EB5C0436
:10A38000C2BFD4EB0C0541EA045170BD41F4801109
:10A390004FF0000E013C90E645EA060E8DE60CEA11
:10A3A000135594EA0C0F08BF95EA0C0F3FF43BAF2E
:10A3B00094EA0C0F0AD150EA01347FF434AF95EAE5
:10A3C0000C0F7FF425AF104619462CE795EA0C0FC9
:10A3D00006D152EA03353FF4FDAE1046194622E796
:10A3E00050EA410618BF52EA43067FF4C5AE50EA70
:10A3F00041047FF40DAF52EA43057FF4EBAE12E760
:10A400004FF0FF3C06E000BF4FF0010C02E000BF40
:10A410004FF0010C4DF804CD4FEA410C7FEA6C5C23
:10A420004FEA430C18BF7FEA6C5C1BD001B050EAC6
:10A43000410C0CBF52EA430C91EA030F02BF90EAB1
:10A44000020F0020704710F1000F91EA030F58BF70
:10A45000994208BF90422CBFD8176FEAE37040F0D2
:10A46000010070474FEA410C7FEA6C5C02D150EA70
:10A47000013C07D14FEA430C7FEA6C5CD6D152EA2B
:10A48000033CD3D05DF8040B704700BF84461046F0
:10A4900062468C461946634600E000BF01B5FFF7EF
:10A4A000B7FF002848BF10F1000F01BD4DF808EDBF
:10A4B000FFF7F4FF0CBF012000205DF808FB00BF90
:10A4C0004DF808EDFFF7EAFF34BF012000205DF8EA
:10A4D00008FB00BF4DF808EDFFF7E0FF94BF012037
:10A4E00000205DF808FB00BF4DF808EDFFF7CEFF38
:10A4F00094BF012000205DF808FB00BF4DF808ED77
:10A50000FFF7C4FF34BF012000205DF808FB00BF47
:10A510004FEA410C7FEA6C5C02D150EA013C0AD15F
:10A520004FEA430C7FEA6C5C02D152EA033C02D151
:10A530004FF0000070474FF0010070474FEA4102B2
:10A5400012F5001215D211D56FF47873B3EB625285
:10A5500012D94FEAC12343F0004343EA505311F0AC
:10A56000004F23FA02F018BF404270474FF000003E
:10A57000704750EA013005D111F0004008BF6FF07C
:10A58000004070474FF00000704700BF1FB51C46E9
:10A59000094B1B680546D86852B1084B0091CDE9BC
:10A5A000013207492B46224600F028F800F0BAFD98
:10A5B000044B1A46F2E700BF60000020C8D4000038
:10A5C000D5D4000032C20000014B1868704700BFAC
:10A5D0006000002008B5074B044613B10021AFF31B
:10A5E0000080054B1868836A03B19847204601F044
:10A5F00071FB00BF0000000004D500000EB403B5DD
:10A60000014603AB054853F8042B0068019300F0A2
:10A6100081F802B05DF804EB03B0704760000020E1
:10A6200070B50D4E0D4CA41BA4100025A54209D1F8
:10A630000B4E0C4C01F050FBA41BA4100025A542AE
:10A6400005D170BD56F8253098470135EEE756F82C
:10A65000253098470135F2E7300200203002002013
:10A66000300200204002002010B5431E0A449142EF
:10A6700000D110BD11F8014B03F8014FF7E78842F4
:10A6800010B501EB020307D8421E99420AD011F817
:10A69000014B02F8014FF8E78342F5D98118D21A2D
:10A6A000D34200D110BD13F8014D01F8014DF7E779
:10A6B00002440346934200D1704703F8011BF9E7B7
:10A6C0009368013B002B10B4936008DA9469A342AD
:10A6D00001DB0A2903D15DF8044B00F063BC136869
:10A6E000581C1060197008465DF8044B7047F8B5A7
:10A6F00006460F461446D518AC4201D1002007E0AB
:10A700003A4614F8011B3046FFF7DAFF431CF3D139
:10A71000F8BD00002DE9F04F9DB00C46174603939D
:10A72000064618B183690BB900F0F4FD7B4B9C42DF
:10A7300057D17468A38918075DD52369002B5AD0B7
:10A740000023099320238DF8293030238DF82A30F7
:10A750004FF0010BB846454615F8013B0BB1252BD0
:10A7600054D1B8EB070A0BD053463A46214630463F
:10A77000FFF7BDFF013000F0C280099B53440993ED
:10A7800098F80030002B00F0BA8000234FF0FF3221
:10A79000CDE90523049307938DF853301A93A84607
:10A7A000052218F8011B5E4800F0C2FE049B78BB2E
:10A7B000D90644BF20228DF853201A0744BF2B220C
:10A7C0008DF853202A782A2A2AD0079AA8460020F2
:10A7D0000A25414611F8013B303B092B69D960B38A
:10A7E00024E0504B9C4201D1B468A3E74E4B9C42FD
:10A7F00008BFF4689EE72146304600F025FC00289B
:10A800009ED04FF0FF301DB0BDE8F08FA846A2E704
:10A81000434A801A0BFA00F0184304904546BEE7FD
:10A82000039A111D12680391002A01DB079204E0CC
:10A83000524243F002030792049398F800302E2B03
:10A840000ED198F801302A2B38D1039B1A1D1B68B2
:10A850000392002BB8BF4FF0FF3308F102080593B5
:10A86000324D98F800100322284600F061FE40B1F6
:10A870004023401B03FA00F0049B034308F1010846
:10A88000049398F800102A488DF82810062208F141
:10A89000010700F04DFE002837D0264B1BBB039B61
:10A8A000073323F0070308330393099B4B440993B1
:10A8B00050E705FB0232012088468AE7002308F1B1
:10A8C0000108059319460A25404610F8012B303A35
:10A8D000092A03D9002BC3D00591C1E705FB01214B
:10A8E00001238046F0E703AB00932246124B04A9F4
:10A8F0003046AFF30080B0F1FF3F8146D5D1A38948
:10A900005B063FF57EAF09987DE703AB00932246D7
:10A91000094B04A9304600F087F8ECE75CD500004D
:10A9200008D500007CD500003CD500000ED5000005
:10A9300012D5000000000000EFA600002DE9F0474E
:10A9400091461F468A680B69DDF820809342B8BFA4
:10A950001346C9F8003091F8432006460C4612B160
:10A960000133C9F800302368990642BFD9F8003096
:10A970000233C9F80030256815F0060507D104F147
:10A98000190AE368D9F800209B1AAB4228DC94F836
:10A9900043302268003318BF012392062DD404F1FE
:10A9A000430239463046C047013020D02368E5686D
:10A9B000D9F8002003F00603042B08BFAD1AA368E2
:10A9C00022690CBF25EAE57500259342C4BF9B1A96
:10A9D000ED184FF000091A344D451AD1002008E057
:10A9E0000123524639463046C047013003D14FF06B
:10A9F000FF30BDE8F0870135C3E7E1185A1C30206D
:10AA000081F84300224494F8451082F84310023341
:10AA1000C5E70123224639463046C0470130E6D01B
:10AA200009F10109D8E700002DE9F04301F1430CD9
:10AA30000C46097E85B06E291746064698460C9A44
:10AA400000F0B38022D8632936D00AD8002900F05C
:10AA5000B980582900F0838004F1420584F842103F
:10AA600032E0642901D06929F6D12068136805060F
:10AA700003F104012AD51B681160002B03DA2D2293
:10AA80005B4284F843206F480A2239E0732900F0C2
:10AA90009D8008D86F2920D07029DDD1236843F02C
:10AAA0002003236003E0752917D07829D4D17823B7
:10AAB00084F84530644855E01368191D1B6811601F
:10AAC00004F1420584F8423001238CE01B681160D8
:10AAD00010F0400F18BF1BB2CFE713682568181D90
:10AAE0001060280601D51B6802E06806FBD51B88AC
:10AAF00054486F2914BF0A220822002184F8431009
:10AB00006568A560002DC0F29580216821F00401E0
:10AB10002160002B3DD1002D40F08E806546082A33
:10AB20000BD12368DB0708D5236962689A42DEBF30
:10AB3000302305F8013C05F1FF35ACEB050323613B
:10AB4000CDF800803B4603AA21463046FFF7F6FECB
:10AB500001304DD14FF0FF3005B0BDE8F0833948EA
:10AB600084F84510136821681D1D1B6815600A06CE
:10AB70000BD5CA0744BF41F0200121601BB92268F0
:10AB800022F0200222601022B7E74D0648BF9BB298
:10AB9000EFE76546B3FBF2F102FB1133C35C05F846
:10ABA000013D0B460029F5D1B9E7136825686169B5
:10ABB000181D106028061B6801D5196002E06A069E
:10ABC000FBD51980002323616546B9E71368191D79
:10ABD00011601D6862680021284600F0A9FC08B1D8
:10ABE000401B606063682361002384F84330A7E75B
:10ABF00023692A4639463046C0470130AAD0236827
:10AC00009B0713D4E068039B9842B8BF1846A3E79C
:10AC100001234A4639463046C04701309AD00135B3
:10AC2000E368039A9B1AAB42F2DCEBE7002504F1E0
:10AC30001909F5E7002BACD1037884F8423004F110
:10AC400042056CE719D500002AD5000038B50D4B38
:10AC50001C68A36B05467BB9182000F04DFC0A4A1E
:10AC60000A4BA063C0E90023094B83600B23838157
:10AC700001220023C0E90423A36B00221D615A6155
:10AC800038BD00BF600000200E33CDAB34126DE63E
:10AC9000ECDE050038B5134B1C68A36B7BB918209C
:10ACA00000F02AFC104A114BA063C0E90023104BAE
:10ACB00083600B23838101220023C0E90423A16B5D
:10ACC0000C480A694B690C4C504304FB0300A2FB7F
:10ACD00004230344541C43F10005C1E9044525F055
:10ACE000004038BD600000200E33CDAB34126DE65D
:10ACF000ECDE05002DF451582D7F954C0CB430B589
:10AD0000174B0C1E9DB01D6808DA8B232B604FF08B
:10AD1000FF301DB0BDE8304002B070474FF4027301
:10AD2000ADF8143014BF04F1FF33234604930793A6
:10AD30004FF6FF7302900690ADF81630209A21ABC3
:10AD400002A92846019300F06BFD431CBCBF8B2376
:10AD50002B60002CDDD0029B00221A70D9E700BFC7
:10AD6000600000200EB400B59CB01DAB02900690B0
:10AD70006FF00041094807910491094953F8042BE9
:10AD800005910068019302A900F04AFD029B002290
:10AD90001A701CB05DF804EB03B07047600000202F
:10ADA0000802FFFF10B503461A785C1C3AB9013B54
:10ADB00011F8012B03F8012F002AF9D110BD234609
:10ADC000F2E7C9B2034610F8012B1AB18A42F9D151
:10ADD00018467047002918BF0023F9E710F8012B27
:10ADE00011F8013B012A28BF9A42F7D0D01A7047C8
:10ADF000034613F8012B002AFBD1181A01387047BB
:10AE000010B56AB10139841810F8013B11F8012F0F
:10AE1000934203D1A04201D0002BF5D1981A10BD66
:10AE20001046FCE770B50139044602B970BD2346EF
:10AE300011F8015F03F8015B561E2DB91444A342BB
:10AE4000F4D003F8015BFAE71C463246EDE7F0B5B3
:10AE500003787BB1044623782046661C7BB14A1EEA
:10AE6000631E12F8015F4DB113F8017FAF42344603
:10AE7000F7D0F0E70B78002B18BF0020F0BD184684
:10AE8000FCE72DE9F0478046894692461E460F466C
:10AE90003D46089815F8014B00F0C6FA2044437867
:10AEA00013F0080332D12D2C32D17C78BD1C012245
:10AEB000002E5DD0102E09D1302C07D12B7803F055
:10AEC000DF03582B4FD16C7810260235002A14BFAF
:10AED0004FF000416FF000410027B1FBF6FC38460F
:10AEE00006FB1C1EA4F13003092B17D81C46A642F2
:10AEF00023DD7B1C07D084451CD301D1A64519DB7B
:10AF000000FB0640012715F8014BEBE72F46BFE792
:10AF10002B2C04BFBD1C7C781A46C9E7A4F1410361
:10AF2000192B01D8373CE2E7A4F16103192B04D8AF
:10AF3000573CDCE74FF0FF37E5E77B1C08D12223C5
:10AF4000C8F800300846BAF1000F07D1BDE8F08715
:10AF500002B14042BAF1000FF8D00FB105F1FF394C
:10AF6000CAF80090F2E73024002EAFD10826ADE7F2
:10AF7000302CA3D00A26A9E7084B37B51C68084D2A
:10AF8000236A002B08BF2B46009313460A4601464E
:10AF90002046FFF776FF03B030BD00BF6000002001
:10AFA000C4000020F8B50E461446054618B1836962
:10AFB0000BB900F0AFF9214B9C422AD16C68A36910
:10AFC000A360A3891A072ED5236963B32369206878
:10AFD000C01A6369F6B28342374604DC214628462C
:10AFE00000F02EF928BBA368013BA36023685A1C1C
:10AFF00022601E7063690130834204D0A389DB079D
:10B0000019D50A2E17D12146284600F019F990B11A
:10B010000FE00B4B9C4201D1AC68D0E7094B9C423E
:10B0200008BFEC68CBE72146284600F00DF8002861
:10B03000CCD04FF0FF373846F8BD00BF5CD50000DC
:10B040007CD500003CD50000324B70B51D6806462B
:10B050000C4625B1AB6913B9284600F05BF92E4BBD
:10B060009C420FD16C68B4F90C309AB215072CD4FD
:10B07000D00611D40922326043F04003A3814FF07F
:10B08000FF303EE0254B9C4201D1AC68EBE7244BFE
:10B090009C4208BFEC68E6E7510712D5616B41B1ED
:10B0A00004F14403994202D0304600F091FA0023A3
:10B0B0006363A38923F02403A381002363602369CE
:10B0C0002360A38943F00803A38123694BB9A389B3
:10B0D00003F42073B3F5007F03D02146304600F01F
:10B0E000CBF9A28912F001030CD00023A36063699D
:10B0F0005B42A361236953B9B4F90C3013F08000AB
:10B10000BAD170BD920758BF6369A360F2E700200F
:10B11000F7E700BF600000205CD500007CD5000090
:10B120003CD5000008B5062000F0A8FC012000F086
:10B13000D1FD00008A892DE9F041054610070C4633
:10B1400058D44B68002B05DC0B6C002B02DC002074
:10B15000BDE8F081E66A002EF9D0002312F4805297
:10B160002F68216A2B6032D0606DA3895A0705D5FC
:10B170006368C01A636B0BB1236CC01A00230246CC
:10B18000E66A216A2846B047431CA38906D129688C
:10B190001D2948D8294ACA40D60744D500226260F2
:10B1A000D9042269226004D5421C01D12B6803B95D
:10B1B0006065616B2F600029C9D004F14403994296
:10B1C00002D0284600F004FA00206063C0E70123A3
:10B1D0002846B047411CC8D12B68002BC5D01D2B79
:10B1E00001D0162B01D12F60B1E7A38943F04003B2
:10B1F000A381ADE70F69002FA9D093070E6808BFA0
:10B200004B690F6018BF0023A6EB07088B60B8F1ED
:10B21000000F9CDD43463A46216AA66A2846B0479D
:10B22000002806DCA38943F04003A3814FF0FF30E0
:10B230008EE70744A8EB0008E9E700BF01004020C3
:10B2400038B50B6905460C46DBB118B183690BB9FB
:10B2500000F060F80C4B9C4209D16C68B4F90C30DA
:10B260007BB121462846BDE83840FFF763BF074B56
:10B270009C4201D1AC68F1E7054B9C4208BFEC68E9
:10B28000ECE7002038BD00BF5CD500007CD5000095
:10B290003CD50000002310B50446C0E900338360AC
:10B2A00081814366C281C0E9043383611946082263
:10B2B0005C30FFF7FDF9054B6362054BA362054B5C
:10B2C000E362054B2462236310BD00BFB5BA0000E2
:10B2D000D7BA00000FBB000033BB0000014900F0EB
:10B2E00085B800BF41B2000070B54A1E68255543BD
:10B2F0000E4605F1740100F0B9F9044640B1002191
:10B30000C0E900160C30A06005F16802FFF7D0F923
:10B31000204670BD836910B5044633BBC0E91233C3
:10B320000365124B124A1B688262984204BF0123D4
:10B33000836100F01FF86060204600F01BF8A060F9
:10B34000204600F017F80022E06004216068FFF753
:10B35000A1FF01220921A068FFF79CFF0222122110
:10B36000E068FFF797FF0123A36110BD04D500003B
:10B37000DDB20000F8B51B4B1E68B369074613B970
:10B380003046FFF7C7FF4836D6E90134013B03D505
:10B39000336833B13668F7E7B4F90C506DB16834EF
:10B3A000F4E704213846FFF79FFF30600028F1D111
:10B3B0000C233B6004462046F8BD0B4B6566C4E990
:10B3C0000055A560C4E90335C4E90555082229469E
:10B3D00004F15C00FFF76CF9C4E90D55C4E912559E
:10B3E000E9E700BF04D500000100FFFF2DE9F843A5
:10B3F0008046894600F14804002614B93046BDE86D
:10B40000F883D4E90175013F01D52468F5E7AB89DC
:10B41000012B07D9B5F90E30013303D02946404638
:10B42000C84706436835EEE7D0F8EC00704770B5C2
:10B430000E46B1F90E10002996B014461D4607DAE3
:10B4400000232B60B3891A0610D44FF480630EE0FA
:10B450006A4600F0A1FB0028F2DB019A02F4704278
:10B46000A2F500535A425A412A60EEE740230020D9
:10B47000236016B070BD00008B8973B59D0706462A
:10B480000C4607D504F14703236023610123636160
:10B4900002B070BD01AB6A46FFF7C9FF00990546CF
:10B4A000304600F0E3F848B9B4F90C309A05EFD40F
:10B4B00023F0030343F00203A381E3E70D4BB362E0
:10B4C000A389206043F08003A381009B6361019BFB
:10B4D00020615BB1B4F90E10304600F06FFB28B16B
:10B4E000A38923F0030343F00103A381A3891D4330
:10B4F000A581CDE7DDB20000024B0146186800F0DF
:10B50000B5B800BF6000002082B001B901A942B106
:10B510004BB113780B601278101C18BF012002B0D9
:10B5200070471046FBE76FF00100F8E700000000ED
:10B5300001F0FF01102A2BDB10F0070F08D010F8E4
:10B54000013B013A8B422DD010F0070F42B3F6D1E8
:10B55000F0B441EA012141EA014122F007047FF001
:10B5600000070023F0E80256083C85EA010586EA58
:10B57000010685FA47F5A3FA87F586FA47F6A5FA94
:10B5800087F68EB9EED1F0BC01F0FF0102F00702A0
:10B5900032B110F8013B013A83EA010313B1F8D14B
:10B5A0000020704701387047002D06BF354603382C
:10B5B000073815F0010F07D1013015F4807F02BF65
:10B5C000013015F4C03F0130F0BC0138704700BFB6
:10B5D00038B50546002945D051F8043C0C1F002B16
:10B5E000B8BFE41800F00CFB1F4A1368104633B9CB
:10B5F000636014602846BDE8384000F002BBA342F7
:10B600000CD921686218934204BF1A685B686360B2
:10B6100004BF521822600460ECE713465A680AB16E
:10B62000A242FAD919685818A0420BD120680144E7
:10B63000581882421960DDD1106852685A6001447E
:10B640001960D7E702D90C232B60D3E720682118B3
:10B650008A4204BF11685268626004BF0918216001
:10B660005C60C7E738BD00BFF47C012070B5CD1C1D
:10B6700025F0030508350C2D38BF0C25002D064696
:10B6800001DBA94203D90C233360002070BD00F018
:10B69000B7FA214A1468214691B9204C23681BB996
:10B6A000304600F0B3F920602946304600F0AEF98C
:10B6B000431C24D10C233360304600F0A2FAE4E7A7
:10B6C0000B685B1B18D40B2B0FD90B60CD50CC181B
:10B6D000304600F096FA04F10B00231D20F007001D
:10B6E000C31AD3D05A42E250D0E78C424B6816BFFF
:10B6F000636013600C46EBE70C464968CCE7C41C5A
:10B7000024F00304A04205D0211A304600F07EF94F
:10B710000130CFD02560DBE7F47C0120F87C0120EC
:10B72000F8B5074614460E4621B91146BDE8F84063
:10B73000FFF79CBF22B9FFF74BFF25462846F8BD0F
:10B7400000F060FAA0420FD221463846FFF78EFF84
:10B7500005460028F2D031462246FEF785FF3146E5
:10B760003846FFF735FFE9E73546E7E72DE9F047CB
:10B770008E689E4282460C469046994637D88A8902
:10B7800012F4906F31D0256809696F1A6569022338
:10B7900005EB450595FBF3F509F101033B449D429B
:10B7A00038BF1D46530530D52946FFF75FFF0646D3
:10B7B00050B90C23CAF80030A38943F04003A38199
:10B7C0004FF0FF30BDE8F0873A462169FEF74CFFA5
:10B7D000A38923F4906343F08003A381266165610C
:10B7E0003E44ED1B2660A5604E464E4500D94E46B0
:10B7F000324641462068FEF742FFA3689B1BA360C8
:10B8000023681E4426600020DCE72A46FFF788FFF5
:10B8100006460028E2D121695046FFF7D9FEC8E765
:10B820002DE9F04F9DB0804603938B891D060C4691
:10B8300016460FD50B696BB94021FFF717FF206043
:10B84000206128B90C23C8F800304FF0FF30C7E062
:10B85000402363610023099320238DF8293030238E
:10B860008DF82A304FF0010B37463D4615F8013B65
:10B870000BB1252B3ED1B7EB060A0BD0534632460F
:10B8800021464046FFF772FF013000F0A480099B7B
:10B89000534409933B78002B00F09D8000234FF028
:10B8A000FF32CDE90523049307938DF853301A93A3
:10B8B0002F46052217F8011B4F48FFF739FE049B5E
:10B8C000D0B9D90644BF20228DF853201A0744BFAF
:10B8D0002B228DF853202A782A2A15D0079A2F4632
:10B8E00000200A25394611F8013B303B092B4DD980
:10B8F000B8B10FE02F46B8E73F4A801A0BFA00F0C4
:10B90000184304903D46D3E7039A111D1268039132
:10B91000002A01DB079204E0524243F0020307923F
:10B9200004933B782E2B0CD17B782A2B33D1039BAD
:10B930001A1D1B680392002BB8BF4FF0FF3302376C
:10B9400005932E4D397803222846FFF7F1FD38B1D3
:10B950004023401B03FA00F0049B03430137049388
:10B96000397827488DF8281006227E1CFFF7E0FD65
:10B97000002838D0234B13BB039B073323F0070366
:10B9800008330393099B4B4409936DE705FB02328F
:10B9900001200F46A6E700230137059319460A2523
:10B9A000384610F8012B303A092A03D9002BC8D0A9
:10B9B0000591C6E705FB012101230746F0E703AB2C
:10B9C00000932246104B04A94046AFF30080B0F12B
:10B9D000FF3F8146D6D1A3895B063FF536AF099874
:10B9E0001DB0BDE8F08F03AB00932246064B04A9BF
:10B9F0004046FFF719F8EAE708D500000ED5000029
:10BA000012D50000000000006DB7000038B5064CEC
:10BA1000002305460846236000F046F9431C02D186
:10BA2000236803B12B6038BD889001201F2938B5E9
:10BA300004460D4604D9162303604FF0FF3038BD8D
:10BA4000426C12B152F821304BB9204600F030F868
:10BA50002A4601462046BDE8384000F017B8012BC1
:10BA60000AD0591C03D1162303600120E7E7002404
:10BA700042F82540284698470020E0E7024B01465F
:10BA80001868FFF7D3BF00BF6000002038B5074C2F
:10BA90000023054608461146236000F0EDF8431CDC
:10BAA00002D1236803B12B6038BD00BF889001200C
:10BAB00000F0D2B810B50C46B1F90E1000F0AAF89B
:10BAC0000028ABBF636DA3891B1823F48053ACBF60
:10BAD0006365A38110BD2DE9F0411F468B89DB050D
:10BAE00005460C46164605D502230022B1F90E1074
:10BAF00000F074F8A389B4F90E1023F48053A381E5
:10BB000032463B462846BDE8F04100F023B810B568
:10BB10000C46B1F90E1000F061F8431CA38915BF63
:10BB2000606523F4805343F48053A38118BFA3813D
:10BB300010BDB1F90E1000F01FB849B1FF2A85BF42
:10BB40008A2303600A704FF0FF3098BF01207047CE
:10BB50000846704738B5074C05460846114600228E
:10BB600022601A4600F0AEF8431C02D1236803B1EC
:10BB70002B6038BD8890012038B5064C002305465F
:10BB80000846236000F058F8431C02D1236803B133
:10BB90002B6038BD8890012038B5074C002305463E
:10BBA00008461146236000F04FF8431C02D1236879
:10BBB00003B12B6038BD00BF8890012038B5064C1A
:10BBC000002305460846236000F04EF8431C02D1CE
:10BBD000236803B12B6038BD8890012038B5074C2D
:10BBE000054608461146002222601A4600F04CF82D
:10BBF000431C02D1236803B12B6038BD889001201B
:10BC00007047704751F8043C181F002BBCBF0B58FD
:10BC1000C018704738B5074C054608461146002243
:10BC200022601A4600F038F8431C02D1236803B1A1
:10BC30002B6038BD88900120024B58221A604FF0CB
:10BC4000FF30704788900120024B58221A604FF055
:10BC5000FF30704788900120024B58221A604FF045
:10BC6000FF30704788900120024B58221A60002054
:10BC7000704700BF88900120024B58221A604FF095
:10BC8000FF30704788900120024B58221A604FF015
:10BC9000FF30704788900120024B58221A604FF005
:10BCA000FF30704788900120044A05491368002B33
:10BCB00008BF0B461844106018467047FC7C0120F2
:10BCC00090900120024B58221A604FF0FF307047CD
:10BCD00088900120FEE700BFF8B500BFF8BC08BCA3
:10BCE0009E467047F8B500BFF8BC08BC9E4670473A
:10BCF000646174610000000084BD00001D03000049
:10BD00008DBD00000D04000095BD0000790B000002
:10BD10009CBD0000890C0000A1BD000019060000B8
:10BD2000A7BD000091070000B2BD0000770400002D
:10BD3000B7BD0000C50E0000C3BD00004F030000EA
:10BD4000CDBD0000590A0000DBBD00000D0B000056
:10BD5000E8BD00001D090000F4BD00005907000007
:10BD600072616E646F6D00616C6C006C6173740065
:10BD700066616C7365007472756500252E313573CC
:10BD80002E2E2E006D616B654C69737400616464C6
:10BD90004C6173740064656C657465006A6F696EEC
:10BDA0000073706C697400636F707946726F6D54C4
:10BDB0006F0066696E64006A6F696E537472696EB3
:10BDC000677300756E69636F6465417400756E69B1
:10BDD000636F6465537472696E67006E657742794C
:10BDE0007465417272617900617342797465417260
:10BDF00072617900667265654D656D6F72790000DC
:10BE000065BE00003D1300006ABE0000571300002D
:10BE100095BD00005B13000070BE000041130000E0
:10BE20007ABE00005F13000083BE000063130000B1
:10BE30008DBE00006713000098BE00006B13000069
:10BE4000A4BE000045130000ADBE00004F1300006B
:10BE5000B7BE000049130000C2BE0000531300002B
:10BE600066696C65006F70656E00636C6F7365006A
:10BE7000656E644F6646696C6500726561644C6905
:10BE80006E650072656164427974657300617070FB
:10BE9000656E644C696E6500617070656E644279B0
:10BEA0007465730066696C6553697A6500737461C3
:10BEB00072744C697374006E657874496E4C697362
:10BEC000740073797374656D496E666F00000000CD
:10BED000201700003017000044170000B8170000BA
:10BEE000EA1700001A1800004C1800006E18000035
:10BEF000AE180000E818000038190000761900009C
:10BF0000D6190000161A0000361A00006A1A00003E
:10BF1000AA1A0000CC1A0000F61A0000201B00002C
:10BF2000D0300000CC1B0000941C0000061D000057
:10BF3000501D0000B41D0000D01D0000EE1D0000CB
:10BF40002C1F00006C1F0000DE1F00000C200000F2
:10BF50003C2000006A200000CE20000032210000BA
:10BF600096210000FA2100006E220000E822000065
:10BF70004A230000AC230000E22300002624000036
:10BF80006C240000B2240000042500005A250000A3
:10BF9000982500000C2600004026000086260000A0
:10BFA000CC260000122700004C270000922700003A
:10BFB000D827000034290000F61A00006A1A000091
:10BFC0004C2800002017000080280000A628000050
:10BFD000DA280000002900002017000020170000C8
:10BFE0002017000020170000AA290000E629000001
:10BFF000262A0000762A00009C2A00000A2B000056
:10C00000542B0000842B0000201700002017000094
:10C01000A22B0000D42B0000062C00003A2C0000BC
:10C020005E2C0000BC2C0000E02C0000022D000063
:10C03000242D0000562D0000882D0000AC2D00009E
:10C04000D02D0000022E0000262E00002017000038
:10C050002017000020170000201700002017000004
:10C06000582E00007E2E0000A42E0000CA2E0000D4
:10C07000F02E0000242F0000582F00008C2F00000D
:10C08000C02F0000E62F00000C3000004030000000
:10C0900020170000201700002017000020170000C4
:10C0A00020170000201700002017000020170000B4
:10C0B00020170000201700002017000020170000A4
:10C0C000663000006630000044310000743100002A
:10C0D0005B2564206974656D206C6973745D00284C
:10C0E00025642062797465732900286F626A65632C
:10C0F0007420747970653A20256429005374616353
:10C100006B20756E646572666C6F7700626F6F6C22
:10C1100065616E006E756D62657200737472696E32
:10C1200067006C6973740062797465206172726172
:10C130007900000007000000030000009DC100001E
:10C140008D320000A5C1000039330000AEC10000EF
:10C1500087340000B7C1000091320000C0C1000068
:10C160008B340000C8C1000079340000D1C1000048
:10C17000C5330000000000000100000002000000C4
:10C1800003000000040000000A0000001D00000081
:10C190006D6963726F3A6269742076320068617308
:10C1A000546F6E6500706C6179546F6E65006861E4
:10C1B00073536572766F00736574536572766F00A2
:10C1C000646163496E697400646163577269746580
:10C1D000007371756172655761766500474320741D
:10C1E0006F6F6B2025642075736563733B206672E7
:10C1F000656520256420776F726473003C496E7416
:10C20000656765723E003C4C6973743E003C4F624A
:10C210006A6563743E003C4279746541727261796B
:10C220003E000D0A564D2050616E69633A20257319
:10C230000D0A006D697363006DC200003142000099
:10C2400076C20000B54100007AC200000141000042
:10C2500082C20000A34000008CC2000035400000F4
:10C2600098C20000373F00006E756C6C00686578FE
:10C27000546F496E740073696E006A736F6E476520
:10C2800074006A736F6E436F756E74006A736F6EBD
:10C2900056616C75654174006A736F6E4B657941C8
:10C2A0007400000030C300009142000038C3000059
:10C2B0009542000042C30000A74200004BC30000AB
:10C2C000AD42000056C30000B342000062C300004C
:10C2D000B942000070C30000BF42000078C30000F4
:10C2E000C54200007EC30000CB42000093C30000A3
:10C2F000D1420000A8C30000D7420000B4C3000030
:10C30000DD420000C4C30000E3420000D0C30000CF
:10C31000E9420000DDC30000EF420000ECC3000072
:10C320009B420000FFC30000A14200006E65740044
:10C33000686173576946690073746172745769461E
:10C34000690073746F70576946690077696669534D
:10C350007461747573006D794950416464726573DA
:10C3600073007374617274535349447363616E0054
:10C3700067657453534944006D794D4143006874B7
:10C380007470536572766572476574526571756530
:10C39000737400726573706F6E64546F4874747058
:10C3A000526571756573740068747470436F6E6E56
:10C3B00065637400687474704973436F6E6E65636F
:10C3C0007465640068747470526571756573740087
:10C3D00068747470526573706F6E73650077656210
:10C3E000536F636B65745374617274007765625345
:10C3F0006F636B65744C6173744576656E7400771A
:10C400006562536F636B657453656E64546F436C00
:10C4100069656E7400000000040000000300000065
:10C420000A000000070000000600000000000000F5
:10C430000008080800080A4A4000000A5FEA5FEAAC
:10C440000ED92ED36E19324489330C924C924D087A
:10C450000800000004880808040804848488000A8E
:10C46000448A4000048EC480000000048800000E4E
:10C47000C000000000080001224488100C925252B3
:10C480004C048C84848E1C824C901E1EC244924CA0
:10C4900006CA525FE21FF01EC13E02448ED12E1F1B
:10C4A000E24488100ED12ED12E0ED12EC488000861
:10C4B00000080000048004880244880482000EC042
:10C4C0000EC008048244880ED126C0040ED135B3B4
:10C4D0006C0C925ED2521C925C925C0ED010100ECC
:10C4E0001C9252525C1ED01C901E1ED01C90100E2E
:10C4F000D013712E12525ED2521C8808081C1FE203
:10C5000042524C1254981492101010101E113B7588
:10C51000B131113935B3710C9252524C1C925C906E
:10C52000100C92524C861C925C92510ED00C825C84
:10C530001FE4848484125252524C1131312A441126
:10C540003135BB7112524C9252112A4484841EC45C
:10C5500088101E0EC808080E10080482410EC24240
:10C56000424E048A400000000000001F08048000C2
:10C5700000000ED2524F10101C925C000ED0100E14
:10C5800002424ED24E0C925C900E06C81C88080ED9
:10C59000D24EC24C10101C925208000808080240EB
:10C5A00002424C10149814920808080806001B75E3
:10C5B000B131001C925252000C92524C001C925C01
:10C5C00090000ED24EC2000ED010100006C8049883
:10C5D00008080EC807001252524F0011312A4400B9
:10C5E000113135BB00124C8C9200112A4498001E68
:10C5F000C4881E06C48C8486080808080818080C1D
:10C60000881800000C83600000000000010000009A
:10C61000020000000300000004000000050000000C
:10C6200006000000070000000800000009000000EC
:10C630000A0000000B0000000C0000000D000000CC
:10C640000E0000000F0000001000000012000000AB
:10C650001400000016000000180000001A0000007E
:10C660001C0000001E00000020000000230000004D
:10C6700026000000290000002C0000002F00000010
:10C6800032000000360000003A0000003E000000CA
:10C6900042000000460000004B0000005000000077
:10C6A000550000005A000000610000006800000012
:10C6B0006F000000760000007D0000008400000094
:10C6C0008B0000009200000099000000A000000014
:10C6D000A7000000AE000000B5000000BC00000094
:10C6E000C3000000CA000000D1000000D800000014
:10C6F000DF000000E6000000ED000000F400000094
:10C70000FB000000FF00000000000000020000002D
:10C7100004000000010000000300000080C70000CA
:10C72000094300008BC700007947000095C700004F
:10C73000C5430000A2C70000E5450000A9C70000EE
:10C7400031460000B2C7000081460000BEC70000AD
:10C7500075450000CFC7000019440000DCC7000089
:10C76000FD44000015000000160000001700000046
:10C770001800000019000000646973706C61790092
:10C780006C696768744C6576656C006D62446973AA
:10C79000706C6179006D62446973706C61794F6689
:10C7A00066006D62506C6F74006D62556E706C6FD8
:10C7B00074006D62447261775368617065006D62E8
:10C7C0005368617065466F724C6574746572006E73
:10C7D000656F506978656C53656E64006E656F5067
:10C7E0006978656C53657450696E004E6F7420658E
:10C7F0006E6F75676820726F6F6D206576656E204D
:10C80000616674657220636F6D70616374696F6EC9
:10C8100000436F6D70616374656420466C6173687A
:10C8200020636F64652073746F72650A25642062EB
:10C83000797465732075736564202825642525291E
:10C84000206F6620256400426164207265636F7208
:10C850006420666F756E6420647572696E67206906
:10C860006E697469616C697A6174696F6E002564C0
:10C870002025642025642028256420776F72647346
:10C8800029002564207265636F7264732C2025640F
:10C8900020776F7264732C206D6178494420256481
:10C8A0002C20636F6D70616374696F6E20637963B0
:10C8B0006C657320256400526573746F7265642023
:10C8C00025642073637269707473005374617274A9
:10C8D000656400726164696F000000006CC900004B
:10C8E0006550000079C90000D952000089C90000D4
:10C8F0006D52000097C9000039540000A2C9000021
:10C900008D500000B2C900001D510000C6C90000D2
:10C9100001510000D5C9000015560000E1C9000012
:10C9200091550000EAC9000035550000F5C9000026
:10C930008554000000CA0000BD54000009CA000070
:10C94000ED54000012CA00009D50000021CA0000F2
:10C950007D5000002ACA0000AD5000006E6F6E6569
:10C96000006F746865720070616972006469736158
:10C97000626C65526164696F006D657373616765B0
:10C980005265636569766564007061636B657452B6
:10C99000656365697665007061636B657453656E88
:10C9A00064007265636569766564496E7465676580
:10C9B000720072656365697665644D65737361675E
:10C9C0006554797065007265636569766564537452
:10C9D00072696E670073656E64496E74656765722F
:10C9E0000073656E64506169720073656E645374A0
:10C9F00072696E67007365744368616E6E656C0082
:10CA000073657447726F757000736574506F7765E6
:10CA100072007369676E616C537472656E677468D7
:10CA2000006465766963654944006C6173744D65A3
:10CA30007373616765494400556E6B6E6F776E2046
:10CA40007072696D6974697665205B25733A257328
:10CA50005D00000000000000963007772C610EEEAC
:10CA6000BA51099919C46D078FF46A7035A563E945
:10CA7000A395649E3288DB0EA4B8DC791EE9D5E06C
:10CA800088D9D2972B4CB609BD7CB17E072DB8E76B
:10CA9000911DBF906410B71DF220B06A4871B9F3C0
:10CAA000DE41BE847DD4DA1AEBE4DD6D51B5D4F4F9
:10CAB000C785D38356986C13C0A86B647AF962FD5E
:10CAC000ECC9658A4F5C0114D96C0663633D0FFAAB
:10CAD000F50D088DC8206E3B5E10694CE44160D5B1
:10CAE000727167A2D1E4033C47D4044BFD850DD29B
:10CAF0006BB50AA5FAA8B5356C98B242D6C9BBDBAE
:10CB000040F9BCACE36CD832755CDF45CF0DD6DCA8
:10CB1000593DD1ABAC30D9263A00DE518051D7C84F
:10CB20001661D0BFB5F4B42123C4B3569995BACFDA
:10CB30000FA5BDB89EB802280888055FB2D90CC6FB
:10CB400024E90BB1877C6F2F114C6858AB1D61C174
:10CB50003D2D66B69041DC760671DB01BC20D29893
:10CB60002A10D5EF8985B1711FB5B606A5E4BF9F20
:10CB700033D4B8E8A2C9077834F9000F8EA8099613
:10CB800018980EE1BB0D6A7F2D3D6D08976C64917E
:10CB9000015C63E6F4516B6B62616C1CD830658597
:10CBA0004E0062F2ED95066C7BA5011BC1F4088274
:10CBB00057C40FF5C6D9B06550E9B712EAB8BE8BB5
:10CBC0007C88B9FCDF1DDD62492DDA15F37CD38C3E
:10CBD000654CD4FB5861B24DCE51B53A7400BCA33C
:10CBE000E230BBD441A5DF4AD795D83D6DC4D1A46E
:10CBF000FBF4D6D36AE96943FCD96E34468867AD45
:10CC0000D0B860DA732D0444E51D03335F4C0AAAE3
:10CC1000C97C0DDD3C710550AA41022710100BBEE6
:10CC200086200CC925B56857B3856F2009D466B92D
:10CC30009FE461CE0EF9DE5E98C9D9292298D0B062
:10CC4000B4A8D7C7173DB359810DB42E3B5CBDB70F
:10CC5000AD6CBAC02083B8EDB6B3BF9A0CE2B60390
:10CC60009AD2B1743947D5EAAF77D29D1526DB0445
:10CC70008316DC73120B63E3843B64943E6A6D0D90
:10CC8000A85A6A7A0BCF0EE49DFF099327AE000ADB
:10CC9000B19E077D44930FF0D2A3088768F2011E6E
:10CCA000FEC206695D5762F7CB67658071366C1905
:10CCB000E7066B6E761BD4FEE02BD3895A7ADA1026
:10CCC000CC4ADD676FDFB9F9F9EFBE8E43BEB71707
:10CCD000D58EB060E8A3D6D67E93D1A1C4C2D83891
:10CCE00052F2DF4FF167BBD16757BCA6DD06B53FF7
:10CCF0004B36B248DA2B0DD84C1B0AAFF64A033636
:10CD0000607A0441C3EF60DF55DF67A8EF8E6E31B4
:10CD100079BE69468CB361CB1A8366BCA0D26F25FD
:10CD200036E2685295770CCC03470BBBB91602224A
:10CD30002F260555BE3BBAC5280BBDB2925AB42B5F
:10CD4000046AB35CA7FFD7C231CFD0B58B9ED92C74
:10CD50001DAEDE5BB0C2649B26F263EC9CA36A75D9
:10CD60000A936D02A906099C3F360EEB8567077290
:10CD700013570005824ABF95147AB8E2AE2BB17BF7
:10CD8000381BB60C9B8ED2920DBED5E5B7EFDC7C7E
:10CD900021DFDB0BD4D2D38642E2D4F1F8B3DD68D5
:10CDA0006E83DA1FCD16BE815B26B9F6E177B06FD0
:10CDB0007747B718E65A0888706A0FFFCA3B0666BD
:10CDC0005C0B0111FF9E658F69AE62F8D3FF6B614A
:10CDD00045CF6C1678E20AA0EED20DD75483044EEC
:10CDE000C2B30339612667A7F71660D04D4769497A
:10CDF000DB776E3E4A6AD1AEDC5AD6D9660BDF408D
:10CE0000F03BD83753AEBCA9C59EBBDE7FCFB2473F
:10CE1000E9FFB5301CF2BDBD8AC2BACA3093B35324
:10CE2000A6A3B4240536D0BA9306D7CD2957DE542D
:10CE3000BF67D9232E7A66B3B84A61C4021B685D06
:10CE4000942B6F2A37BE0BB4A18E0CC31BDF055A7F
:10CE50008DEF022D416C6C207461736B73207374C1
:10CE60006F707065640076313230002025732025A4
:10CE700073004D656D6F727920636C6561726564D6
:10CE8000004E6F2066726565207461736B20656E5D
:10CE9000747269657300000008CF00000D6E000019
:10CEA00015CF00003166000021CF0000DD6D0000CD
:10CEB00027CF0000ED6D00002DCF0000FD6D0000BC
:10CEC00033CF0000B56C000049CF00006166000060
:10CED00053CF0000656E00005BCF0000996A000030
:10CEE00064CF00005968000070CF0000696700003F
:10CEF00079CF0000B167000081CF0000C969000050
:10CF000073656E736F727300616363656C657261E4
:10CF100074696F6E0074656D7065726174757265A9
:10CF20000074696C74580074696C74590074696C8D
:10CF3000745A00736574416363656C65726F6D65E7
:10CF400074657252616E676500746F7563685265CF
:10CF500061640069326352656164006932635772CB
:10CF60006974650073706945786368616E67650010
:10CF700073706953657475700072656164444854D8
:10CF8000006D6963726F70686F6E650065BE00004A
:10CF9000757000006ABE00001D710000BBCF00006C
:10CFA00041710000C0CF0000F96F0000C9CF000040
:10CFB000C171000073657269616C00726561640023
:10CFC00072656164496E746F007772697465000000
:10CFD0004CD00000557200005AD00000657200006D
:10CFE00067D000005972000070D000006972000024
:10CFF0007AD000006D72000083D0000071720000D2
:10D0000088D00000757200008DD000007972000099
:10D0100099D000007D720000A0D000008172000055
:10D02000A9D0000085720000AED000008972000017
:10D03000B9D000008D720000C3D000005D72000006
:10D04000CDD000006172000074667400656E61628C
:10D050006C65446973706C617900736574426163D7
:10D060006B6C6967687400676574576964746800FD
:10D07000676574486569676874007365745069789A
:10D08000656C006C696E65007265637400726F7523
:10D090006E6465645265637400636972636C6500F5
:10D0A000747269616E676C6500746578740074668B
:10D0B00074546F756368656400746674546F756347
:10D0C000685800746674546F7563685900746674A8
:10D0D000546F75636850726573737572650076611D
:10D0E0007273000004D10000F57600000ED100003C
:10D0F000D576000017D10000B176000023D10000E2
:10D1000041760000766172457869737473007661C8
:10D11000724E616D6564007365745661724E616D27
:10D120006564007661724E616D65466F72496E642A
:10D1300065780057656C636F6D6520746F204D696D
:10D1400063726F426C6F636B732100705F73706901
:10D1500020213D204E554C4C002F686F6D652F6788
:10D1600069742F2E706C6174666F726D696F2F70A9
:10D1700061636B616765732F6672616D65776F724E
:10D180006B2D61726475696E6F6E6F726469636E28
:10D190007266352F6C69627261726965732F5350C4
:10D1A000492F5350492E63707000535049436C61AE
:10D1B00073733A3A535049436C617373284E524625
:10D1C0005F5350495F547970652A2C2075696E74DD
:10D1D000385F742C2075696E74385F742C20756903
:10D1E0006E74385F74290000000000000000000029
:10D1F000C978000081780000B7780000BD78000091
:10D20000C3780000B57800000200000003000000B1
:10D21000040000001F0000001C0000000E000000C1
:10D22000250000000B0000000A00000009000000BB
:10D230001E000000170000000C000000110000009C
:10D24000010000000D00000022000000FFFFFFFFB2
:10D25000FFFFFFFF1A000000200000001500000083
:10D26000160000000F00000018000000130000006E
:10D270002400000000000000140000000500000071
:10D280001000000008000000190000002800000045
:10D29000060000000000000000000000AB7E00005F
:10D2A000A1850000217F00002D7F0000277F000066
:10D2B000A97E0000A17E0000357F0000C57E000031
:10D2C0009D7E000000C0014000100240002002408E
:10D2D00000D00240000000000000000000003043C9
:10D2E00000000000000030C3737172740000000081
:10D2F000FB21F93FFB2109407CD91240FB21194059
:10D300007A6A1F407CD92240BBFD2540FB21294081
:10D310003A462C407A6A2F405C4731407CD93240F3
:10D320009C6B3440BBFD3540DB8F3740FB213940DF
:10D330001BB43A403A463C405AD83D407A6A3F4096
:10D340004C7E40405C4741406C1042407CD942409A
:10D350008CA243409C6B4440AC344540BBFD4540EF
:10D36000CBC64640DB8F4740EB584840FB21494045
:10D3700083F9A200444E6E00FC291500D157270006
:10D38000DD34F50062DBC0003C999500419043001C
:10D390006351FE00BBDEAB00B761C5003A6E2400EE
:10D3A000D24D42004906E00009EA2E001C92D1004D
:10D3B000EB1DFE0029B11C00E83EA700F5358200F8
:10D3C00044BB2E009CE98400B4267000417E5F00BF
:10D3D000D6913900538339009CF439008B5F840067
:10D3E00028F9BD00F81F3B00DEFF97000F980500ED
:10D3F000112FEF000A5A8B006D1F6D00CF7E360093
:10D4000009CB2700464FB7009E663F002DEA5F001C
:10D41000BA277500E5EBC7003D7BF100F73907003F
:10D4200092528A00FB6BEA001FB15F00085D8D001D
:10D43000300356007BFC4600F0AB6B0020BCCF00F5
:10D4400036F49A00E3A91D005E619100081BE60016
:10D4500085996500A0145F008D40680080D8FF00AA
:10D4600027734D0006063100CA561500C9A873007F
:10D470007BE260006B8CC00000000040FB21F93FA4
:10D48000000000002D44743E000000809846F83CE7
:10D490000000006051CC783B00000080831BF03915
:10D4A0000000004020257A38000000802282E33608
:10D4B000000000001DF369350200000003000000B9
:10D4C00004000000060000002C2066756E6374697D
:10D4D0006F6E3A2000617373657274696F6E2022FB
:10D4E000257322206661696C65643A2066696C6503
:10D4F00020222573222C206C696E652025642573FB
:10D5000025730A0064000020232D302B2000686C56
:10D510004C00656667454647003031323334353656
:10D52000373839414243444546003031323334358F
:10D5300036373839616263646566000000000000B8
:10D5400000000000000000000000000000000000DB
:10D5500000000000000000000000000000000000CB
:10D5600000000000000000000000000000000000BB
:10D5700000000000000000000000000000000000AB
:10D58000000000000000000000000000000000009B
:10D59000000000000000000000000000504F534950
:10D5A0005800002020202020202020202828282863
:10D5B0002820202020202020202020202020202063
:10D5C00020202088101010101010101010101010B3
:10D5D00010101004040404040404040404101010C3
:10D5E000101010104141414141410101010101016F
:10D5F00001010101010101010101010101011010FD
:10D600001010101042424242424202020202020242
:10D6100002020202020202020202020202021010CE
:10D6200010102000000000000000000000000000BA
:10D6300000000000000000000000000000000000EA
:10D6400000000000000000000000000000000000DA
:10D6500000000000000000000000000000000000CA
:10D6600000000000000000000000000000000000BA
:10D6700000000000000000000000000000000000AA
:10D68000000000000000000000000000000000009A
:10D69000000000000000000000000000000000008A
:08D6A000000000000000000082
:08D6A800982BFF7F0100000038
:10D6B000FFFFFFFFE803000001000000E803DC05B6
:10D6C000DC05DC05DC050000FFFFFFFFFFFFFFFFBF
:10D6D0001800000019FCFFFFFFFFFFFF0200000021
:10D6E00040420F00FF000000030000000090D00344
:10D6F000FFFFFFFFFFFFFFFFFFFFFFFFFFFFFFFF3A
:10D700000A00000001000000080000000100000005
:10D7100064000020000000005CD500007CD5000003
:10D720003CD50000000000000000000000000000E8
:10D7300000000000000000000000000000000000E9
:10D7400000000000000000000000000000000000D9
:10D7500000000000000000000000000000000000C9
:10D7600000000000000000000000000000000000B9
:10D770000000000043000000000000000000000066
:10D780000000000000000000000000000000000099
:10D790000000000043000000000000000000000046
:10D7A0000000000000000000000000000000000079
:10D7B0000000000043000000000000000000000026
:10D7C0000000000000000000000000000000000059
:10D7D0000000000043000000000000000000000006
:10D7E0000000000000000000000000000000000039
:10D7F00000000000430000000000000000000000E6
:10D800000000000000000000000000000000000018
:10D8100000000000430000000000000000000000C5
:10D8200000000000000000000000000000000000F8
:10D8300000000000430000000000000000000000A5
:10D8400000000000000000000000000000000000D8
:10D85000000000003BBB000009B500000000000014
:10D86000A2D5000082BD000032C2000032C200001A
:10D8700032C2000032C2000032C2000032C20000D8
:10D8800032C2000032C2000032C20000FFFFFFFFC0
:10D89000FFFFFFFFFFFFFFFFFFFF000001004153FD
:10D8A00043494900000000000000000000000000A3
:10D8B00000000000000000000000000000004153D4
:10D8C0004349490000000000000000000000000083
:10D8D0000000000000000000000000000000000048
:10D8E000250200004D780000A97C00003581000071
:04D8F0000102000031
:0400000300007D6517
:00000001FF
